:020000040800F2
:100000000050002021530108C1530108093D010897
:10001000C1530108C1530108C15301080000000089
:10002000000000000000000000000000C1530108B3
:10003000C153010800000000C15301082322010838
:10004000C1530108C1530108C1530108C15301083C
:10005000C1530108C153010825A8000821A80008C0
:10006000C1530108C1530108C1530108C15301081C
:10007000C1530108C1530108A9B10008C1530108C7
:10008000CDE80008C1530108C1530108C15301085C
:10009000C1530108C1530108C15301081DA800083C
:1000A000C1530108D9C00008C1530108E9C00008C4
:1000B000C9C00008B9C00008A9C0000881610008D3
:1000C00085610008796100087D610008C15301085D
:1000D000C1530108A1B1000899B1000891B100080D
:1000E00031220108C1530108C1530108000000007A
:1000F0000000000000000000000000000000000000
:0C01000000000000000000005FF808F1A3
:100110002DE9F04F764B774EA3B033600023736028
:1001200010F08AFC18B910F0A9FC08F02BFE08F0BA
:10013000CBFE714A714C1378714D43F0010313707B
:1001400000230A930B930C934FF4E0130D93236851
:10015000A87B43F480332360A36943F01003A361B9
:10016000236803F400330B930A9B01330A930B9B20
:100170001BB90A9BB3F5A06FF2D123685F4913F452
:10018000003301D0022315E00A6842F001020A6040
:100190000A93236803F002030B930A9B01330A932B
:1001A0000B9B1BB90A9BB3F5A06FF2D123689A078A
:1001B00039D501230C93534B53491A6842F010026E
:1001C0001A601A6822F003021A601A6842F00202EA
:1001D0001A606368636063686360636843F48063A4
:1001E00063604A4B1A68043B22F070425A60484AE6
:1001F0001160616821F47C116160596841F000412F
:100200005960D96821F40041D9609B681B0449BF3B
:10021000404B4FF4E01313604FF480130D930C9B8D
:10022000012B01D117E0FEE7022B18D168B10D9B1D
:10023000B3F5801F02D14FF4A01305E00D9BB3F579
:10024000E01F02D14FF400130D930D9963680B4327
:1002500043F4803302E0636843F46013636023680F
:1002600043F0807323602168244B8F01FBD55968CC
:1002700021F003015960596841F002015960636837
:100280001E4903F00C03082BF9D14B68DFF890806E
:1002900003F00C03042B03D0082B03D01A4B12E0FD
:1002A000136810E04B684868C3F38343C00303F14D
:1002B000020301D4184905E0496811F4003F1168B0
:1002C00018BF49084B43C8F800306368134FC3F3A5
:1002D00003133B44197ED8F800300697CB40C8F88A
:1002E00000301368084A93421CD101221EE000BF6F
:1002F0005B850008D8000020B833002000100240C1
:10030000F02900200020024000127A000410014071
:100310002C000020001BB70000093D00B09B010825
:1003200060000020A94A934202D10222A84B1A7011
:10033000DFF800B3A74BDFF8C492CBF80C30A36909
:100340004FF0000A43F00103A361636AA248B3605F
:10035000636A43F080736362A36943F01C03A36183
:1003600022AB04934FF6FF73049A8DF85EA022F837
:100370002C3D114604920EF0B4FB484604990EF051
:10038000B0FB049995480EF0ACFB954A049853686D
:1003900043F0007353600DF09BFE924A179B514649
:1003A000B3FBF2F3904A914813600C2217F01BF94B
:1003B000D8F800304FF47A72B3FBF2F38C4A013B69
:1003C0005360F0238BF823300723C2F808A0136092
:1003D000AB68DFF86482049FDFF860B2C8F80030D1
:1003E0009BE80F0087E80F00A369179843F0080304
:1003F000A361A36918A943F00803A3610823C9F8FE
:1004000010301023C9F810300EF06BFB19981AA9A0
:100410000EF067FBD8F80030DFF824A21B0751D597
:100420009AF89231012B4DD8049BDBF81000194645
:10043000186048469AF893A10EF053FB0A2011F079
:10044000DBFED9F8083003F020039BB2002B39D132
:10045000684A9268D70040F11A86D80732D5664BB1
:10046000DFF898A11868DFF870914FF0100BCAF808
:1004700014B00499179048460EF033FB0823C9F8CE
:1004800010303C2011F0C3FECAF810B04FF0000B42
:1004900095F893319B4515DA584B4FF0080AC3F88D
:1004A00010A078200593C9F814A011F0A5FE059BB3
:1004B0007820C3F814A0C9F810A011F09DFE0BF12C
:1004C000010BE5E7642011F0A2FEA0224C480021B8
:1004D00017F089F8E369002243F00703E361A36999
:1004E00043F4006343F00C03A361424B4FF0000957
:1004F00003F10C0102F8019001320E2AF5D1FF221E
:100500009A76DA761A775A773E4B3F4A49461A600E
:100510003E483C22D8F8004017F065F84946C4F33D
:10052000801805233A4ADFF8E4E0885C0C224A434D
:1005300002F80E00B8F1000F08D11E3801289FBF45
:10054000FF2003F1FF3302F80E00DBB20131052971
:10055000E8D1304A95F805B013702F4B2F4983F836
:1005600000B02F4B234A3362C0330B602D4BA106E2
:1005700003EBCB035B7848BF01235362002340F2B7
:10058000DC51294A22F813100133082BF7D110A8A7
:1005900000211C2217F027F814F4007A04F40069F3
:1005A00050D0A3040BD4B9F1000F0AD01F4B95F81B
:1005B0008611A3F10C02012908BF134602E01C4B6F
:1005C00000E01A4B0593049B16933DE0001BB70017
:1005D000E33300200005FA05000801400010014047
:1005E0000000014040420F00E0270020BC12002024
:1005F00010E000E0D8000020EC9B0108000C014056
:100600002828002004130020E02B002008130020DD
:10061000C7C601083D100020B8080020442900206A
:10062000042A00207CC40108A80F0020BC9B0108FC
:10063000B09B010800ED00E090290020D89B010844
:10064000F0290020CDF814A0BBF10E0F03D00BF061
:10065000EF03082B02D101238DF85230012011F055
:10066000B3FC18B14088003018BF0120C4F3400328
:100670008DF84630C4F3403300F001008DF840306F
:10068000C4F3C0338DF845008DF848808DF84330B1
:10069000B9F1000F07D095F8869109F1FF37D7F12E
:1006A000000949EB0709C4F300438DF84930736A28
:1006B0001AF1000A18BF4FF0010A003318BF0123D6
:1006C0008DF84B30C4F30053B5F848018DF84C3029
:1006D000B5F84A31ADF85600ADF85030E004B5F841
:1006E000563148BFB848ADF84E30C4F3804348BFD8
:1006F000B0F850018DF84730B5F8543148BFADF827
:100700005600B3F5FA7FADF8543084BF0023ADF83E
:10071000563095F8D631AD4886F82830002386F853
:10072000293043709DF8523004F00101002BC4F3CE
:10073000C0028DF844908DF841108DF842208DF85C
:100740004AA00CBF0023022301B902B10133069A6B
:100750004FF0000802EB83073B6CA3F102091A3348
:1007600006934FF6FF7339F8022F9A4200F08B81FF
:100770009DF84510D3B2120AD5B219B1991E0129BC
:1007800040F27D819DF8481031B1914819014058DF
:100790009049884200F073819DF8497037B18C48C8
:1007A000190140588B49884200F069819DF8461034
:1007B00051B18748884C00EB03104168A14203D136
:1007C0000189102900F05B819DF8431051B18048E8
:1007D000814C00EB03104168A14203D10189022939
:1007E00000F04D819DF8441051B179487B4C00EBED
:1007F00003104168A14203D10189022900F03F8121
:10080000169E7EB1724C316804EB03146068884216
:1008100008D12189B088884200F03181F08888426F
:1008200000F02D81022A02D19DF8402003E0012A28
:1008300004D19DF84120002A00F021819DF84B2031
:10084000634C1E015AB19DF8522042B9A3F108022F
:10085000012A04D8A25962498A4208BF04259DF89A
:100860004C20344452B19DF852203AB917B10C3B98
:10087000012B01E0043B032B40F2E980012D47D11D
:10088000584FFF2387F8703087F87130504B4FF086
:10089000000A9A19517B506802F1080B12898DF8F1
:1008A0005E10ADF85C2017A9022287F874A0C7F883
:1008B000804007938DF85F2087F82CA0C7F830A000
:1008C000C7F834A0C7F838A0C7F86CA087F872A0A2
:1008D00087F873A00EF005F9079B9BF80210985952
:1008E000524609F0ECFD204651462A460AF0ACFB80
:1008F0003D4BC7F88CA0C7F884303C4B2046C7F866
:10090000883007F1840107F188020AF0E5FBB6E0C0
:10091000022D49D15FFA88F31C2101FB03FC2C4A0C
:10092000304B911903EB0C0A91F80DE001F108032B
:100930004868098900274FF0010B8AF87580ADF8E7
:100940005C108AF8767017A98AF87E708AF874B0FD
:10095000CAF88040CDF824C08DF85EE00892079375
:100960008DF85F500EF0BDF8079B089A9978905962
:100970003A4609F0A4FD204639465A460AF064FB7F
:100980001B4A184BDDF824C0CAF884209C44194A3D
:100990000CF18401CAF88820CAF88C7020460A1D20
:1009A0000AF09AFBD8446AE0032D4ED19DF84730F7
:1009B0000C4D114E13B395F82A70204608214FF6BE
:1009C000FF72002335E000BFF02900200101002064
:1009D000CCBE01080004004000080140000C0140AA
:1009E000002C0140D80000202D9F00080DA0000819
:1009F000F9A40008039F0008F4270020BDF8542044
:100A000095F82A70B2F5FA7FBDF856300BD98549B2
:100A10002046B1FBF2F2082192B209F0A5FD824B0B
:100A200046F827000AE081492046B1FBF2F2012195
:100A300092B209F099FD7E4B46F82700C36095F805
:100A40002A30013385F82A3019E0042D17D1BDF87A
:100A50004E20764B774D93FBF2F22046BDF8503096
:100A6000012192B295F8296009F07EFD95F82930B0
:100A700005EB86060133C6F8540185F82930069B3C
:100A800099457FF46EAE6B4D6B4B95F82920002491
:100A900085F87421694A1C7016789846A6F11702E9
:100AA000022A19D82B6A0021185903EB040913F004
:100AB000E7FB10B16B6A5BBB25E0614F99E80F0063
:100AC000274487E80F0098F8003010340133C02C19
:100AD00088F80030E6D1EDE75A4B13F836E003EB27
:100AE000C603D3F804C088F800E0BCF1000FE1D0E1
:100AF0007445DFDA524F23011F4463440FCB0134A6
:100B000087E80F00F4E7504F3B68DA0424D41DE077
:100B10004E4B4F4A13F8360003EBC6035C68107067
:100B2000002CF0D000238342EDDAC3EBC30162183E
:100B3000D2F800C0DFF840E1013341F80EC001EB0C
:100B40000E079188B9809279BA71ECE706F0EF034D
:100B5000082B404B25D126E098F80030012BF5D921
:100B60003D4C04EB031303F1100810344445EDD061
:100B700054F8100C4FF07C5113F0EEF94FF07C510B
:100B800044F8100C54F8140C13F0E6F94FF07C51B3
:100B900044F8140C54F80C0C13F0DEF944F80C0C67
:100BA000E3E70E2E08D11A78182E42F010021A70C0
:100BB00008D111F0B3FD05E01A78192E22F01002C9
:100BC0001A70F5E711F08EFD3B68244C5B035EBFA5
:100BD000234B01221A70234B23481A78994642F07E
:100BE00004021A70214A11789046022934BF142356
:100BF00010238DF85E304FF002038DF85F30A3694B
:100C00004FF4805243F00403ADF85C2038BF002657
:100C1000A36128BF012617A90DF063FF144B6EB323
:100C2000144A2CE000127A002DA0000840420F0068
:100C30001DA00008D800002024280020B8080020AB
:100C4000F40700207CC4010890290020B8AD0108F9
:100C5000D0280020A4100020FC0700200010024033
:100C6000200D0020B833002000080140E3330020AD
:100C7000C8330020A11F0108D1280020724A00209B
:100C80001A6011F0E3FA714B714E93E80300049B74
:100C90004FF0030B83E80300A369179843F00803A0
:100CA000A36118A90DF01DFFE369304643F48043AA
:100CB000E3612369049943F48043236118238DF889
:100CC0005E304FF42043ADF85C308DF85FB00DF02E
:100CD00008FF04224FF48043304604998DF85E20CB
:100CE00006924FF4805AADF85C300DF0FAFE1023F6
:100CF000304604998DF85E30ADF85CA00DF0F1FE41
:100D00002369322043F480432361236923F4804321
:100D10002361504B198801F4415141F4457141EA76
:100D20000B011980998B21F400610904090C998346
:100D300007211982198889B241F0400119809F2347
:100D4000C6F810A08DF83C3000238DF83D308DF8AA
:100D50003E308DF83F3011F05AFA069AC6F814A0CA
:100D600004980FA912F006F9C6F810A09DF85E309D
:100D70009DF85D201B0243EA02439DF85F20134368
:100D8000354A934215D0322011F041FAC6F814A02A
:100D9000F52012F025F9FF2012F022F97028C6F88C
:100DA00010A006D198F80030022B04BF2B4B83F81B
:100DB00000B098F80030032B0CBF1F20022007F072
:100DC000D2FA98F80030032B03D001200EF0DAF8A5
:100DD00007E0022011F0F8F80028F6D04388002B35
:100DE000F3D03E684FF0100B06F40043049306F472
:100DF000006306931A4B002118465A46079398F849
:100E0000008016F0F0FB4FF6FF72079BADF83C2018
:100E100002224FF0000A16EA02018DF83E208DF8FA
:100E20003FA01E4620D022A921F84CBD0D480DF050
:100E3000FBFA042333700722012386F801A0B37064
:100E4000F2709A4611E000BFB51F0108009C01082E
:100E5000000C01400038004015202000E333002042
:100E6000B8230020000801408A46B8F1010F12D9CA
:100E7000202222A921F84C2D89480DF0D5FA05220F
:100E800001233272B3720AF10102072386F809A026
:100E9000F3725FFA82FA049B8BB122A9022221F835
:100EA0004C2D7F480DF0C0FA01220AEB0201072306
:100EB00086F805A03271B271F3715FFA81FA069B70
:100EC00093B1022222A921F84C2D76480DF0ACFAFC
:100ED000092201233273B3730AF10102072386F852
:100EE0000DA0F3735FFA82FA62686F4842F44042E1
:100EF00062606269DFF8B08142F001026261A2695A
:100F000042F40072A2610DF06BF8684A0024179257
:100F1000674ABAF1010F189294BF224680221C92B0
:100F20004FF480721D924FF480621E922022404640
:100F30001F9217A94FF4005220921994CDF868A07F
:100F40001B94219408F05EFFD8F80020594942F024
:100F50000102C8F800204A68BAF1010F22F4702299
:100F600094BF0020012022F4807242EA00224A60ED
:100F70008868514A0AF1FF33024042F4602242F08D
:100F800002028A60CA6ADBB222F4700242EA0353A8
:100F9000CB62012332199178002963D0305D591C4E
:100FA0000928C9B2D278DFF80CC112D9A0F10A0E13
:100FB000DCF80CA00EEB4E0E4FF0070808FA0EF806
:100FC0002AEA080802FA0EF248EA0202CCF80C20DB
:100FD0000FE0DCF8108000EB400A4FF0070E0EFA2D
:100FE0000AFE28EA0E0E02FA0AF24EEA0202CCF8D3
:100FF0001020062BDFF8BCE010D8013BDEF83420CF
:1010000003EB83034FF01F0C0CFA03FC22EA0C02E3
:1010100000FA03F31343CEF8343022E00C2B10D83F
:10102000073BDEF8302003EB83034FF01F0C0CFA74
:1010300003FC22EA0C0200FA03F31343CEF830302B
:101040000FE0A3F10D02DEF82C8002EB82021F23D9
:10105000934028EA030C00FA02F34CEA0303CEF8AB
:101060002C300B460434102C94D1124B9A6842F465
:1010700080729A609A6842F001029A609A6842F01F
:1010800008029A6099680B4A0C0717D5FAE70AF12B
:10109000FF33092B8CBF00230123FFF7DEB900BF0C
:1010A00000080140000C0140080002404C240140AF
:1010B000C823002000240140FDF7F1FF936843F0AE
:1010C00004039360C14B9E6816F00406FAD1C04C2D
:1010D0009A68B4F85C0142F4A0029A60002840F0DB
:1010E0000286B4F95E31002B40F0FD85B4F9603121
:1010F000002B40F0F8853B6898031FD5C82011F0FD
:1011000086F8AE200DF0A9FE08B10DF0ABFE85F813
:101110007501C82011F07BF8AE4B0021C5F878317D
:10112000AD4D0C22284616F05EFA0223EB700CF04F
:10113000B6F911F047F8A94B0344AB60A84D94F8F9
:101140006CC12B68B4F86401B3F956E094F86311EC
:1011500094F86B21CDF800E0B4F80CE06346CDF8CC
:1011600004E094F80FE0CDF808E008F063F910B956
:10117000032011F0BFF899F80030102243F0020369
:1011800089F80030974B4FF00A085A6108221A611B
:10119000DFF850921920D9F80C3008F1FF3883F0AD
:1011A0001003C9F80C30D9F80C3083F00803C9F8E3
:1011B0000C3011F02CF8012011F048F8192011F032
:1011C00026F8002011F042F818F0FF08E0D10823BB
:1011D000C9F810304FF0100A834BC9F810A01A68F4
:1011E000984612F0080F09D0804BC9F814A01B686C
:1011F00098477F4B0122C9F810A01A707D4BDFF889
:101200001C921B68187B12F053FE7B4912F0A4FE5F
:1012100007F08CFC8246B9F8000012F049FE5146F6
:1012200012F09AFE16F0ECFB744B1880B9F800002F
:1012300012F03EFE0146724812F042FF714912F070
:101240003FFF714B6C491860704B186912F084FEB7
:101250006F4912F081FE6F4BFF2118606E4B1A220E
:10126000184616F0C0F9DFF8B8E1002273460270A4
:10127000D8F80020012112F0020F8EF800101FBFD5
:10128000417003218EF80010022118BF81705107B0
:1012900041BF9EF8001001F1010E83F800E04FF00D
:1012A000030E48BF00F801E012F00A0F0ED01A78C2
:1012B00004218154511CC9B24FF0050E00F801E021
:1012C000D11C02321970D2B20621815439688F06BE
:1012D00041BF1A78571C1F70072748BF87540A065A
:1012E00008D51A7809278754971C01321F70D2B28B
:1012F0000A2787546779082F01D00E2F08D11A7852
:1013000002F1010E83F800E04FF00B0E00F802E04E
:101310001A7811F4803F4FF00C0C00F802C002F173
:10132000010E1CBFDFF8F8C002325FFA8EFE83F8B0
:1013300000E01FBF8CF80020374A4FF00E0C02F877
:101340000EC04A0748BF1A784FF0120C41BF02F195
:10135000010E83F800E04FF0100E00F802E01A785A
:1013600011F4806F02F1010E5FFA8EFE83F800E047
:1013700000F802C00ED094F81CC2BCF1000F09D0D6
:10138000DFF89CC002328CF80020234A4FF0130C87
:1013900002F80EC01A7811F4007F4FF0140C00F818
:1013A00002C002F1010E1CBFDFF874C002325FFA06
:1013B0008EFE83F800E01FBF8CF80020164A4FF025
:1013C000150C02F80EC0182F40D12BE0002401406C
:1013D000F02900207A2B002090240020404B4C0064
:1013E000B80F0020000C0140A0100020F4120020D3
:1013F000F40500200426002035FA8E3C202600202B
:101400000AE81C4100401C46000700204C12002046
:10141000BD37863500260020810F00201C000020EB
:10142000800F00201A784FF0160E00F802E002F14B
:10143000010E5FFA8EFE4FF0170C00F80EC002F19D
:10144000030E0232D2B283F800E087540F0341BF8B
:101450001A78511C1970192348BF8354002198220F
:101460009C4816F0C0F807F018FF9B4A9B4B9C491C
:101470001A6000234B800B71B4F8980199490A60F7
:1014800081B2994A22F813100133122BF9D1974FE8
:101490003B68D9045CBFB4F89E1111801B0740F172
:1014A000C58094F89231062B00F2BA80DFE803F091
:1014B00004070E395474740045F2F05201E042F60C
:1014C000F8228B4B1A8007F071FFA8E042F6F82251
:1014D000874B1A8012F0ECFC864912F03DFD8649DC
:1014E00012F030FC12F024FF0023844A42F823005B
:1014F0000133122BF9D1824A824940201160824A7D
:10150000137010F099FD002800F08A8001234FF03D
:10151000070A90F9000040218DE808047B4A7C4BC3
:1015200078E042F6F822724B40201A80794A744BD8
:101530001A60754B10221A7010F07EFD00286FD0D3
:1015400001234FF0000990F9000040218DE80802C6
:10155000714A4FF4E1335DE042F6F822644B4020DB
:101560001A806E4A664B1A60674B08221A7010F098
:1015700063FD002854D001234FF0000C90F90000C7
:1015800040218DE80810664A4FF4E13306F018FF59
:10159000644BC3F87C013FE042F6F821544A062B25
:1015A000118059494FF00C02DFF8B0C1DFF8B0E10B
:1015B0005D4C5E480A700FD0002323708CF8003019
:1015C0008EF800301B230370594B4FF4E1341A702E
:1015D000584B05221A700CE0002121708CF8001085
:1015E0008EF80010212101705149534C0A70514A64
:1015F0001370524A424B40201A6010F01DFD78B122
:1016000001234FF0000E90F900008DE808402346BA
:101610004B4A402106F0D4FE003018BF012028B903
:10162000082007F075FB474A354B1A603B68364A7D
:1016300013F4804F1FBF082111704348304918BF71
:10164000086042F20101194099B144F6206028492E
:101650000880980441BF082111703C48284948BFC0
:101660000860D90741BF0C2111703948244948BF8F
:10167000086011781C06A1F10401517040F1AC80A2
:101680002848DFF8E0A04FF00009324CC0F880A1F4
:101690004946152200F5C270DFF8CCB084F80190FD
:1016A000C4F80490C4F8089015F09DFFAAF1050352
:1016B0004846CBF800300AF038FA274B02201B6866
:1016C000E36010F0B9FC002850D1802007F020FB27
:1016D0007BE000BF9C1100207A2B00205C0E0020D4
:1016E000AC0D002060240020CC290020902900208F
:1016F00060070020CDCCCC3F0000B04494220020F5
:101700002000002019DD00083812002091DF0008B9
:10171000A086010005DD0008E5DE0008EDDC00081C
:1017200099DE0008D8000020FC220020FE220020C4
:1017300021220020FF22002090D0030015DC0008A9
:1017400079DD000875DD000849DD000865DD000869
:1017500055DD00081C070020B429002022220020AB
:10176000FD220020E02B00203C07002090F805E03F
:101770006378C7490C2202FB03125278724504D0E9
:101780000133DBB2042BF4D900236370DBF80030A3
:1017900062781B7890F90000002B4FF00C0303FBDC
:1017A000021314BF4FF0030E4FF0010E00225B78BE
:1017B000CDF800E00192022106F002FEB54B186060
:1017C000002882D001200AF0B0F92868B24B00F559
:1017D000C5721A600AF050FA3B68980553D5AF4AB3
:1017E000AF4C059B102523609369AE4843F001037D
:1017F0009361059B0EA91B888DF83A50ADF83830DF
:1018000002238DF83B300DF06CF92368A5485B8806
:101810000EA9ADF8383004238DF83A300DF061F997
:1018200023680120197A0DF047F923689E4A5B6806
:101830004FF00009536117A88DF8615001251793E7
:101840008DF860908DF862500CF0B0FD23680FA801
:101850005B7A8DF83E908DF83C3003238DF83D3057
:101860008DF83F5011F068FB904B914A1B683C3B50
:101870001360D8F800304FF0FF3243F01003C8F87F
:1018800000308C4B1A608C4B8C4A8D4C13608D4A07
:10189000803313603B680025D903257040F1AF8089
:1018A00040F22A39DFF854A2DFF8F0B10FF09CFDC6
:1018B0004FF001084A465046294684F8008015F04A
:1018C00092FEDBF81830804843F00403CBF8183060
:1018D0004023ADF8383018238DF83B300EA9032390
:1018E0008DF83A300CF0A0FDDBF81C30774A43F05D
:1018F0000203CBF81C30764B764C1B68ABF6947B1E
:10190000B3FBF2F32288013B22F45C721204120C46
:1019100022809BB21D22A2852385A4F81480238CEB
:1019200023F001031B041B0C2384238CA188228B2E
:1019300023F0020322F0730212041B04120C1B0C8E
:1019400089B242F0600243EA0803A1802283A5869F
:101950002384238B23F008031B041B0C43F0080390
:101960002383B4F844306FEA43436FEA53439BB296
:10197000A4F84430DBF8A83F43EA0803CBF8A83FBB
:1019800058460CF02DFB544BCDF860A017938023E4
:101990001C934FF480734FF0100A1D9358464FF478
:1019A000005317A920931B951E951F952195CDF8DF
:1019B00064A0CDF8689008F025FAA3890FA89BB21F
:1019C00043F40073A381DBF8003043F00203CBF84B
:1019D00000308DF83CA08DF83D808DF83E508DF89C
:1019E0003F8011F0A9FA3D4B1A683D4B43F8262081
:1019F0000136202EF7D10CF081FF0CF07FFF3B6801
:101A00005A0540F18F80374C374BD4F8C46404201A
:101A10001E6010F011FB0421C4F8C80410F0E8FAAD
:101A2000324B84F8CC0408201E6010F005FB304BCC
:101A30000821186010F0DCFA2E4D84F8CD04002146
:101A400028462C2215F0CFFD8E236B704FF07C09B9
:101A5000E0234FF07D08EB7085F8009085F82B802F
:101A6000254D2C220021284615F0BDFD8A236B70E0
:101A70001020A023EB7085F8009085F82B80C4F827
:101A8000D06410F0D9FA1021C4F8D40438E000BFB3
:101A9000789C01088C240020B00E00200010024029
:101AA00018070020000C014000040140B429002068
:101AB00014070020D80F00201C2C002074110020D7
:101AC000210D0020D02400200008014000366E01C6
:101AD000600000200004004034040040089C01081D
:101AE000220D0020D800002094100020EC100020CF
:101AF00038110020BC100020F110002071020020DD
:101B000010F076FA84F8D8042020C4F8DC6410F0D1
:101B100093FA2021C4F8E00410F06AFA84F8E4048F
:101B20000BF094FB804B814C1B78022B65D1804AD3
:101B300000251388322023F040031B041B0C138064
:101B400013884FF4805623F038031B041B0C1380BA
:101B500013889BB243F0400313809F238DF83C30E1
:101B60008DF83D508DF83E508DF83F5010F04FFBF2
:101B70008DF85D506F4D04226E6117A80FA911F00A
:101B8000F9F92E619DF85E309DF85D201B0243EA55
:101B900002429DF85F301343674A934219D00AD836
:101BA000A2F51A42033A93420CD002F51A420232CD
:101BB000934209D01CE0614A934205D0013293421E
:101BC00007D015E0202300E0802323804FF48073AA
:101BD00002E04FF4807323806380A38822881B0275
:101BE000A3605343E360564B012283F8E52404E0ED
:101BF000002323806380A360E360E46804B3240CC3
:101C000026464FF00008A04514DA08EB04056D10D5
:101C10000DF15C092804494610220DF0CFF800238D
:101C200059F8232001325AD10133042BF8D12E4622
:101C30002C46E8E70AF0D2F9414B3604C3F8E864D1
:101C40003B68404A13F4002318BF0123137010F0BF
:101C5000B9FA3D4B18603D4B5A791946052A02BF27
:101C60003B4B4FF4C8721A803A4B4FF47A721A8089
:101C7000394BC8221A80394A137843F0080313708D
:101C8000374A137823F00203137040F602033A68D0
:101C900013406BB13348344B1860344B0320187039
:101CA000334B0120187033480023038032480380EF
:101CB000930341BF314B04221A71DA7844BF42F0DA
:101CC0000102DA708B6801223B602D4B1A702D4A9D
:101CD000137863F07F03137023B0BDE8F08F05F134
:101CE00001082546A4E7284B00221A7000B212F022
:101CF000DFF8264912F030F91790B4F95E0112F0BE
:101D0000D7F8224912F028F91890B4F9600112F0BE
:101D1000CFF81E4912F020F91D49199017A806F0B6
:101D20000FFFFFF7E8B900BFE33300200C000020ED
:101D300000380040000C014018BA20001740EF00A6
:101D4000D8000020D0310020A40D0020F029002070
:101D5000CC250020DE330020D8330020A410002042
:101D6000E13300206C2B00208C100020F0100020AC
:101D700054000020500F0020520F0020902400201B
:101D8000200D0020B83300203000002035FA8E3CB2
:101D900094230020834A2DE9F04F1368824C03F509
:101DA0009C4320332360A38889B00133A3807F4BF9
:101DB000059219689B4611F4804F05D10CF0E6FCA2
:101DC00010B9237B013323730027794BFDB21E78B2
:101DD000DFF8F481AE4230D9D8F80030072D98BF33
:101DE000595D744B88BF29461B6871489847032D7D
:101DF0001ED8D8F8002005F10E0302EB8303998862
:101E0000DA88A8B14FF47A73401A5843531A90FBFA
:101E1000F3F040F6C90300F57A70984205DC40F211
:101E2000EE239842B8BF184601E040F6CA0080B2DF
:101E300004EB4505E8810137C7E7277B0325B7FB9E
:101E4000F5F50F2384F8323094F8333005EB45056F
:101E5000019394F834307D1B0393D8F80030DFF8F9
:101E600070910293EBB204930025B54254DA524BC1
:101E70004FEA450833F815A0019B53B90CF086FCD6
:101E800028B1039B002B08BF4FF0000A01E0DDF8EA
:101E900004A0029B988A504502D8D88A50450ED299
:101EA000E8B20CF049FC032D8246DFBF94F832E023
:101EB0000120A8402EEA0000D8BF84F832000CF0C0
:101EC00065FC18B13D4828F800A021E0049B94F877
:101ED0007E0029F813A028B9022F15D9324B012012
:101EE00083F87E00B9F80000B9F802300344B9F86D
:101EF0000400034432489BB228F800301BB2032090
:101F000093FBF0F39BB200E053462C4828F80030D6
:101F1000013509F10609A8E794F83250224BA5F1E2
:101F20000F004542454184F898503DB19A8811B25E
:101F30001429CCBF143A00229A800BE083F8335066
:101F4000B54207DAE8B20CF0F7FB1C4B23F815009A
:101F50000135F5E7DBF80030D90405D5194B1B68CE
:101F6000DA0701D411F072FC059B1F68164B1A6842
:101F7000907A78B31149137B013831F810001BB106
:101F8000C0F53B60083080B200B2A0F57A70B0F5C1
:101F90007A7FA8BF4FF47A7020EAE07011F088FFD2
:101FA0000A494DE0C0330020A80D002090290020F0
:101FB0003812002020000020B60D0020CC2900207F
:101FC000280E00207C0F00206024002000007A44AE
:101FD000DE0D0020DBF800301B043AD5D4F89C302D
:101FE000A64DFB1A002B34DB07F59C432033C5F8C4
:101FF0009C30A34BD27A5979A24B33F8113095F823
:10200000A0109BB293FBF2F3013101F00F0285F8AF
:10201000A0202A4482F8A13003469B4A825C01300A
:10202000134410289BB2F8D11BB293FBF0F000B21E
:102030006428A8BF642020EAE07011F039FF9349BA
:1020400012F03EF8924911F087FF12F071F9914BAE
:102050001880DBF80030904D13F4807F8F4E7FD0D6
:102060008F4B9F4204D9237A13B9844B01221A72F1
:10207000B4F904E03778BEF1140FCCBF4FF0000E76
:102080004FF0010E7D4BC7F38007BEF1000F06D065
:102090004FF0000883F80A8083F8098001E04FF0D0
:1020A0000308D4F8B430A07A0193D4F8B8C0B4F9D6
:1020B0000490617AE3882A88032847D8DFE800F093
:1020C000020E1B36BEF1000F02D02A8000222BE048
:1020D000002F40F05C862A80A77239E09CF800004F
:1020E00000EB8000814502DC2A8001221CE00120F7
:1020F00067B300F0BDBE47B1019A4FF00208D28924
:102100006A80AA80BCF80200E8809CF800A09CF8D5
:102110000100504400EB8000814500F33B86002F16
:1021200000F038862A800222A27211E02A8003225F
:10213000A2726172E3806FB13378002243F0020330
:1021400033704E4B5A7211F081FB03E02A80A0726B
:102150006172E380B8F1000F02D0404610F090F8B1
:10216000504FB7F8520111F0ACF90197824668B9A7
:1021700011F0BCFD4C4B0022C3F800A0C3F804A032
:10218000C3F808A0494B1A605A609A6033785F0719
:1021900037D5DBF80030D80633D5454B1B78D90648
:1021A0002FD4444B1B789BB1019B93F8DE31BAF1DD
:1021B000000F15D17BB1404B1A68D4F8BC309B1A84
:1021C000002B08DA11F042FB2C4B83F8C0A018E07A
:1021D000BAF1000F0DD1102010F052F801230EE0DB
:1021E0003BB1354A4FF47A71126801FB0323C4F8FE
:1021F000BC3094F8C03023B110F02EF8002384F8DE
:10220000C030019B93F8DC9193F8DD11B3F89A711B
:10221000B3F89CE10023184635F913208008BA4230
:10222000C4BF60F07F00C0B201337245B8BF40F058
:102230004000042BF0D194F8C130104A834205D1FC
:1022400092F8C230F92B04D8013300E0002382F861
:10225000C230184A84F8C1001078084B174F9046D6
:1022600000283CD13A68D2072AD5BAF1000F36D1FE
:102270003378DB0733D511F03DF930E0A80D0020AD
:10228000B8230020C8230020490E00200000C842C7
:1022900000C07F44DC0F0020CC290020E133002067
:1022A000404B4C00F0290020002500204021002058
:1022B000A410002008000020B42900207C0F00207A
:1022C000327850070BD593F8332042B15B7A33B99B
:1022D00011B111F0BBFA02E0BAF1000FF9D094F895
:1022E000C2307B4A142BDFF818A240F08F8098F898
:1022F000003019F1000918BF4FF001096BB392F8D3
:10230000C1305F2B11D1337803F0040303F0FF01D8
:1023100013B111F09BFA08E00B20039102920FF029
:10232000AFFF029A039982F8C210B9F1000F14D0DE
:1023300094F8C1307D2B10D1337803F0040303F0FF
:10234000FF0213B111F082FA07E00B2002920FF0A6
:1023500097FF5F4B029A83F8C220337803F004039F
:1023600003F0FF01002B51D194F8C130584A572B8C
:1023700016D1584B4FF47A721A80DBF800301906E8
:1023800001D509F0C9FC544B1B685A0742BF534A98
:102390000A21118013F0080338D1514A138035E027
:1023A000DBF80000400716D55A2B14D14D4B187896
:1023B00020B119704C4B01221A7027E092F8C330FB
:1023C00083F0010382F8C3300BB10C2000E00D2034
:1023D0000FF056FF1AE05D2B00F0DF845B2B00F05E
:1023E000DE845E2B02D1032000F0DABC562B01D133
:1023F00006F02CFF98F80030002B00F0E78494F8EA
:10240000C1306F2B40F0DC8411F074F8DBF8003041
:102410005B0732D594F8C330A3B13378580711D590
:10242000019BB5F90620B3F89A319A420ADD3B6860
:1024300013F0010301BF2D4A32211180244A08BF45
:1024400082F8C3303B68D9030AD5294B1A782AB9D8
:10245000244A127812B9254A3221118001220BE058
:10246000204A13784BB1337803F0040303F0FF01E3
:102470001BB91D4B117001221A70DAF8008000237D
:102480003B6008F17B0608F1CB093278737816F8C7
:10249000010C9A420BD231460FF036FE38B116F8D5
:1024A000022C012303FA02F23B6813433B6004361B
:1024B0004E45EAD10F4B1B7823B30F4DDFF8188040
:1024C0002B680E4F13F0020F40F0408338E300BF3B
:1024D000A80D0020DE330020A0100020D8330020FB
:1024E0007C100020F9250020FA250020E02500209E
:1024F000F8250020E63300207C0F00206811002022
:10250000B80F002008F1CA0608F589773278737889
:1025100016F8010C9A4225D231460FF0F5FD08B3AA
:1025200096F804E00C21B37801FB0E41B74A013B59
:1025300003EB43031344D1F8C82096F803809A4272
:10254000B3480FD0C1F8C830002390F8F420C1F888
:10255000CC30012303FA0EF322EA030381F8C4808E
:1025600080F8F4300636BE42D0D1AA4BDFF8B892DC
:102570001F68A94B4FF0000A1B68029394F8333090
:102580000393D9F80010002900F0C48291F800806C
:10259000B8F1000F00F0BE82D9F80430029AD31AC5
:1025A000002B0CDB02F5FA73C9F8043094F8F42020
:1025B000012303FA0AF322EA030384F8F430039BAD
:1025C000002B00F0A78219F8042C4B780432D2B209
:1025D000002B40F06082914B35F91200B3F898213E
:1025E00002F1C80398428A4B01DD8E7814E0C83AA4
:1025F000904202DA89784E420EE093F8F4100122FC
:1026000002FA0AF221EA020283F8F420029B03F59F
:10261000FA73C9F804307DE293F8F42042FA0AF222
:10262000D20700F17782002ECCBF02200120049354
:102630000FF048FE08F1FF32049B132A00F261827A
:10264000DFE812F0140021002E003E0057005E006B
:10265000C30038019D01CA01F9015F023E004D002F
:102660005E00C300380195000A016F0139783846D1
:102670000E44FA2EA8BFFA2626EAE6763E700FF040
:1026800029FD01201AE0797838460E44642EA8BF4F
:10269000642626EAE6767E700FF01CFD02200DE02F
:1026A000F97838460E44642EA8BF642626EAE676FA
:1026B000FE70D3F8F8100FF0C5FC03203146B7E1E7
:1026C00079790D2031446429A8BF642121EAE171A0
:1026D00079710FF063FDB8F10D0F00F012823979B6
:1026E0000E2031446429A8BF642121EAE1713971C7
:1026F0009EE1B9790520314481F30801B97197E170
:10270000D3F8FC301A78022A22D13046049311F013
:10271000CFFB434911F0D4FC049B596A059311F097
:1027200013FB0021049011F0B5FD059B48B9049AF4
:102730003C49104611F0CCFD049A059B10B1394A72
:1027400000E000225A620F2011460FF012FD0AE04D
:1027500099780F203144C829A8BFC82121EAE17126
:1027600099700FF01BFDB8F10F0F00F0CA81284BD4
:10277000D3F8FC8098F80030022B1AD1304611F0C3
:1027800097FB274911F09CFCD8F8201011F0DCFAD7
:102790000021064611F07EFD30B93046214911F086
:1027A00097FD10B11F4E00E00026C8F820601220EF
:1027B00061E198F8011012203144C829A8BFC8214E
:1027C00021EAE17188F8011032E1D3F8FC301A787F
:1027D000022A32D13046049311F06AFB114911F0FC
:1027E0006FFC049B196B059311F0AEFA0021049065
:1027F00011F050FD059BC8B9049A0A49104611F022
:1028000067FD049A059B90B1064A10E070A001088C
:10281000A80D0020E00F0020B4290020F02900209E
:10282000000020410000C842700E002000221A6300
:10283000102011460FF09DFC0AE0197B1020314456
:10284000C829A8BFC82121EAE17119730FF0A6FCBD
:10285000B8F1100F00F05581B34BD3F8FC8098F815
:102860000030022B1AD1304611F022FBAF4911F093
:1028700027FCD8F82C1011F067FA0021064611F059
:1028800009FD30B93046A94911F022FD10B1A74E1B
:1028900000E00026C8F82C601320ECE098F80B103C
:1028A00013203144C829A8BFC82121EAE17188F862
:1028B0000B10BDE0D3F8FC301A78022A22D1304642
:1028C000049311F0F5FA9A4911F0FAFB049BD96BC5
:1028D000059311F039FA0021049011F0DBFC059BFF
:1028E00048B9049A9149104611F0F2FC049A059BEC
:1028F00010B18E4A00E00022DA63112011460FF079
:1029000038FC0AE0997D11203144C829A8BFC821AC
:1029100021EAE17199750FF041FCB8F1110F00F057
:10292000F080814BD3F8FC8098F80030022B1AD14C
:10293000304611F0BDFA7E4911F0C2FBD8F83810CC
:1029400011F002FA0021064611F0A4FC30B930461D
:10295000764911F0BDFC10B1744E00E00026C8F8B5
:102960003860142087E098F8151014203144C829E5
:10297000A8BFC82121EAE17188F8151058E0D3F802
:10298000FC8098F80030022B1AD1304611F090FAF2
:10299000684911F095FBD8F8281011F0D5F90021FD
:1029A000064611F077FC30B93046604911F090FCD2
:1029B00010B15E4E00E00026C8F8286009205AE0F9
:1029C00098F8031009203144C829A8BFC82121EA7A
:1029D000E17188F803102BE0D3F8FC8098F8003000
:1029E000022B1AD1304611F063FA504911F068FBFE
:1029F000D8F8341011F0A8F90021064611F04AFC6D
:102A000030B93046494911F063FC10B1474E00E03F
:102A10000026C8F834600A202DE098F80D100A202E
:102A20003144C829A8BFC82121EAE17188F80D10F6
:102A30000FF0B4FB65E0D3F8FC8098F80030022B6F
:102A40001DD1304611F034FA394911F039FBD8F86C
:102A5000401011F079F90021064611F01BFC30B945
:102A60003046324911F034FC10B1304E00E00026FF
:102A7000C8F840600B2031460FF07BFB41E098F82E
:102A800017100B203144C829A8BFC82121EAE171E1
:102A900088F81710CCE7012B33D135F9123088783C
:102AA000B3F5617F05DB40F633029342A8BF1346BE
:102AB00001E04FF46173B8F10C0F22D14FF496622C
:102AC00092FBF0F0A3F5617393FBF0F31A4ADEB2C8
:102AD0001378B34215D0042E34BF3346022313704B
:102AE000019A08FB0323154A03F2B67313600DF035
:102AF00080FF404631460FF051FB701CC0B20FF012
:102B0000E1FB0949012391F8F42003FA0AF3134386
:102B100081F8F4300AF1010ABAF1040F09F10C0945
:102B20007FF42FADC9E400BFA80D00200000C8420B
:102B300000007A440000204148290020E00F0020D6
:102B4000DBF80030DB050FD5637A6BB1D8F80030C5
:102B50009E0709D53B8813F001060AD111F0C6F88B
:102B6000012006F0C5F804E0012006F0B0F80123CA
:102B700000E000232A6850070CD55BB1012006F065
:102B8000A6F83B88990708D411F0B0F8022006F0A7
:102B9000AFF802E0022006F09AF83B88B74A13F03B
:102BA000030F4FF0100114BF51611161D8F80020DC
:102BB00012F00A0F23D02A68D20609D55E070AD47C
:102BC000042006F095F8AE4B1B88A4F8003102E013
:102BD000042006F07CF82B68980606D53B88590639
:102BE00006D4402006F084F802E0402006F06FF89A
:102BF0002B685A0642BFA24B1B88A4F80231D8F8B2
:102C000000309B0608D42B681F0540F18E804FF4DE
:102C1000807006F06DF88CE09A4B1B789E074FD5BC
:102C2000994B1B78042B4BD92B68984E13F40078E2
:102C30000ED03B88DC0637D4102006F059F820204F
:102C400006F045F89248011D08F0D0FF022327E066
:102C50003C8804F01004A4B22CB1102006F037F820
:102C6000012486F804812B68580512D5D6F808315E
:102C700088495A89B1F90030002BB8BF5B429342B2
:102C800007DAB1F90230002BB8BF5B429342C0F2C1
:102C900011813B88990608D5202006F018F80023FA
:102CA00086F80431012400E0002496F80C31B3B911
:102CB0000E200FF0E5FA754B012283F80C210EE08F
:102CC0003B8803F03003002B9DD0102005F0FFFF60
:102CD000202005F0FCFF002384F8043101E0002CE3
:102CE00091D0002006466C4B002423F816406B4B15
:102CF0001A1D03F10A0122F8164000224250014435
:102D00004C608A6023F8164003F132015A33425076
:102D1000C250014403444C608A605C609A60143085
:102D2000002E7FF470AF0126DDE74FF4807005F0D0
:102D3000CEFF5B4B5A791C46082A01D00E2A02D1DD
:102D4000402005F0C4FFDBF800305A0540F1C78091
:102D500094F81C3223B9534B1B7813F0040F02E094
:102D60002B6813F4002F0BD04F4B00221A703C201D
:102D700007F016F8002800F0B2800FF011FEF6E719
:102D80000AF064FA09B0BDE8F04F06F086BA0120F7
:102D9000FFF792B90320FFF78FB9012000E002206E
:102DA0005FFA80F8019A08F1FF3382F8B43705F032
:102DB000E9FF06F089F840460FF084FAFFF726BBDA
:102DC000B9F1000F02D07E2B3FF41EAB94F8C13056
:102DD000972B05D1354B4FF4C8721A80FFF716BBFD
:102DE000A72B06D1274A137843F004031370FFF78B
:102DF0000DBB0022BB2B079201D1022303E0B72BAE
:102E000004D14FF6FE73ADF81E3009E0BE2B01D1A0
:102E1000022303E0BD2B1AD14FF6FE73ADF81C3030
:102E2000DAF80030BDF81C10B3F858200A44A3F8B3
:102E30005820BDF81E10B3F85A200A44A3F85A20AF
:102E400006F004FA002384F8C230FFF7DFBA792BCA
:102E500004D1174AD37823F0010306E07A2B7FF4DC
:102E6000D5AA134AD37843F00103D370FFF7CEBA43
:102E7000013301469BB20220FFF71EB9000C01404E
:102E80007C100020A4100020AA100020A80D002013
:102E9000E80F002084100020DA330020B60E002056
:102EA000F0290020E133002000130020CC25002071
:102EB000902400203B889B063FF5F7AE202005F0CC
:102EC00017FF084B08481A685B68011D43600260E1
:102ED00008F08CFE054B012483F80441E5E609B0B7
:102EE000BDE8F08FAC100020F00F0020A80D0020EE
:102EF000BA4B2DE9F04FB3F90610B94B89B01F68F2
:102F000001937A8991420EDBB1F5FA6FFC79BFBF6C
:102F10008B1A6343A2F5FA6493FBF4F4ACBFC4F1DB
:102F20006404643400E06424AE4BAF4A1868B2F81D
:102F300098A1054692F96221049092B205920293FB
:102F4000002240F2E630A54B4FEA420B33F9123033
:102F50000393CAEB030303F2F316864203D8002B54
:102F6000B8BF5B4201E04FF4FA73022A049E4FF0AF
:102F700064002FD096F811E1BEF1000F04D0734524
:102F8000CCBFCEEB0303002393FBF0FCDFF8A0E201
:102F90006FF063093EF81C8009FB0C390CF1010C41
:102FA0003EF91CE00FFA88FCCCEB0E0E0EFB09FE7E
:102FB0009EFBF0FE8D4EC64426F80BE0BE18367917
:102FC00073438B4E93FBF6F364339BB2634393FBE3
:102FD000F0F02DE096F812E1BEF1000F04D0734539
:102FE000CCBFCEEB0303002393FBF0F0DFF82C8281
:102FF0006FF0630C0CFB003938F910E0013038F940
:103000001000002BCEEB000000FB09F999FBFCF946
:103010000598CEEB090909FB00F97448B8BF5B427B
:10302000A0F80490B8794343714893FBF0F0643002
:103030006B784FF0640E434393FBFEF36D4E022A10
:10304000B354EB7A6C4E00FB03F393FBFEF3B354E3
:103050006B7D664E00FB03F090FBFEF0674B9854CF
:10306000674B0FD183F802E0039B53450EDB5E4CA8
:10307000B4F89A21914215DBB1F5FA6FA8BF4FF46D
:10308000FA6110E09C54039B534504DA36F80B3088
:103090005B4226F80B300132032A05F101057FF46B
:1030A00050AFE4E71146891A4FF47A735943C2F5D9
:1030B000FA62B1FBF2F1642791FBF7F2DFF874E1F9
:1030C0006FF063033EF8120003FB021101323EF978
:1030D000122003B2D21A514391FBF7F30344F38059
:1030E000484B424D1B8858063BD5474A474B1088F2
:1030F0001B88181A00B210F0DBFE454910F02CFFB7
:10310000074605F013FD8046384605F09CFC07464F
:10311000B5F9020010F0CCFE8146B5F9000010F0C0
:10312000C7FE4146824610F017FF3946834648469F
:1031300010F012FF0146584610F004FE11F0D2F8CC
:1031400041462880484610F007FF394680465046E1
:1031500010F002FF0146404610F0F6FD11F0C2F8F3
:1031600068802C4F3B68990740F19F8045F207210A
:10317000294B2A4D1A686B69D31A8B4240F395800C
:103180006A610BF0BFFA264BDFF8AC901A789846CC
:10319000032AB9F8003051D10A2B59D9002328202D
:1031A00088F800300FF033F80BF0ACFA1D4B18889C
:1031B0000BF092FA1C4B1A68D37890FBF3F00130B5
:1031C00008281A4BA8BF08201870537980B24343CF
:1031D0002B831379584368833AE000BFCC29002041
:1031E000E00F0020B80F0020F029002084100020FC
:1031F0000CFEFFFF4C210020460F00206021002024
:10320000E024002068110020AA0E00207C1000207D
:1032100035FA8E3C90290020C0330020380F002062
:10322000F0100020D02300208C100020540000203B
:10323000D2270020BA270020901000200A2B07D8A0
:1032400003239C4A88F80030002313702B836B8380
:1032500098F80030984A012B0CD002D3022B1BD0D7
:1032600023E02A8BB9F800309A421EDD012388F84A
:1032700000300FE0B9F800106B8B8B4202DD0223A7
:1032800013700FE08D4B1B8B0133994202DD00233D
:1032900013700AE0082006E06B8BB9F800200133B8
:1032A0009A42E3DC07200EF0EBFF3D682A0576D555
:1032B000834B824F1A68FB69C3EB020845F2072370
:1032C00098456CDD7F4BB6F906B0D3F800904FF40B
:1032D0007A7199F80A30FA61012B98FBF1F8B4F889
:1032E0005201ABF57A7B784E03D041D3022B20D02C
:1032F00040E0764B386A5A7B754B4FF0080E33F836
:10330000122090FBFEF392B2C01A83183B6293FB2B
:10331000FEF3BA8440F6E4429BB25343B9F8082066
:10332000C2EB13335943B9F9063091FBF3F1316025
:1033300020E0684BB9F808A01B78C6F800A05B072E
:1033400018D510F0BEF820B915F0100F18BF4FF0C7
:10335000000B0BFB0BF3322293FBF2F3B9F90620BF
:103360005B445A434FF47A7392FBF3F3534400E007
:10337000002333603368D7E90A0103FB08F84FF4F0
:103380007A7398FBF3F810EB080041EBE871002327
:10339000C7E90A01504A10F0EBFF504B1860504E3D
:1033A0003368D90427D52A0622D54E4B1B789B07B4
:1033B0001ED54D4B187804281AD900224B4B0521F5
:1033C000D718951C4FF00A0E122AD154E9B287F88B
:1033D00001E004D0B0EB510F2A46EFD800E01421F1
:1033E0005A18322002F8010CFF225A540F2000E034
:1033F0000A200EF045FF3E4D2A68002A51D03D4B71
:103400003D4F18683968984681424AD83B4BDFF8EF
:10341000F89019785268E1B94FF0010A83F800A0DA
:10342000B9F80030D35C23B350460EF00FFF344B95
:1034300083F800A00BF0B6F9B9F80030CBB92B68CF
:103440001B78053B534514D80EF0BCFE2D4B18607D
:103450000FE04FF0000A83F800A0B9F80030D35C09
:103460003BB150460EF0F2FE254B83F800A00BF066
:1034700099F92B68B9F800205B6823499B5CFE2B07
:1034800002D100230B800CE0FF2B02D10EF0E4FEF2
:1034900007E0D8F800000A2505FB030301323B6072
:1034A0000A800C4D2B785F0732D5184B08225A61E1
:1034B0006CE000BF54000020F0100020380F002006
:1034C000C03300208C10002098100020B82300206A
:1034D000C8230020E1330020407E05009C1000201E
:1034E0007C0F0020A4100020AA10002068290020D2
:1034F000F0270020B4290020E8270020E42700203E
:103500006424002084330020EC270020000C0140BC
:103510003268D0075CBF43F001032B70A84B1B78C7
:1035200019075EBF2B7823F001032B70D30248BF2D
:103530002B78A44A44BF23F001032B70A24B1B68D5
:1035400013F0040F02D0A149098851B9A049098894
:1035500009B19F0705D49F4B1B88003318BF012377
:1035600033B1022313702B7823F001032B7004E096
:103570002978CE0758BF022313700EF023FE964B16
:103580001B68C01A002801DB0BF00CF909F05EFE85
:10359000924B1E780393002E00F0A980904F3B6859
:1035A000002B00F0218738680EF0F8FE002800F0AC
:1035B0001B878B4B8B4C18680EF0EDFE092801D051
:1035C0003F2852D14FF000094D462668DFF850825F
:1035D00036B18548D8F80010324614F051F810B9C9
:1035E000C14605B94546814B08F110089845EFD30F
:1035F000EDB1D5F800C0D9F8008023681CF803E0CD
:1036000018F80300704512D15A1C774958B92D2B70
:1036100009D8DFF8D0E1CEF800204FF0200E01F8F5
:1036200003E0885403E001F803E02260E5E7236843
:103630000BB14D4510D06E480FF0A8FA4D4507D894
:1036400055F8100B0FF0A2FA09200FF097FAF5E7E2
:1036500068480FF09BFA002623689E42A3D2624B73
:10366000985D0FF08BFA0136F6E72368002B40F0E7
:10367000A086042840F0DC865B480BF019FF00F0C0
:10368000B3BED8F80000DFF87CA10EF087FE20B3AF
:10369000DAF800000EF07FFED9F80030834693F888
:1036A000482092BB242869D1012283F84820D9F808
:1036B0000030DFF84CA193F848B0BBF1060FE0D121
:1036C00093F8490000F042FF002800F0AB800FF0B3
:1036D000B5F93B68002283F84820474B93F8353012
:1036E000002B40F054864C36982E00F07D86434BDC
:1036F000F21892F84A100129F5D1414FF3583A6077
:10370000404AB94613609046BBE7012A04D14D28D0
:1037100014BF00220222C8E7022A04D13C2814BFA9
:1037200000220322C1E7032A0AD140284FF00002F9
:103730009FBF1A71DA715871987198BF0422B4E76B
:10374000042A08D19A7983F8490080EA020B83F8A9
:1037500006B00522A9E7052AA9D159791A7991421B
:10376000997906D941409971511C19711344187205
:103770009DE781420CBF0622002296E72B7859076D
:1037800095D42328DAF800300CD1039901220A706D
:10379000134A1D481360184A13630FF0F7F91548D0
:1037A0000FF0F4F9194B1B681B785B4501BF184AF1
:1037B000184B1A60184A04BF184BDA6077E700BF4D
:1037C000A410002064240020A0100020D833002082
:1037D000CC250020DE33002068240020E6330020C2
:1037E00064290020CC2400209C240020F8AC01088F
:1037F000D3C20108D8C20108380F00209C11002054
:10380000481100204C11002008C3010804130020B7
:10381000EFBEADDEF04F00200400FA0500ED00E041
:1038200018AB0108DAF8002092F849304C2B00F070
:10383000858400F29080352B00F0588239D82B2BEC
:1038400000F0548420D8252B00F02C8404D8232B9E
:1038500000F0138200F0E8BD272B00F02984292B0B
:1038600040F0E2850FF0C6F8A4F882010FF0C2F82C
:10387000A4F884010FF0B4F884F886010FF0BAF8C8
:10388000A4F8880100F07EBD2F2B00F0F78404D847
:103890002D2B00F02F8400F0C7BD312B00F00385E5
:1038A000332B40F0C1850FF09BF884F8940100F0B1
:1038B00069BD412B00F09C8418D8392B00F0058499
:1038C00004D8372B00F0A18400F0AEBD3C2B00F0F3
:1038D000CC803E2B40F0A8850FF082F884F8DE0102
:1038E0000FF07EF884F8DD0100F04CBD442B00F0B1
:1038F0000E8525D8432B40F097850FF071F80023F3
:10390000A36060710FF080F805F00AFA0FF068F814
:1039100084F892010FF06EF8A4F85C010FF06AF8D9
:10392000A4F85E010FF066F8A4F860010FF062F8E9
:10393000A4F882010FF05EF8A4F8840100F022BD23
:10394000482B00F044834A2B40F06E850FF052F86C
:10395000A08100F017BDD12B00F0638320D8CC2BC1
:1039600000F006820FD8C82B62D004D84E2B00F08E
:10397000118400F059BDC92B00F02C83CA2B00F034
:10398000838000F051BDCE2B00F01483C0F009837A
:10399000CF2B00F04182D02B00F0F88200F044BD24
:1039A000D82B00F000810BD8D32B3BD027D3D42BBE
:1039B00000F07682D62B40F037854FF0000864E2A5
:1039C000F22B00F0BB8212D8EF2B40F02D85DFF8F0
:1039D0007C83D8F800900FF00DF8A9F85A00D8F8B9
:1039E00000800FF007F8A8F8580000F0CBBCF32BCC
:1039F00000F09284FA2B00F0E68200F015BD2B78DF
:103A000003F0040303F0FF08002B40F0BB840EF02A
:103A1000E7FF022884F8B40740F2BE82C74B83F860
:103A2000B487B9E20EF0E6FFC54B188000F0AABCDF
:103A300092F805804FEA5808B8F1120F03D906F042
:103A4000ABF900F09FBC4FF00009C14507D20EF062
:103A5000D1FFBC4B23F8190009F10109F5E7BA4B76
:103A6000012283F8342000F08DBCDFF8E082D8F822
:103A700000900EF0B5FF89F80000D8F800301878F3
:103A80000CF090FF00F07EBCB04B1A68984612789C
:103A9000022A6BD14FF00008DFF8B09208F1080B52
:103AA000D9F800A00EF09CFF10F0FEF9A84910F024
:103AB00007FB4AF82B00D9F800A00EF091FF08F19F
:103AC0000A030AEB830A10F0EFF9A24910F0F8FAA2
:103AD000CAF80400D9F800A00EF082FF10F0E4F953
:103AE0009D4910F0EDFA08F10E0B08F10108B8F14C
:103AF000030F4AF82B00CFD1B8F1070FD9F800A077
:103B00001AD10EF06DFF10F0CFF9914910F0D8FAEC
:103B1000CAF84400D9F800A00EF062FF10F0C4F912
:103B20008B4910F0CDFACAF84800D9F800A00EF081
:103B300057FF8AF84C0012E00EF052FFC2448AF898
:103B40000100D9F800A00EF04BFFC2448AF80B0028
:103B5000D9F800A00EF044FFC2448AF8150008F11D
:103B60000108B8F10A0FC7D100F00CBC4FF00009F2
:103B7000D8F800A00EF034FFCA448AF80100D8F843
:103B800000A00EF02DFFCA448AF80B00D8F800A060
:103B90000EF026FFCA4409F10109B9F10A0F8AF8AB
:103BA0001500E5D1EEE38046DFF8A09108F1080B9F
:103BB000D9F800A00EF01EFF10F076F9664910F05B
:103BC0007FFA4AF82B00D9F800A00EF013FF08F195
:103BD0000A030AEB830A10F067F95F4910F070FAE4
:103BE000CAF80400D9F800A00EF004FF10F05CF948
:103BF000594910F065FA08F10E0B08F10108B8F107
:103C0000030F4AF82B00CFD1B8F1070FD9F800A065
:103C10001AD10EF0EFFE10F047F94F4910F050FAAC
:103C2000CAF84400D9F800A00EF0E4FE10F03CF908
:103C3000494910F045FACAF84800D9F800A00EF03A
:103C4000D9FE8AF84C0012E00EF0D4FEC2448AF885
:103C50000100D9F800A00EF0CDFEC2448AF80B0096
:103C6000D9F800A00EF0C6FEC2448AF8150008F18B
:103C70000108B8F10A0FC7D184E30EF0B1FE132892
:103C800082463FF6DCAEDFF8C490D9F800800EF033
:103C9000A7FE002331490C2202FB0312117A814254
:103CA00020D1137808EB8A0888F879300EF098FE56
:103CB00088F87A000EF094FE88F87B000EF090FEF3
:103CC000274A284B88F87C001A60D9F80000264B58
:103CD0000021186079300EF03BFA244B80F001008F
:103CE00018704FE301331B2BD4D1A8E60EF078FEF9
:103CF0000B2880463FF6A3AE144BD3F800900EF08D
:103D00006FFE03283FF69BAE0BFB089B8BF8CE00A3
:103D10000EF066FE8BF8C9000EF062FE8BF8CA004A
:103D20000EF05EFE8BF8CB000EF05AFE8BF8CC0046
:103D30000EF056FE8BF8CD0024E300BFF0290020E2
:103D4000A80E0020CC290020380F0020B80F00203A
:103D5000000020410000C84200007A44DCA00108B5
:103D6000342B0020A00E0020A40E0020080000200C
:103D70005379092B7FF663AE019BD3F800800EF0D8
:103D80002FFE019B88F80000D3F800800EF028FE7B
:103D900088F801000EF024FE019B64281B68A8BF70
:103DA000642018710EF01CFE019B64281B68A8BFDC
:103DB000642058710EF014FE019BFF281B68A8BFF9
:103DC000FF2098710EF00CFE019B6428D3F8008050
:103DD00028BF642088F807000EF002FE019B88F8D7
:103DE0000200D3F800800EF0FBFD019B88F8030071
:103DF000D3F800800EF0FEFDDAF80030A8F80A00D3
:103E00005B790A2B40F2BE82D34BD3F800800EF0D0
:103E1000E7FD88F80800B5E20EF0ECFD6FF4AF6244
:103E200083189BB2C62B98BFA4F898010EF0E2FD50
:103E3000A4F844010EF0DEFDA4F846010EF0DAFD10
:103E4000A4F848010EF0D6FDA4F8DA010EF0C8FD82
:103E500084F8EB010EF0C4FD0EF0C2FD84F8EC0115
:103E60000EF0BEFD84F887010EF0BAFD84F89401CF
:103E70000EF0B6FDB94BD3F800800EF0BBFD00EBA1
:103E800080004000A8F856001FE10EF0B3FDB44BCF
:103E900023F8180008F10108B8F1080FF5D171E214
:103EA00053790F2B7FF4CBAD0EF09AFD0728804697
:103EB0003FF6C5AD029BD3F800900EF09BFD0E239C
:103EC00003FB08F8029BC144A9F81901D3F800903C
:103ED0000EF090FDC144029BA9F81B01D3F800909D
:103EE0000EF088FDC144029BA9F81D01D3F8009093
:103EF0000EF076FDC144029B89F81F01D3F80090B3
:103F00000EF06EFDC144029B89F82001D3F80090A9
:103F10000EF066FDC144029B89F82101D3F80090A0
:103F20000EF05EFDC144029B89F82201D3F8009097
:103F30000EF06AFDC844C8F8230123E20EF050FDDC
:103F40000F2880463FF67BAD0EF04AFDC8EBC8084F
:103F5000A04488F8D4000EF043FD88F8D5000EF098
:103F60003FFD88F8D6000EF03BFD88F8D7000EF034
:103F700037FD88F8D8000EF033FD88F8D9000EF030
:103F80002FFD88F8DA000EF0C9FBFBE12B785B0708
:103F900000F1F8810CF072FD04F0F4FE04F094FFDF
:103FA000F0E12B78580700F1ED816E4B4FF4C872A9
:103FB0001A80E7E12B78590700F1E4816A4A137807
:103FC00043F004032BE02B785A07E5D52CE208F0E8
:103FD00043F8D7E10EF004FD634B1A7810B142F0BC
:103FE000020201E022F002021A700EF0F9FC5F4BAF
:103FF000DFF8988118700EF007FDC8F800000EF089
:1040000003FDC8F804000EF0F5FC594B18800EF0C3
:10401000F1FC584B584A1880137843F00203137090
:10402000B0E10EF0DDFC83460EF0EEFC82460EF0B1
:10403000EBFC81460EF0E8FC80460EF0DBFC0EF057
:10404000D9FC0EF0CDFCBBF1000F14D14B4B10206E
:10405000C3F800A0C3F8049004F039FE424A137874
:1040600043F001031370B8F1000F00F08B81444B53
:10407000C3F8008086E1BBF1100F40F08381414B13
:10408000C3F800A0C3F80490B8F1000F02D03C4B75
:10409000C3F800803B483C4B0222011D1A7007F018
:1040A000A5FD6FE1A0600EF0AFFC04F039FE69E100
:1040B0000EF0A0FCA4F85C010EF09CFCA4F85E01DC
:1040C0000EF098FCA4F860015CE10EF089FC84F825
:1040D0007C010EF085FC84F880010EF081FC84F8F0
:1040E0007F010EF07DFC84F881014BE10EF078FC3D
:1040F000607147E10EF074FC84F892010EF07AFCD6
:10410000A4F89C010EF076FCA4F898010EF072FC65
:10411000A4F89A010EF064FC3B6884F893015B7983
:10412000DFF86C80082B40F22D810EF063FCA8F8BC
:104130009E010EF05FFCA8F8A00123E10EF050FCF8
:1041400084F8D8010EF04CFC84F8D9010EF052FC32
:10415000A4F8DA0116E100BFE00F0020B80F00203C
:104160004A290020CC250020A4100020AA100020FD
:10417000A8100020A6100020E60F0020E80F002065
:10418000F80F0020F00F0020AC0E0020AC10002033
:10419000F029002092F805800323B8FBF3F8B8F16A
:1041A000120F3FF64CACDFF8A0934FF0000AC24567
:1041B00080F0E8800EF014FC89F8A2010EF01AFCE1
:1041C00040F2ED23984205DD40F6CA039842A8BFAD
:1041D000184601E040F2EE20A0F2EE20192390FBF9
:1041E000F3F00AF1010A89F8A30109F10209DEE7F7
:1041F00080460EF0F5FB04EB080308F10108B8F166
:10420000080F83F88A01F4D1BCE053794FF0070915
:10421000B3FBF9F9C9EBC9029B1A13F0FF0F7FF446
:104220000EAC5FFA89F909F1FF395FFA89F9B9F142
:10423000FF0F00F0A7800EF0D3FB5FFA80FA4FFA71
:104240008AF00DF0C1FE804600283FF4F8AB80F8FC
:1042500000A00EF0CFFBA8F802000EF0C1FB88F81A
:1042600004000EF0BDFB88F805000EF0B9FB88F8DD
:1042700007000EF0B5FB88F80600D4E7DFF8C88227
:1042800008F140090EF0B6FBA8F8AC020EF0A8FB4E
:1042900088F8AE020EF0A4FB08F1040888F8AB021F
:1042A000C845EFD16EE00EF09BFB1F2880463FF61D
:1042B000C6AB3B685B79082B7FF4C1AB0EF09AFB71
:1042C00008F18A0804EB880800F03F00A8F806000F
:1042D0000EF090FBB8F80630800100F4FE50184351
:1042E000A8F806000EF07CFB000188F804000EF030
:1042F00077FB98F8043000F00F00184388F80400AA
:104300000EF06EFB88F805000DF06EF83AE07A4B7F
:10431000012283F8352035E00EF062FBFF2881464C
:104320001BD100238DF81F309DF81F30052B29D895
:104330009DF81F00714A9DF81F30012102EBC30355
:104340005B6852F83000994089B2482203F042FF7E
:104350009DF81F300133DBB2E4E705283FF66FAB71
:1043600000200EF08FFB0EF069FBD8F800000EF075
:104370000CF818B932200DF04AFFF6E74FFA89F031
:1043800003F036FF00200EF07DFBFFF7A0B95C4B79
:1043900098590DF0FAFF18B932200DF038FFF6E702
:1043A0000EF07CF904F0C4FC564A574BDA60FFF774
:1043B0009AB90C283ED00A2845D1544D54480EF0E5
:1043C000E5FB2846232113F044F908B1401B206087
:1043D0002368002B5AD14D4800213022236013F06E
:1043E00002F9039B1B7843BB4A4B1B689B0614D501
:1043F000494B41491B688A6B9A1A002A0DDB474AD0
:104400001278042A09D903F5123303F5F873444AE4
:104410008B63D36883F01003D360424B9B68002BFF
:1044200067D04148984764E005F0B6FCFFF74FB904
:104430000C2804D13D480EF0A9FB3D480DE07F2833
:1044400012D1FFF7B0B80D28B7D07F2809D12F4A75
:10445000013B002137482360D1540EF097FBFFF752
:10446000A2B82F2B3FF69FA8A0F12002D2B25E2A5D
:104470003FF699A813B920283FF495A85A1C22604A
:10448000224AD0540EF07AFBFFF78DB85A1EA95C71
:10449000202901D113469CE71C4A00212360D154F6
:1044A000254B264DD3F80090D5F800A0DFF85C80AE
:1044B000504613F0DCF8064651463246404613F0AB
:1044C000DFF81F4A28B918F806304B445B785807C4
:1044D00003D010359542E7D306E0954204D2701C14
:1044E000EB684044984702E016480EF04FFB00236B
:1044F00071E709B0BDE8F08F380F002070C60108E1
:104500009C1100200400FA0500ED00E09C2400202E
:1045100028D20108A0100020C0330020AA100020DB
:10452000000C01404C120020740F0020DDC2010875
:10453000D8C2010804C301086800002018AB0108B4
:10454000F8AC0108E8C20108F02900202DE9F04785
:104550004B28A0B0044600F0378600F2B480302823
:1045600000F0C28651D8222800F0838423D8032883
:1045700000F0608114D8012800F05081022840F03A
:104580001E8704200EF07EFA43200EF046FA4C20DF
:104590000EF043FA46200EF040FA4C2000F048BEE0
:1045A000042800F05181052840F009871A200EF0F8
:1045B00069FA00245BE1282800F0D48515D8242866
:1045C00000F0BB85262840F0FA86B54C06200EF098
:1045D00059FAB4F85C010EF058FAB4F85E010EF026
:1045E00054FAB4F8600100F0A5BD2C2800F0CD8588
:1045F0002E2800F048862A2840F0E18601200EF09F
:1046000041FAA74B587900F013BE3D2800F0F38221
:104610001ED8362800F01D860BD8322800F00286FE
:10462000342840F0CC8648200EF02CFA002500F00B
:1046300042BC3A2800F0B3823B2800F013843828AB
:1046400040F0BD8604200EF01DFA954C00F07BBDB5
:10465000452800F0A18627D8402800F0EC854228A4
:1046600040F0AD868E4C10200EF00CFA60790EF002
:10467000D4F9A0680EF012FA94F892010EF0CDF978
:10468000B4F85C010EF001FAB4F85E010EF0FDF929
:10469000B4F860010EF0F9F9B4F882010EF0F5F902
:1046A000B4F8840100F046BD472800F05386C0F0FE
:1046B0004086492840F0838602200EF0E3F9784BCB
:1046C000988900F037BD702800F0E88258D8692832
:1046D00000F045822AD8652800F0FE8015D84D28C4
:1046E00000F08185642840F06A8607200EF0CAF940
:1046F000E7200EF092F96A4B58790EF08EF90020FF
:104700000EF08BF9042000F056BE672800F0AA8155
:1047100000F2188212200EF0B5F9624B00241B88BB
:10472000B3F5806F8CBF082501257EE16C2800F071
:10473000298217D86A2800F083846B2840F03F86CE
:1047400005200EF09FF9584B18880EF09EF9574B34
:1047500018880EF09AF9564B93F86E0000F001009D
:1047600000F066BD6E28524D00F0208200F26E828D
:1047700006200EF087F9E86D0EF090F94D4B0CE233
:10478000782800F07C8119D8742800F0B5830BD804
:10479000722800F01584732840F0118608200EF06E
:1047A00071F9012400F045BC762800F0698400F21C
:1047B000E7832F200EF066F93F4C4BE3A42800F06E
:1047C000858414D87B2800F0EB82A02840F0F78580
:1047D0000C200EF057F9394B18680EF05FF9384B82
:1047E00018680EF05BF9374B186800F0E4BDF1284B
:1047F00000F08181FE2800F09084F02840F0DF85F1
:104800002B4C04200EF03EF9236CB3F85A000EF046
:104810003CF9236CB3F8580000F08CBC03200EF078
:1048200031F900200EF0F9F820460EF0F6F80C20D1
:1048300000F0FEBC0EF026F901200EF0EEF80A2082
:104840000EF0EBF800F040BC06200EF01BF9412002
:104850000EF0E3F857200EF0E0F846200EF0DDF8F9
:1048600031200EF0DAF8184B187800F063BC174BC3
:10487000185D01340EF0D1F80B2CF8D10024144B44
:10488000185D01340EF0C9F8082CF8D10024114B42
:10489000185D01340EF0C1F8072CF8D100F08DBD81
:1048A000F02900201C0000201E11002020110020F3
:1048B000780F002074100020ABA00108E8F7FF1F5C
:1048C000ECF7FF1FF0F7FF1FE333002004C00108DF
:1048D00010C00108E5BF0108CC4C0B200EF0D2F847
:1048E00020880EF0D2F8608880B20EF0CEF8C84B67
:1048F0001B68C3F3C000C3F38002800040EA42009B
:10490000C3F340021043C3F3401240EAC20003F075
:10491000100318430EF0B9F8BE4B1A88636812F002
:10492000010F14BF4FF0020C4FF0000C12F0020FF9
:1049300002F0080814BF4FF0040E4FF0000E03F40D
:10494000475912F0040F14BF1027002749EA08093D
:1049500012F0400F03F4804814BF2026002649EAD5
:10496000080912F0100F03F4004814BF4FF400754B
:10497000002549EA080912F0200F03F4803814BF1B
:104980004FF48060002049EA080912F4807F03F4A4
:10499000003814BF4FF40061002149EA080912F4FD
:1049A000007F03F480289C4A49EA080903F40028A0
:1049B00049EA0809127803F4801849EA080903F063
:1049C000007349EA0303C2F3800243EA020343EAA5
:1049D0000C0343EA0E0E4EEA070746EA070645EACD
:1049E000060540EA050041EA00014FF000000346D9
:1049F00014BF4FF400184FF0000841EA0808217A6C
:104A00008B420BD2854A9C5C012202FA04F414EA20
:104A1000080F1CBF9A4010430133F1E70EF03EF837
:104A20007F4B93F8B40700F003BC7E4B33F91400BE
:104A3000013490FBF5F080B20EF027F8032CF4D18E
:104A4000724CA08C0EF021F8E08C0EF01EF8208D38
:104A50000EF01BF8608D0EF018F8A08D0EF015F812
:104A6000E08D67E310200EF00DF800246E4B185D0A
:104A700001340DF0D2FF102CF8D100F09EBC702054
:104A80000EF000F800260E247443604D01362B6CA6
:104A90002344B3F819010DF0F8FF2B6C2344B3F84D
:104AA0001B010DF0F2FF2B6C2344B3F81D010DF038
:104AB000ECFF2B6C234493F81F010DF0AEFF2B6C21
:104AC000234493F820010DF0A8FF2B6C234493F8A6
:104AD00021010DF0A2FF2B6C234493F822010DF06D
:104AE0009CFF2B6C1C44D4F823010DF0D7FF082E3B
:104AF000C9D100F062BC70200DF0C4FF484C04F135
:104B0000700594F8D4000DF088FF94F8D5000DF0EE
:104B100084FF94F8D6000DF080FF94F8D7000DF0D4
:104B20007CFF94F8D8000DF078FF94F8D9000DF0D0
:104B300074FF073494F8D3000DF06FFFAC42E0D15E
:104B400000F03BBC10200DF09DFF0024374B185D9A
:104B500001340DF062FF102CF8D100F02EBC344D62
:104B600000242878400000F0FE000DF08BFF2B7829
:104B70009C4280F022842F4B33F814000DF085FF07
:104B80000134F4E72C4C06200DF07CFF20880DF05A
:104B90007CFF60880DF079FF284B1888CAE204205A
:104BA0000DF070FF194B186E00F005BC07200DF0DA
:104BB00069FF234B1888FF28A8BFFF20C0B20DF063
:104BC0002CFF204B186880F3100080B20DF05DFFC1
:104BD000B5F864000DF059FF114B93F887211A4B7B
:104BE000186822B10A23584380F3100001E000F353
:104BF0000F0080B29EE20A4C02200DF043FF94F8B1
:104C0000DE010DF00AFF94F8DD0111E3780F0020BA
:104C1000A010002068110020E1330020810F002047
:104C2000F02900206E100020A80F0020BC0F0020EB
:104C300038120020CC290020882900207C10002078
:104C4000901000209C100020981000200B200DF0E8
:104C500019FFAB6E002618780DF0DFFEAB6E5878AA
:104C60000DF0DBFEAB6EC14C3344187901360DF00C
:104C7000D4FE032EF6D1A36ED8790DF0CEFEA36E2E
:104C800098780DF0CAFEA36ED8780DF0C6FEA36E1C
:104C900058890DF0FAFEA36E187AC9E2B34C1E20B3
:104CA0000DF0F0FE236C00251B78022B65D1236CE0
:104CB00005F1080253F82200AD490FF04DF912F04A
:104CC0009FFE80F30800C0B20DF0A7FE236CA94937
:104CD00003EB8503D86A0FF03FF912F091FE80F3E1
:104CE0000800C0B20DF099FE236C05F10E0253F8D6
:104CF0002200A1490FF030F912F082FE80F3080083
:104D0000C0B201350DF089FE032DD0D1072D236CE3
:104D100021D1586C96490FF01FF912F071FE80F303
:104D20000800C0B20DF079FE236C9149986C0FF029
:104D300013F912F065FE80F30800C0B20DF06DFEAD
:104D4000236C93F84C000FF0AFF812F059FE80F38B
:104D50000800C0B20BE02B4458780DF05EFE236CC7
:104D60002B44D87A0DF059FE236C2B44587D013525
:104D70000DF053FE0A2DC9D11FE3236C2B44587844
:104D80000DF04BFE236C2B44D87A0DF046FE236CBD
:104D90002B44587D01350DF040FE0A2DEDD10CE37A
:104DA0003C200DF06FFE0024704D04F108022B6CC6
:104DB000714953F822000FF0CFF812F021FE80B2B3
:104DC0000DF063FE2B6C6C4903EB8403D86A0FF083
:104DD000C3F812F015FE80B20DF057FE2B6C04F1F3
:104DE0000E0253F8220064490FF0B6F812F008FEE4
:104DF000013480B20DF049FE032CD5D1072C2B6C69
:104E000016D1586C5C490FF0A7F812F0F9FD80B28A
:104E10000DF03BFE2B6C5849986C0FF09DF812F08A
:104E2000EFFD80B20DF031FE2B6C93F84C000BE0DF
:104E3000234458780DF029FE2B6C2344D87A0DF0CA
:104E400024FE2B6C2344587D01340DF01EFE0A2CE9
:104E5000D4D1B2E214F8010F002800F0AE820DF0B8
:104E6000DCFDF7E701200DF00DFE404B1B6C1878C0
:104E7000DEE150200DF006FE00253C4B0C211C6CA1
:104E80003E4B04EB850494F87920013501FB023395
:104E900093F838000DF0C1FD94F87A000DF0BDFDD7
:104EA00094F87B000DF0B9FD94F87C000DF0B5FD91
:104EB000142DE2D181E22D4B1C6C062303FB05442B
:104EC00094F8CE000DF0A9FD94F8C9000DF0A5FDF1
:104ED00094F8CA000DF0A1FD94F8CB000DF09DFDF3
:104EE00094F8CC000DF099FD013594F8CD000DF04B
:104EF00094FD0C2DDFD160E24FF000080126002761
:104F00001A4B1A7A974227DA0933FA5C00240C23E9
:104F100063431A4D05F13001595C914207D12B448E
:104F2000586B12F0A4FB82462EB9B14605E001345D
:104F30001B2CECD10EE080440CE0D1450ADA0C23A6
:104F400003FB04535B6B13F809000DF066FD09F1D8
:104F50000109F2E70137D3E7002E00F02E825FFA55
:104F600088F00DF08FFD0026C9E700BF780F002004
:104F7000000020410000C84200007A44ACA00108B3
:104F8000CC4D0024287A0DF07DFD2B7A9C4280F0D8
:104F90001482C94B0021E65C0C2202FB01F3C748D6
:104FA00000F13007DA5DB24205D1034493F83800CE
:104FB0000DF033FD02E001311B29EDD10134E4E7AE
:104FC000BF4C16200DF05EFDB4F898010DF05DFDAC
:104FD000B4F844010DF059FDB4F846010DF055FD4B
:104FE000B4F848010DF051FDB4F8DA010DF04DFDB3
:104FF00094F8EB010DF011FD00200DF00EFD94F87A
:10500000EC010DF00AFD94F887010DF006FD94F80F
:1050100094010DF002FD00200DF0FFFCA54B0A20CD
:105020001B6CB3F9563093FBF0F080B20DF02DFD00
:1050300089E0E0B201340DF0F0FC092CF9D1BCE1BB
:1050400010200DF01FFD9F4B9F4C187800F00200C0
:105050000DF0E3FC9D4B18780DF0DFFC20680DF09F
:105060001DFD60680DF01AFD994B18880DF00DFDBF
:10507000984B18880DF009FD8E4BB3F86C0059E081
:105080000DF0AEFC074612200DF0FCFC894C17B960
:10509000266F656F05E0102F19BF00252E46A66FFD
:1050A000E56F38460DF0B9FC30460DF0F7FC2846A8
:1050B0000DF0F4FCD4F880000DF0F0FC00200DF0B1
:1050C000E4FC00200DF0E1FC0020B1E0794D00246B
:1050D00095F884002E4680000130C0B20DF0D2FC5D
:1050E00095F884000DF099FC96F884309C4280F08D
:1050F0006481794D285D0DF090FC05F11003185D79
:105100000DF08BFC05F12003185D30350DF085FCAA
:10511000285D0DF082FC0134E6E708200DF0B2FCBA
:1051200000200DF0B2FC00200DF0AFFC00200DF0CF
:10513000ACFC00200DF0A9FC3FE104200DF0A2FC26
:105140005F4B986837E194F87C010DF066FC94F8A9
:1051500080010DF062FC94F87F010DF05EFC94F884
:10516000810165E0564C07200DF08CFCB4F88201FB
:105170000DF08BFCB4F884010DF087FC94F88601E7
:105180000DF04BFCB4F88801D4E74D4C0C200DF029
:1051900079FC94F892010DF040FCB4F89C010DF0FC
:1051A00074FCB4F898010DF070FCB4F89A010DF09D
:1051B0006CFC94F893010DF030FCB4F89E010DF0F6
:1051C00064FCB4F8A001B5E73D4C04200DF05AFC96
:1051D00094F8D8010DF021FC94F8D9010DF01DFCD4
:1051E000B4F8DA01A6E73D4C3D4D2078002600EBEF
:1051F0004000C0B20DF046FC237802359E4280F09C
:10520000DC8015F8020C0DF008FC15F8010C0136D5
:1052100000EB800000EB800000F2EE2080B20DF089
:1052200034FCE9E701200DF02DFC254B93F89401A7
:105230000DF0F3FBC1E008200DF024FC0024204B0E
:10524000234493F88A0101340DF0E7FB082CF6D1D2
:10525000B3E0184B1A4C93F8C50004F12805C0EBD5
:10526000C000C0B20DF00EFC94F8F20100231D4AFC
:10527000D25C904200F0A5800C333C2BF7D108346F
:10528000AC42F1D199E040200DF0FCFB0C4C04F154
:105290004005B4F8AC020DF0F8FB94F8AE020DF046
:1052A000BCFB043494F8AB020DF0B7FBAC42F0D178
:1052B00083E000BF780F0020810F0020ACA0010820
:1052C000F0290020A4100020AC100020AA1000201B
:1052D000A8100020A6100020FD0F0020381200208A
:1052E000922B002008130020E0200DF0CBFB424C55
:1052F00004F18005B4F82E02043400F03F000DF0F4
:10530000C4FBB4F82A02C0F386100DF0BEFB94F87B
:10531000280200090DF081FB94F8280200F00F002C
:105320000DF07BFB94F829020DF077FBAC42E1D144
:1053300043E0324C0D200DF0A5FB09F00BFD0DF004
:105340006CFB20880DF0AAFBE0680DF0A7FB06F0CF
:105350008BFD30E00DF058FB054684200DF092FBEC
:1053600028460DF09BFB254BDC6805F18003A3422A
:105370008CBF641B802406F031FE28462246694615
:1053800009F01CFD05460024AC4216DA1DF80400A5
:105390000DF043FB0134F7E713200DF073FB0024FD
:1053A000174B185D01340DF038FB0B2CF8D10020A1
:1053B0000DF074FB00200DF071FB012018E00020BF
:1053C00016E00DF02AFBB4F8F4010DF05EFB94F842
:1053D000F6010DF022FB94F8F7010DF01EFB94F896
:1053E000F9010DF01AFB94F8F8010DF016FB46E7F1
:1053F00020B0BDE8F08700BFF02900200C0000209D
:1054000004C001086B4B6C4A2DE9F04F5E891468AB
:105410004FEA062AB4EB0A0A9C884FF000054FEACF
:1054200004481C894FF0000BA4FB0A6765EB0B0BCB
:1054300004FB0B77F40944EA476418EB04065C8824
:105440004FF000094FEAE7154FEAC438DC8849EB12
:10545000050787B0CDE90467A4FB0A6704FB0B7757
:10546000340A44EA076418EB04064FEA27259C89AE
:105470004FF0000949EB0507CDE90067AAFB046777
:1054800004FB0B77F40D44EA472414F5FA664FEA5F
:10549000E75545F10007B6F5FA6F77F10003CDE95E
:1054A0000267964666DADDE90489A4FB046704FB1B
:1054B00005F34FF0050C07EB4307A6FB0C230CFB91
:1054C00007335F104FEA3206B8EB06084FEA920640
:1054D00046EA837669EB07099F10DDE90023921BFA
:1054E00063EB0703CDE90023DDE90267334A4FF0A0
:1054F000FF33964277EB0303CDE9048927DA40F6C0
:10550000AC520023A4185D4104FB05F3A4FB044541
:105510006FF0060205EB4305664202FB0566A4FB3D
:105520000223334418EB020649EB0307CDE9046775
:105530000B26A4FB062306FB0533DDE900455B10C3
:105540004FEA3202A41A65EB0305CDE90045DDE917
:1055500002450AFB0BF3AAFB0AAB0BEB430B4FEA2A
:10556000DA7242EA4B02A41A4FEAEB7365EB0305C9
:10557000CDE90245DEF80440009B019DA4FB032316
:1055800004FB05334FEA525848EAC3284FEA6359EF
:10559000DDE90423B8EB020269EB03039946D30B60
:1055A00043EA494300B1036009B1029B0B6007B0B5
:1055B000BDE8F08F6C1200204010002024FAFFFF9D
:1055C0002DE9F04FDFF8589285B00746D9F808006A
:1055D0000E460EF06DFC8E4C804620880EF064FC6A
:1055E0004FF05C51054640460EF0B6FC4FF064515A
:1055F000824628460EF0B0FC014650460EF0A2FB53
:105600004FF06251824640460EF0A6FC4FF06A51C0
:10561000804628460EF0A0FC014640460EF092FB64
:105620000546B4F902000EF043FC014628460EF090
:1056300093FC5146054650460EF08EFC8046B4F968
:1056400004000EF035FC014640460EF085FC014694
:1056500028460EF079FB80460EF044FE6D49054663
:10566000A06140460EF02CFDD9F80C30804628464B
:1056700001930EF01DFC4FF07C510EF06DFC66495D
:105680000EF060FB0546E389B4F90A0002930EF0C0
:105690000FFC29460EF060FC29460EF05DFC4FF031
:1056A00058510EF059FC8146B4F90800B4F810B016
:1056B000B4F80CA00EF0FCFB29460EF04DFC0146A0
:1056C00048460EF041FB4FF058510EF045FC4FF0AC
:1056D00060510EF041FC4FF07E510EF035FB8146DB
:1056E000E0880EF0E1FB014648460EF035FC002153
:1056F00081460EF0C5FD00287BD1294628460EF0D4
:105700002BFC03900FFA8BF00EF0D2FB039B0146AB
:1057100018460EF021FC4FF060510EF01DFC834640
:10572000BDF908000EF0C4FB014628460EF014FC3B
:1057300001460EF009FB014658460EF005FB4FF0FE
:105740007A510EF009FC834601980EF0B1FB014638
:105750004FF093400EF0F6FA05460FFA8AF00EF07D
:10576000A7FB4FF08F410EF0F7FB014658460EF0B5
:10577000EBFA4FF066510EF0EFFB014628460EF0B3
:10578000E1FA26490EF0E8FB49460EF099FC054681
:10579000B4F916000EF08CFB29460EF0DDFB29460D
:1057A0000EF0DAFB4FF040510EF0D6FB8146B4F913
:1057B00014000EF07DFB014628460EF0CDFB4FF0A5
:1057C00060510EF0C9FB014648460EF0BDFA814615
:1057D000B4F912000EF06CFB014648460EF0B4FA24
:1057E0004FF076510EF0B8FB014628460EF0ACFAA9
:1057F00000E0002017B10EF075FD38602EB1404674
:105800000EF070FD64235843306005B0BDE8F08FA2
:10581000CC1200200000A04500007A470050C3458C
:1058200040100020704770472DE9F041324C334D55
:1058300062892B8AB4F904809A1A2389B4F902E0A8
:105840005A43B4F91230D613B4F91420DB023244AF
:1058500093FBF2F232440A26E2615643A2F57A62E1
:1058600002FB02F3B4F90EC002FB0EFE02FB08F2CB
:10587000B4F90C801B130CFB03FC03FB08F31B1493
:1058800003EB62320232E388921002F50042534386
:105890004CF25032B4F920704FEAEE2EB4F90040C9
:1058A0000EEBEC2C0CEB8404BC406D690234A5EBD0
:1058B000A4043A4162434FEAD3384EBFB2FBF8F337
:1058C0005400B4FBF8F340F6DE3448BF5B001A1214
:1058D000524362430A4C08365C43241404EB2242D0
:1058E00002F6CF62361103EB221300B1036001B15F
:1058F0000E60BDE8F08100BF801200204010002043
:1059000043E3FFFF024B4FF480521A80704700BF01
:105910001C0000207720482101220CF0FDBA7720DE
:10592000582101220CF0F8BA7620F42131220CF033
:10593000F3BA074B002193F82020064B9201343232
:1059400019767720F42102F0FC020CF0E5BA00BFD2
:105950008012002040100020034B00221A7677208E
:10596000F4212E220CF0D8BA4010002008B50F21E7
:10597000082218200CF0D0FA0E22182010210CF06A
:10598000CBFA024B4FF480521A8008BD1C00002055
:1059900008B5134B53201B782D2108227BB10CF046
:1059A000BBFA31210A2253200CF0B6FA2C210C222A
:1059B00053200CF0B1FA53203821902209E00CF06A
:1059C000ABFA31210A2253200CF0A6FA53202C21E5
:1059D0000A220CF0A1FA40F20912024B1A8008BD0B
:1059E000681200201C00002007B5002101AB032233
:1059F00077200CF051FA9DF805309DF804001B0249
:105A000043EA00439DF80600184303B05DF804FB29
:105A100008B5FFF7E9FF014B586008BD40100020B2
:105A200008B5FFF7E1FF014B186008BD40100020EA
:105A300007B5F7216B46062276200CF02DFA9DF86B
:105A400000309DF801101B0343EA01139DF802107A
:105A5000094A43EA1113D3609DF803309DF80410FE
:105A60001B0343EA01139DF8051043EA11139360E9
:105A700003B05DF804FB00BF4010002013B5104CCC
:105A8000237E1BB9638B0133638316E0032201ABD2
:105A90007720F6210CF000FA9DF805309DF80420DF
:105AA0001B0243EA02439DF806201343054AB2F95C
:105AB0002020C2F10802D340636102B010BD00BFD4
:105AC000401000208012002013B50B4C237E1BB920
:105AD000638B013363830CE0022201AB7720F62154
:105AE0000CF0DAF99DF804209DF8053043EA022312
:105AF000238202B010BD00BF4010002013B5062263
:105B00000446432168206B460CF0C6F9A0B19DF80D
:105B100000209DF8013043EA022323809DF80220F3
:105B20009DF8033043EA022363809DF804209DF82A
:105B3000053043EA0223A38002B010BD13B506224C
:105B400004463B2168206B460CF0A6F9A0B19DF8F5
:105B500000209DF8013043EA022323809DF80220B3
:105B60009DF8033043EA022363809DF804209DF8EA
:105B7000053043EA0223A38002B010BD13B5012211
:105B80000DF1070304461A2168200CF085F99DF8F1
:105B9000073003B10123237002B010BD13B50222F8
:105BA000044601AB1B2168200CF076F99DF8042017
:105BB0009DF8053043EA022303F54E534FF48C72EF
:105BC000103393FBF2F32333238002B010BD13B5DF
:105BD00004466B461D21062268200CF05DF99DF8F5
:105BE00000209DF8013043EA022323809DF8022023
:105BF0009DF8033043EA022363809DF804209DF85A
:105C0000053043EA0223A38002B010BD13B506227B
:105C100004466B4601211C200CF03EF99DF8013032
:105C20009DF80020042143EA022242F38D0292FBF8
:105C3000F1F29DF8023022809DF8032042EA03220F
:105C400042F38D0292FBF1F29DF8043062809DF8E0
:105C5000052042EA032343F38D0393FBF1F3A38072
:105C600002B010BD13B504466B460221062218206F
:105C70000CF012F99DF800309DF801209B0803EB11
:105C8000022323809DF802309DF803209B0803EB3C
:105C9000022363809DF804309DF805209B0803EBE8
:105CA0000223A38002B010BD2E4B2DE9F3411B78D7
:105CB0000546002B38D0002426462746A046082259
:105CC0006B46532032210CF0E7F89DF801209DF837
:105CD0000030013403EB02231BB29DF803209844EB
:105CE0009DF80230E4B203EB02231BB21F449DF87F
:105CF00005209DF80430202C03EB02231BB21E4428
:105D00009DF8073003F07F0301D0002BD7D198FB1B
:105D1000F4F897FBF4F796FBF4F6134BA5F8008024
:105D20006F80AE801C771AE006226B46532032212A
:105D30000CF0B2F89DF801209DF8003003EB02232F
:105D40002B809DF803209DF8023003EB02236B802B
:105D50009DF805209DF8043003EB0223AB8002B0D0
:105D6000BDE8F081681200204010002008B54FF413
:105D7000804008F04BFB012801BF044B4FF48042E8
:105D80005A61034B08BF187608BD00BF00040140EC
:105D90004010002010B5054C2368186908F036FB48
:105DA00018B123681A69024B5A6110BD64120020B1
:105DB0000004014013B501220DF107033A21044606
:105DC00068200CF069F805200CF016FA9DF80730F1
:105DD00003B10123237002B010BD13B500222A21A4
:105DE0001C200CF099F80E2102221C200CF094F8D3
:105DF0000F2103221C200CF08FF82B2112221C20D3
:105E00000CF08AF8164A02249369164843F00403FA
:105E100093612023ADF8043004230DEB03018DF8CA
:105E200006308DF8074008F05CFE22462C211C202D
:105E30000CF072F82D2101221C200CF06DF82E219F
:105E400000221C200CF068F82A2105221C200CF0EE
:105E500063F8054B4FF480721A8002B010BD00BF8A
:105E600000100240000801401C000020F8B50F4659
:105E70001646074C4FF48055656140F080000DF0E8
:105E8000AFF83846002132460DF074F82561F8BDB0
:105E9000000C014013B501220DF107010446382022
:105EA000FFF7E4FF05200CF0A7F99DF8073003B1D8
:105EB0000123237002B010BD13B504466946432088
:105EC0000622FFF7D3FF9DF800209DF8013043EA3A
:105ED000022323809DF802209DF8033043EA022329
:105EE00063809DF804209DF8053043EA0223A380D7
:105EF00002B010BD13B5044669463B200622FFF7E9
:105F0000B5FF9DF800209DF8013043EA022323806D
:105F10009DF802209DF8033043EA022363809DF838
:105F200004209DF8053043EA0223A38002B010BD8F
:105F300070B50E46054C4FF4805565610DF050F874
:105F400030460DF04DF8256170BD00BF000C0140DA
:105F50001D4B07B51A681D4B9A420ED14FF40053E2
:105F6000ADF8043002238DF80730042318480DEBF8
:105F700003018DF8063008F0B4FD80216B20FFF797
:105F8000D7FF64200CF043F900216B20FFF7D0FF0E
:105F900064200CF03CF96B200121FFF7C9FF1B20A6
:105FA0001821FFF7C5FF1C201021FFF7C1FF094B87
:105FB0001A201978FFF7BCFF19200021FFF7B8FF5E
:105FC00003B05DF804FB00BF2C000020001BB700ED
:105FD0000010014026000020F0B5254D85B06B7FF4
:105FE000002B43D1234C2368002B3FD01A68224E4C
:105FF00012B1B1690A43B2619A889868ADF800207D
:1060000002228DF80320694604228DF8022008F050
:1060100068FDB369002743F00103B36123680126DB
:10602000197D187B08F048FD14480CF099F9236895
:10603000134A1B695361029308230DEB03008DF88B
:106040000D308DF80C708DF80E6008F0AFF92368F4
:1060500001A85B7D8DF806708DF8043003238DF860
:1060600005308DF807600CF067FF6E7705B0F0BD66
:10607000401000206412002000100240955D0008CE
:106080000004014008B5FFF7A7FF6B2180226820BC
:106090000BF042FF64200CF0BAF86B210322682059
:1060A0000BF03AFF0F200CF0B2F8124B19211A78BE
:1060B00068200BF031FF0F200CF0A9F80E4B1A21CD
:1060C0001A7868200BF028FF1B21182268200BF09B
:1060D00023FF1C21102268200BF01EFF3721022213
:1060E00068200BF019FFBDE8084068203821012224
:1060F0000BF012BFE81200202400002008B5FFF7C3
:106100006BFF074B1B7813B1012B03D008BD4FF475
:10611000006201E04FF48052024B1A8008BD00BFBC
:10612000691200201C00002008B519200CF06FF83F
:106130006820152100220BF0EFFE10B903200CF0AF
:10614000D9F80C4B16211A78682042F018020BF08F
:10615000E3FE1721002268200BF0DEFE3D21012224
:1061600068200BF0D9FEBDE8084068203E210122DE
:106170000BF0D2BE250000200BF01ABD0BF040BE84
:106180000BF016BD0BF03CBE73B51D4CA37F53BB8B
:106190001C4A1D4D93694FF4805643F008039361E8
:1061A00010238DF806302846032301A98DF8073007
:1061B000ADF8046008F095FC144A2E61138823F0B2
:1061C00040031B041B0C1380138823F038031B04AB
:1061D0001B0C43F00803138013889BB243F0400369
:1061E00013800123A377752001A90122FFF73EFE4A
:1061F0009DF80400A0F170035842584102B070BDF0
:106200004010002000100240000C01400038004007
:1062100007B523200BF0FBFF6820752101220DF14B
:1062200007030BF039FE28B19DF80700A0F16803C1
:106230005842584103B05DF804FB00BF2DE9FF4709
:10624000C54C07462378C54E002B00F0DA81326832
:106250006368D31A7C2B40F2D481237A62600133C5
:1062600023724FF0000808F12400BB4DC0B206F0C5
:10627000A1FF05F10A0333F918000DF019FEB84B20
:10628000814618880DF014FE014648460DF018FFAF
:10629000B4490DF061FE0EF025F808F1010800B2D6
:1062A00006F076FFB8F1030FDDD1302006F082FF53
:1062B000B5F9100006F06CFF06F074FF2B7A9A0710
:1062C0002CD141F288336A689A4218D9102006F01E
:1062D00071FF68694FF0640890FBF8F000B206F0B7
:1062E00057FF212006F066FF686990FBF8F308FB72
:1062F00013000028B8BF404200B206F049FF142046
:1063000006F058FFB4F9180006F042FF1C2006F012
:1063100051FF002006F03CFF06F044FF237ADFF82F
:1063200038825B0740F04A81022006F043FFD8F82C
:106330001C006423323090FBF3F000B206F028FF1B
:10634000B8F926504FF0050A95FBFAF5032006F040
:1063500031FF854BADB21B78DFF8209213F0040FAC
:106360000BD038460DF0ADF828B9D9F8003013F04D
:10637000100F18BF002528B205E0D8F828309889FA
:10638000B0FBFAF000B206F003FFD9F800309F0727
:1063900065D5DFF8EC91A28D99F800304FF06408D4
:1063A00008FB02325B00B2FBF3F3E78D06203F01EE
:1063B000BFB247EA0327BFB2C3F303231F4306F06C
:1063C000F9FE38B206F0E4FEE38D99F800100133CF
:1063D0009BB293FBF1F201FB1233E385236B5E4D1D
:1063E0009B7B012B05D1392006F0E4FEB5F92C008A
:1063F00019E0AD8D6E235D43152795FBF7F53A2027
:10640000AFB206F0D7FEB7FBF8F528B208FB15755A
:1064100006F0BEFE3B2006F0CDFEA8B2451D0A20C8
:1064200095FBF0F000B206F0B3FE282006F0C2FEA5
:10643000636B0A2093FBF0F000B206F0A9FE042083
:1064400006F0B8FEA36A9B8913B108F01FF903E0B8
:10645000414B986B80F3100000B206F099FEE36B9D
:106460003D4F9D0640F19F8097F8403098071DD51D
:10647000112006F09FFEB7F842004FF4F365684321
:106480003A4B90FBF3F000B206F082FE192006F0C2
:1064900091FEB7F842004543642095FBF0F595FB6B
:1064A000F0F300FB135000B206F072FE94F8403097
:1064B000B4F8445013F0020F08BF0025012006F085
:1064C00079FE28B206F064FE092006F073FE002073
:1064D00006F05EFE264B94F846501A88B2F5967F79
:1064E0000AD91D4B1B7A03F00F03072B04D842F285
:1064F0000F75954228BF1546052006F05BFE236BFD
:106500005B7B0BB928B216E0A5F120000DF0D0FCA2
:1065100018490DF0D5FD002105460DF0BBFE10B960
:106520004FF07C5101E04FF03F4128460DF00CFC4C
:106530000DF0D8FE00B206F02BFE94F84020064B7A
:10654000910703D493F84720012A1BD1012384F833
:10655000473009482EE000BF64100020B429002015
:106560001C00002000007A44E1330020A0860100D6
:10657000560000206666E63FAC10002090290020FF
:10658000540000201D6BBD4968680DF0E5FC0DF05E
:10659000A9FEBA490290A8680DF0DEFC0DF0A2FE3B
:1065A000039002A806E0B64A02AB92E8030083E833
:1065B0000300184606F00EFE06F0F4FD237A282BA1
:1065C0001FD1B04B00221A7233684FF47A70B3FBBC
:1065D000F0F83C27172006F0EDFDB8FBF7F5B5FB0A
:1065E000F7F007FB1050000200B206F0D1FD1820B2
:1065F00006F0E0FD07FB158000B206F0C9FD06F0CD
:10660000D1FD94F850309F4D002B00F05A810BF0D3
:10661000D9FD6B6D9C4AC31A9342074640F2C28073
:10662000002385F85A3085F85C30AB8DDAB21B0A4E
:1066300085F8762085F8773085F86C2085F86D3000
:10664000D5F8842033689A1AD5F88830D97B4FF46E
:106650007A734B439A420ED38C4B1B68C5F8843037
:1066600095F88C30013B012B9FBF102385F85A30E1
:10667000022385F85C30626B0A20A36B92FBF0F278
:1066800093FBF0F384F87420121284F8752084F8D8
:10669000783094F840201B1284F8793094F8463012
:1066A0009207784984F8A73003D42D2381F8A830C5
:1066B00077E0D4F848907648DFF8E0C199FBF0FA2B
:1066C0000CFB0A924FF0060E042B0EFB02F28CBF5D
:1066D0003323322381F8A8306E4BE66C92FBF3F142
:1066E00096FBF0F003FB1122642592FBF5F20CFB04
:1066F000006C0EFB0CFE84F89920121284F89A208C
:106700009EFBF3F203FB12E393FBF5F30AEB8A0A19
:106710004FFA81F80AEB8A0A08EB8A0189B284F8F9
:10672000971000EB8000090A84F8981000EB8000B5
:1067300051B201EB800292B284F89C20120A84F8D4
:106740009D2084F89E30B4F842201B1284F89F30BC
:106750002423534393FBF5F5B4F8BA300A2284F8A6
:10676000A0301B0A84F8A130B4F844304FEAD9793C
:10677000B3FBF2F303F5FA739BB284F8A2301B0A61
:1067800084F8A330B4F8BC30F60F84F89450C5F305
:10679000072584F8969084F89B6084F8955084F8D7
:1067A000A930676594F8BE80364DB8F1000F0DD161
:1067B000D5F8C4000BF0F2FD012807D90228364EA7
:1067C00000F04F8206F0D6FC0123B370D4F8C82045
:1067D0002C4D002A75D095F8BE603EB140F6B73119
:1067E000D5F8D030FB1A8B4219D86AE00123D5F8CE
:1067F000C40085F8BE3001F0CFFDD5F8D4300821B3
:1068000093F9000002238DE8480032464FF4964386
:1068100001F0D6FD85F8D860C5F8C4004FE095F8C2
:10682000CC60CEB9D5F8C400C5F8C86085F8BE60A4
:1068300001F0B2FDD5F8D430082193F9000001230E
:106840008DE8480032464FF4964301F0B9FDC5F893
:10685000C40006F08FFC32E0013EF6B285F8CC6051
:1068600095F8D81095F8D930D6B94A1C013385F877
:10687000D82085F8D930D5F8C4001EE08096184B92
:106880002CA20108641000203F0D0300B429002051
:106890008096980040420F001C000020806967FF2E
:1068A00012F8016B01337018314685F8D800D5F81D
:1068B000C400C5F8C82085F8D9300BF072FDC4F8C3
:1068C000D07094F8DA309B4DDBB1D5F8DC30C3B131
:1068D000D5F8E030ABB1C5F8E4301B68964AC5F88E
:1068E000E830D5F8EC301344187AFDF72FFE0CF0A1
:1068F000A5F8D5F8EC300133092B88BF0023C5F883
:10690000EC308E4D94F8F0202E688A4B002A00F06F
:10691000E281D3F8F420002A00F0DD8193F8F8300A
:10692000013B012B00F2D781D4F8F400814F0BF02A
:1069300035FDE0B1D7F8F4000BF02DFD97F8F930F4
:1069400080467E2BD5F800900ED102231B2887F8B5
:10695000F83009D1D7F8F4000BF020FD20B901235D
:10696000C7F8FC9087F8003184F8F980DCE7D7F8A5
:10697000FC202B689B1A41F6583293421DD9032301
:1069800087F8F830A7E16E4A32F8130010B90346D1
:106990004FF403600133B0F5C06FDBB275D01DD981
:1069A000B0F5006F7AD031D9B0F5036F3ED184F8DD
:1069B0000131E36B5F4F99063FD494F8001194F8CE
:1069C0000131002900F04A812A68921B012ADAD994
:1069D00084F80131002384F800317CE1B0F5007FB8
:1069E00042D007D8B0F5807F47D0B0F5887F00F05F
:1069F0008380E6E7B0F5806F00F0A680B0F5826F87
:106A000000F0EB80B0F5047FDBD123E0B0F5E26F5E
:106A100000F08280B0F5E46F00F08380B0F5E06FA5
:106A2000CFD184F80131B4F90A107EE0B0F5046FDB
:106A30006BD0B0F5026FC4D1FAE097F840309A07F6
:106A4000BBD5B7F8421024234B436421123393FB88
:106A5000F1F1FDE084F801313A4B364F1B689B079A
:106A6000ABD5BB8D0A21F2E084F80131354B314FB3
:106A70001B681905A1D5796BEAE084F80131E36B55
:106A80002C4F5A0799D57969E2E084F801312D4BF2
:106A9000284F1B681B0590D5B96BD9E0E16B254ADF
:106AA0008F0684F8013188D592F84010880784D584
:106AB000D90710D5D36C192283EAE371A1EBE371F6
:106AC00001EB5101B1FBF2F1002BACBF41F00041F1
:106AD00041F040410DE0936C192283EAE371A1EB90
:106AE000E37101EB5101B1FBF2F1002BB8BF41F0B2
:106AF00080414FF400608AE084F80131E36B0D4F70
:106B00005B077FF55AAF3969A2E084F80131B4F927
:106B10001830642159437AE084F80131B4F90C103B
:106B200003E0B4F90E1084F801312C2391FBF3F14A
:106B30006DE000BF641000202CA20108B4290020E1
:106B40001CC401089029002084F8013194F8023116
:106B5000624A0133DBB2032B88BF012382F8023182
:106B600042F2107394F8021159435D4B1B78D80719
:106B700048BF01319A0748BF02315F07B4F80431BA
:106B800048BF0431D80748BF0A319A0748BF1431BB
:106B90001F0648BF2831D80548BF28315A0748BFCB
:106BA00064311F0748BFC831980548BF01F5C87157
:106BB0009A0648BF01F57A71DF0648BF01F5FA6110
:106BC000580648BF01F57A614FF4806000F0CCFDB3
:106BD000424B002283F80021EFE6E16BDFF8FC80F6
:106BE00011F0200784F8013117D098F8402012F0F6
:106BF000020F14BF4FF47A71002112F0010F14BF7D
:106C00004FF4FA6300230B4494F84610194400F043
:106C1000ABFD002384F80031CFE6324B1B68190628
:106C20007FF5CBAE394600F09FFD88F80071C4E6D1
:106C300084F80131E36B294F9A067FF5BEAE97F8D1
:106C400040309B077FF5B9AEB7F844306421594313
:106C500000F08AFD002387F80031AEE684F80131A8
:106C600039E0B37823B1C5F8C07086F80280ADE58D
:106C7000D5F8C030FB1AB3F57A6FFFF4A7AD012346
:106C8000D5F8C400B3700BF086FB0646D5F8C400F7
:106C90000BF081FB76067FF499AD8A2802D08E280E
:106CA0000CD093E5EB6B98067FF590AD95F8BE3070
:106CB000002B7FF48BAD05F18D0306E095F8BE3017
:106CC000002B7FF483AD05F15803C5F8C8302D23A0
:106CD00085F8CC307AE504B0BDE8F0876410002078
:106CE000E133002090290020344B354A1B6812689C
:106CF00010B51A60334A11685960516892689960FA
:106D0000DA60314A116819615168926859619A6173
:106D10002E4A1168D9615168926819625A622C4AE8
:106D200011881985518859859188D2889985DA8585
:106D3000284A118819865188598692889A86264A47
:106D40001188D986518892881987194621F83A2FD7
:106D5000224A10780022824206DA214C34F812408E
:106D6000013221F8024FF6E71E4A1288A3F8642088
:106D70001D4A1288A3F866201C4A1188A3F86C10DB
:106D800051889288A3F86E10A3F87020184A3B210E
:106D900012689A66174A126892FBF1F2B2F5967F72
:106DA000C8BF4FF0FF325A67134A1288A3F8782001
:106DB000124A5289A3F85E2010BD00BFEC310020BA
:106DC000C0330020502500205C25002068250020CD
:106DD000841000209C0F00206E100020242800202A
:106DE000BC0F0020D02300205C0F0020A20F002049
:106DF0007810002000000020DC0F0020A80F0020E9
:106E00002DE9F84305460E460D4B002493E8800318
:106E1000B44213DA7B1933F9140008EB050333F994
:106E2000142009EB050333F9143001341344022212
:106E300093FBF2F3C01A0AF0E6F9E9E7BDE8F8833C
:106E4000EC31002010B5134B014693F8DC37012BD1
:106E500019D1114B114C1878421CD2B21A7012067B
:106E600044BF00221A700E4A1B78127821549342B4
:106E700036BFC2F180029B1A9B183F2B09D9BDE88F
:106E8000104005F0C7B8074BBDE8104018680BF07C
:106E900088BA10BDF029002050260020522600207C
:106EA00051260020D431002070B54720FFF7CAFFDB
:106EB000174B1B681B0307D5164B174A5B681068F6
:106EC0001B68C01A0AF08FF9144E154C154D307816
:106ED0000AF089F923682868C01A0AF094F96368EF
:106EE0006868C01A0AF08FF90F4B18880AF07BF90E
:106EF0000E4B18880AF077F90D4B18880AF073F9D1
:106F0000337823742B68A3606B68E36070BD00BFA7
:106F100070330020EC310020C0330020AA10002084
:106F2000D8310020AC100020A8100020A6100020AE
:106F3000E40F00207FB5254C254E264D2649274AD3
:106F4000274B20B127480088B0F5805F30D23088C9
:106F500089791278ADF8040028781C4D1B788DF8DB
:106F600006008DF807108DF8082001A82946062292
:106F70008DF8093010F01CFB28B30198BDF80830DB
:106F80002860AB805320FFF75DFF20880AF02BF9C3
:106F9000A0780AF028F9E37801A8019323790293F5
:106FA000637903930AF084F80E4B00221A800AE0FA
:106FB000308889792080127828781B78A070E17059
:106FC00022716371DEE704B070BD00BF6C11002058
:106FD00068110020A4100020AC0D0020DB0D002063
:106FE000400E0020903300200A4A1388013313809A
:106FF000094A136801331360084A138801339BB2AE
:10700000202B01BF00231380054A138808BF0133DA
:107010001380704790330020783300207C330020A9
:107020007E33002038B5394B05461B780C46083BAB
:10703000012B6AD84520FFF705FF2846FFF702FF1E
:107040000C2D23D004D80A2D0AD014D835B138BD60
:107050000E2D4BD02ED3FF2D50D038BD206849E0E7
:107060002078FFF7EFFE62796378002A14BF802052
:107070000020184300E02078FFF7E4FEA078FFF737
:10708000E1FEE078FFF7DEFE20793BE0B4F9000096
:107090000AF09EF8A078FFF7D5FEE078FFF7D2FE61
:1070A000B4F904000AF094F8B4F90600BDE83840D9
:1070B0000AF08EB8637820788BB180F08000FFF7FB
:1070C000C1FEA468E0B2FFF7BDFEC4F30720FFF7DE
:1070D000B9FEC4F30740FFF7B5FE200E12E0FFF73C
:1070E000B1FE6068BDE838400AF08DB820680AF04B
:1070F0007AF86068BDE838400AF075B804480AF0CC
:1071000086F80020BDE838409CE638BDD03100202C
:107110003CC401082DE9F04FBE4B8BB01A88019397
:10712000BD4F002A40F0A98042F20103B7F8DA0708
:10713000BA4EC21A50425041FFF7FCFEFFF7D4FD91
:10714000346849202546FFF77DFEB54B04F11C0944
:1071500018680AF048F855F8040B0AF044F8284675
:1071600002F08EF804F1100002F08AF84FF01008D7
:10717000AC4D01232A6803FA08F3134203D0D9F86F
:1071800000000AF040F808F10108B8F1130F09F106
:107190000409EDD104F1280002F062F8B7F8443197
:1071A000B4F92E00C01A0AF01EF82B68DB0408D5CB
:1071B0009D4BB4F864001B88181AC0F30D000AF048
:1071C00012F82B68980403D5B4F866000AF00BF89F
:1071D0002B68590503D504F16C0002F041F82B68C7
:1071E0001A0502D5A06E0AF00EF82B685B0402D5D2
:1071F000606F0AF008F82B68180403D5B4F878001B
:1072000009F0F1FFA04604F1300002F029F804F182
:10721000360002F025F8B7F8443138F93C0F012761
:10722000C01A09F0E0FF814B1B789F4208DA38F959
:10723000020FB4F93C300137C01A09F0E4FFF2E75D
:107240002B68990505D5B4F95E00A0F2DC5009F071
:10725000DAFF326876487260B260121A9110754A8D
:107260004A43531C032293FBF2F202EB42029A1AA6
:107270007C2303FB02033360D6E16F4B6F4A1B682C
:1072800011688B4206D00AA941F8203D0020136006
:10729000FFF7C8FE019B97F8DA171B8897F8DB0702
:1072A0000B44013BB3FBF0F200FB12338B4280F046
:1072B00086815A4F0120FFF73DFEFFF715FD502054
:1072C0003E687D68FFF7BEFDBA683B6810681B68C2
:1072D0007A680344106806F11C0BA3EB400009F028
:1072E00092FF6A68736802A89B1A0293AA68B3683F
:1072F00005F11C089B1A0393EA68F36810249B1A93
:10730000049301F0BDFF2A69336902A89B1A029316
:107310006A6973699B1A0393B369AA699B1A0493F8
:1073200009F0C6FE3F4901220B68A2401A428A4674
:1073300006D0DBF80000D8F80030C01A09F063FF6F
:107340000134132C0BF1040B08F10408EAD106F107
:10735000260005F12601002331F9024F30F9022FF2
:10736000121B02AC44F823200133042BF4D1032177
:107370004FF000094FEA89035FFA83F902AB53F833
:1073800021206AB102F108000F2802D849F0010952
:1073900006E08032FF2A94BF49F0020949F0030950
:1073A00011F1FF31E6D248460024FFF74BFDA0461D
:1073B0000DF1080B09F00302022A16D0032A1DD092
:1073C000012A4ED1B8F1000F05D1DBF800409046FC
:1073D0002401E4B245E0DBF800004FF0000800F0C3
:1073E0000F002043FFF72EFD3BE0B8F1000F0CD05B
:1073F000DBF80000C0F3031020432CE0B8F1000FCD
:107400001ED19BF80100FFF71DFD9BF80000FFF760
:1074100019FD26E07C330020F0290020EC3100200B
:1074200078330020703300206C33002024280020A3
:10743000F8310020DF7BEFBD843300208033002053
:10744000DBF80000C0F303302043FFF7FBFCDBF860
:107450000000C0F30710FFF7F5FCDBF80040240143
:10746000E4B20BF1040B06AB9B454FEA9909A1D19D
:10747000B8F1010F02D12046FFF7E4FCDAF8003042
:1074800013F480541FBFB6F86420B5F864100124CB
:10749000521A18BF02929A040AD50AAA02EB840172
:1074A000B5F86600B6F866200134121A41F8202CAF
:1074B000580513D502AA02EB840C06F16A0E05F1F9
:1074C0006A0000223EF9021F30F9028FC8EB010169
:1074D0004CF822100132032AF4D10334190508D5DF
:1074E0000AAA02EB8400A96EB26E0134521A40F867
:1074F000202C5A0408D50AAA02EB8400696F726F27
:107500000134521A40F8202C18040BD50AAB03EBB7
:107510008402B5F87810B6F8783001345B1A42F876
:10752000203C00E0FCB1012C03D1029809F06BFE75
:1075300019E0631E002002AA52F823204000C0B2C6
:107540000AB140F00100013BF5D5FFF77BFC4FF09D
:10755000000802AB53F8280008B109F054FE08F106
:107560000108A045F5DB30200321FFF749FC362058
:107570000321FFF745FC2F4B3C201978FFF740FC17
:10758000DAF80030990506D5B6F95E00B5F95E3037
:10759000C01A09F038FE3A6827487B687A60121AE8
:1075A0009110264ABB604A43531C032293FBF2F21C
:1075B00002EB42029A1A7C2303FB02033B60204B3E
:1075C0001B681A0630D51F4C1F4D22682B689A4243
:1075D0000BD162686B689A4207D1019B1B88102B04
:1075E00011D11A4B1B885B060DD14820FFF72AFCEE
:1075F000206809F008FE606809F005FE23682B602A
:1076000063686B600EE0124A0F4B11782A7C91423E
:1076100008D1104A99681068884203D15268DB6823
:107620009A4201D0FFF740FC09F030FD0BB0BDE8F5
:10763000F08F00BF24280020F8310020DF7BEFBD51
:1076400090290020E80F0020D83100207E33002050
:10765000AA100020AC1000202DE9F84F0C9EC2EBC0
:10766000030B394C0B9B002914BF4FF0060A4FF057
:10767000040AF61A636805460133904613D123685D
:1076800053455ED2314A032B98BF294652F8232036
:107690002F4809F027FE63680022013363602D4BF9
:1076A00005469A7113E0002511E02B4A12789542A5
:1076B00040DA0B9BE3B109FB06F2995C01228A4098
:1076C000264909680A4213D1636801336360D4F81C
:1076D00004900A9B1C4F9945E7DB2BD10A20FFF74A
:1076E000B1FB3B6801333B604FF0FF337B6021E02F
:1076F000184A917921B12C20FFF7A4FB013501E054
:107700000121917109FB0BF3226808EB030752B9C1
:1077100058F8030009F07BFD97F9041005444B1C51
:10772000D2D00F4802E03A440E48117909F0DAFD50
:107730000544C9E7206850452CBF00200120BDE862
:10774000F88F0020BDE8F88F8833002040A20108A0
:1077500047C401086C110020640000207033002031
:1077600056C40108B9C7010830B585B004AC00257E
:1077700024F8025D0091ADF806002146102005F0C6
:10778000DBFC9DF80600214605F0D6FC9DF80700BD
:10779000214605F0D1FC9DF80000214605F0CCFC07
:1077A0009DF80100214605F0C7FC9DF80200214626
:1077B00005F0C2FC9DF80300214605F0BDFC9DF8D4
:1077C0000E002946C043C0B205F0B6FC05B030BD7E
:1077D000F8B504460E4617460025204620210FF036
:1077E00038FF0446D0B1013420460FF095FFB0F5C4
:1077F000617F05DB40F634039842A8BF184601E0DC
:107800004FF46170A0F56170192390FBF3F00DB98E
:10781000307000E070703B7801333B700DB901258A
:10782000DBE72046F8BD30B505460C461346294631
:107830002246BDE83040014801F0D6B84CC50108E9
:107840007FB504780646E4B9354B1921186800EB7A
:10785000840090F87B5090F879204D4305F56175D0
:1078600090F87A30009590F87C00414301F5617101
:1078700001912C482146013401F0B6F8142CE3D1D3
:107880004BE00FF049FF1328054641DC244B701CE8
:107890001C68202100238DF80F300FF0DAFE1E3512
:1078A000064670B1013630460FF036FF19289FBFEB
:1078B00004EB850358709DF80F30013398BF8DF8A5
:1078C0000F30304620210FF0C4FE064670B101365D
:1078D00030460FF021FF0D289FBF04EB8503987001
:1078E0009DF80F30013398BF8DF80F3004EB8504FD
:1078F0003046E11C0DF10F02FFF76AFF9DF80F30D3
:10790000042B0AD0601C002104220FF06CFE04E05E
:10791000054800211322FFF786FF04B070BD00BFA9
:10792000B80F00206BC5010880C5010801480BF0A5
:107930002DB900BF86C501082DE9F04304788FB04A
:107940000546002C59D17B4B0021142209A807AE13
:10795000D3F800800FF047FE0722304600210FF0D9
:1079600042FE00231A46A70005A8059308EB070569
:1079700083807149B5F802E031F813C01CEA0E0F9C
:107980000AD00E310DF1380C595C02F1010E62443F
:1079900002F81C1C5FFA8EF20133072BE9D100219B
:1079A0000B46664AB5F802E011F802C01CEA0E0F59
:1079B0000AD006320DF1380C8A5C03F1010E6344E3
:1079C00003F8242C5FFA8EF301310629E9D118F867
:1079D00007308DE841006A785949029209A81A09CE
:1079E00003F00F0300F0EBFF2146564809AA0134CB
:1079F00000F0FAFF202CA6D198E00FF08DFE1F2892
:107A0000044600F3868028462021E4B20FF021FED0
:107A10001F2C02D9FFF78AFF88E0464B451C1B68E4
:107A2000002103EB8404204604220FF0DCFD002734
:107A3000454B09AE304600210A2217F803905FFA41
:107A400087F80FF0D0FD002315F8012B32B10A2B77
:107A500004D04A4502D0F2540133F5E74A455ED1DD
:107A600008F1FF33032B09D8DFE803F01005023FCC
:107A70000DF1230134E00DF123011EE030460FF03B
:107A80004BFE2378C0B243EA001006E030460FF008
:107A900043FE237800F00F001843207031E00133DB
:107AA000062B0AD0244800F11B069E5D9642F6D1B3
:107AB00003445A7D63881343638011F8012F02B396
:107AC0000023EFE70133072B0AD01B4800F10E0615
:107AD0009E5D9642F6D130F813206388134363808D
:107AE00011F8012F6AB10023EFE730460FF014FEC2
:107AF0000F2804DC30460FF00FFE607001E0002319
:107B000063700137052F93D1012409F06DFC6CB926
:107B100080E70E4800211F22FFF785FE06E0204681
:107B2000002104220FF05FFD0024EEE70FB0BDE856
:107B3000F08300BF7411002058A201086DA2010853
:107B400094C50108A3C5010879A2010880C50108F0
:107B5000F8B50478064674B9304D2146B5F8C6210B
:107B6000B5F8C8312E48013400F03EFF042C05F171
:107B70000405F2D1F8BD2B490FF03EFDA8B9274B03
:107B80004FF47A714FF4FA62A3F8C611A3F8C82132
:107B9000A3F8CA11A3F8CC21A3F8CE11A3F8D021E1
:107BA000A3F8D211A3F8D421F8BD30460FF0B4FDEC
:107BB000032805462BD8304620210FF04AFD044605
:107BC00030B1013420460FF0A7FD0126074600E042
:107BD0000646204620210FF03CFD10B9BDE8F840D4
:107BE000A4E601300FF098FD012EF7D140F2DC53EE
:107BF000A7F2EE229A42F1D8A0F2EE229A42EDD8F4
:107C0000064B703503EB8503DF801881F8BD06480D
:107C100000210322BDE8F84005E600BFF02900205E
:107C2000AFC50108C2C5010870D301082DE9FF41A5
:107C300004780546002C34D16D480AF0A7FF6D4D3D
:107C4000686900210CF01CFB002840F0CE80214622
:107C5000694800F0C9FE6869694600F04BFD0146BD
:107C6000664800F0C1FEA869694600F043FD014680
:107C7000624800F0B9FEE869694600F03BFD014644
:107C80005E4800F0B1FE286A694600F033FD013419
:107C900001465B4800F0A8FE0C2C05F11005CFD181
:107CA000A3E0584905220FF0EBFC38B9514B0022F4
:107CB00003441030C0285A61F8D196E02846524952
:107CC00004220FF0DDFC04462846002C3FD1202181
:107CD0000FF0BFFC002800F08880451C28460FF0FC
:107CE000C6FC0746494B53F824601EB948480AF0C1
:107CF0004DFF7AE028463146FAB20FF0C1FC01345C
:107D00000028EFD13B4B0021C2181030C028516130
:107D10009E46F7D13F4B03EBC402D2F804C098460D
:107D2000BCF1000F04D131463B4800F05DFE53E04A
:107D3000002718F834309F42F5DA3B010EEB0305BB
:107D4000143563440FCB013785E80F00F1E70FF0DE
:107D5000E3FC0B28064643DC284620210FF079FC83
:107D6000054648B10135284600F02EFC214B012480
:107D700003EB0613586100E00446284620210FF06B
:107D800068FC054640B10135284600F01DFC194B42
:107D9000013403EB06139861284620210FF059FCAB
:107DA000054640B10135284600F00EFC114B013468
:107DB00003EB0613D861284620210FF04AFC10B9C6
:107DC000FFF7B4FD11E0013000F0FEFB094B032C7E
:107DD00003EB06163062F3D11048FFF727FF04E0EB
:107DE0000F4801210C22FFF71EFD04B0BDE8F08111
:107DF000C8C50108F0290020E3C50108E9C501084C
:107E0000CCD00108C2C50108EDC50108F8AC0108D5
:107E1000F2C501087CC4010801C6010807C30108B6
:107E200080C50108F0B5047887B0064614BB514BF5
:107E300019201968062303FB041191F8CA5091F820
:107E4000CE20454305F5617591F8C930009591F84C
:107E5000CB50C831684300F56170019008790290F9
:107E60004979454803912146013400F0BDFD0C2CB1
:107E7000DDD17CE00FF050FC0B28044672DC3D4B5A
:107E8000701C1D68202100238DF817300FF0E1FBD6
:107E9000064680B1013630460FF03EFC03289FBFF6
:107EA000062303FB045383F8CE009DF817309CBFD4
:107EB00001338DF81730304620210FF0CAFB0746FA
:107EC00080B1013738460FF027FC0D289FBF0623ED
:107ED00003FB045383F8C9009DF817309CBF01339E
:107EE0008DF8173006266643A9193846CA310DF1B8
:107EF0001702FFF76DFC20210FF0ABFB074670B1B6
:107F0000013738460FF008FC14289FBF9DF8173042
:107F10007619013386F8CC0098BF8DF817303846B3
:107F200020210FF096FB78B101300FF0F5FB0D2802
:107F30009FBF062303FB045383F8CD009DF8173041
:107F40009CBF01338DF817309DF81730062B0ED0EB
:107F5000062202FB04500021C9300FF044FBFFF75A
:107F6000E5FC04E0054800210B22FFF75CFC07B0AC
:107F7000F0BD00BFB80F00200DC6010880C5010884
:107F8000F0B5027887B08AB94A4C04F1280694F813
:107F9000F2210023484950B2595681426DD00C332A
:107FA0003C2BF7D10834B442F1D180E00022049296
:107FB0000592451C0FF0B0FBC4B260B20AF004F8A1
:107FC000074618B18DF81040012400E00446284609
:107FD00020210FF03EFB054638B1013528460FF051
:107FE0009BFB0134ADF81200E4B2002628462021A4
:107FF0000FF02FFBB0B3451C28460FF08DFB00227D
:108000002E495FFA82FE51F82230834204D00132B9
:10801000082AF5D1002300E0734651F8232082425C
:1080200020D1022E0FD0032E12D05A1E012ED2B212
:1080300004D0042A13D88DF814300EE0042A0ED888
:108040008DF8153009E0052B09D88DF8173004E0BC
:108050009A1E052A03D88DF816300134E4B2013691
:10806000042EC3D1052C03D807B0BDE8F0405DE471
:1080700004AB03CB3860796019E094F8F7010F4B3B
:1080800094F8F65153F82000B4F8F421009094F8D5
:10809000F90153F82000019094F8F80153F82000FA
:1080A00053F825300290064800F09EFC7AE707B0AE
:1080B000F0BD00BFF02900200813002044A70108EC
:1080C0002DC601082DE9F341047880464CB92046BD
:1080D00001A90BF0E5F90134FFF7F4FF122CF6D1FA
:1080E0006AE00FF019FBC6B2112E60D8344C06F1CD
:1080F000D00704EB470308F1010020219D780FF021
:10810000A8FA18B9AA1E5542554139E04378682BA0
:1081100006D0732B07D0612B13D14FF0000804E079
:108120004FF0010801E04FF00208A8F102035D42A0
:1081300000F101004FF020015D410FF08AFAD8B143
:1081400015B9FFF7F3FB37E001300FF0E5FA40F225
:10815000ED2380B2984205DD40F6CA039842A8BFDD
:10816000184601E040F2EE20A0F2EE20192290FB2A
:10817000F2F004EB4703D87004EB470383F8028066
:1081800004EB47040F4AA378134493F826204DB11B
:10819000E17819234B430C48314603F2EE2300F0FB
:1081A00023FC09E03146094800F01EFC04E00848C1
:1081B00000211122FFF737FB02B0BDE8F08100BFBC
:1081C000F029002058A201084CC601085EC601082B
:1081D00070D3010807B50123ADF8041001A98DF88B
:1081E00006208DF8073006F07CFC03B05DF804FB38
:1081F0002DE9F047814672B6514C4FF400774FF4A9
:1082000080616161204667614822FFF7E3FF3946DC
:1082100020461022FFF7DEFF1FFA89F6494A4FEA8F
:10822000C60802EB0803596852F83650464B4FEA2D
:10823000D10E05EB8E00586055F82E0001F00701B5
:1082400098608900D8600F208840C043D3F80CC0E4
:1082500052F839A000EA0C0CC3F80CC0D3F808C0DF
:1082600002EBC90900EA0C009860D8684FF0080CCE
:108270000CFA01FC4CEA0000D860D3F808C00120D9
:1082800000FA01F141EA0C019960996845F82E1055
:10829000D9F80410994600FA01F5CAF81050276180
:1082A0001746A3685805FCD4D9F80830D9F804203B
:1082B000082113604FF40073CAF814506361234B14
:1082C00019611021596140F60553A16849051AD476
:1082D000013BFAD1D9F80C3057F83600136007EBA0
:1082E00008025268C168012393400B43C3604FF4F6
:1082F000007113481822FFF76DFF62B6BDE8F04722
:10830000322009F084BF4822CAF810505046A9B262
:10831000FFF760FF0D4B10221A61A268084B52054F
:10832000C2D5DAF808204FF400701542074A4FF022
:10833000080115BF1861586111615161EDE700BF77
:108340000008014070C6010874110020000C0140B3
:1083500010B5044620460AF018F818B90A2009F0AA
:1083600056FFF7E710BD30B5094900220B78094CDC
:108370001557854202BFFF25155503F1FF3302F162
:108380000C0208BFDBB23C2AF1D10B7030BD00BF3C
:108390003D10002008130020002208490C2303FB95
:1083A00002135968814204D10022C2621A725A60D3
:1083B00070470132052AF0D1704700BF0813002032
:1083C0002DE9F743064689469DF8288011461A464E
:1083D0009DF82C3000250C2068431D4FC419C05750
:1083E000B04202D1207A20B12BE00135052DF2D127
:1083F00027E0022E0FD005DC56B1012E21D10093CB
:1084000014480AE01E2E0DD01F2E1AD1012009E0BB
:108410000093114801E011480093434602F0E0FE4A
:10842000044605E001F090FF4146044609F0AAFF2A
:108430004CB10C2303FB0575267185F808906C6020
:1084400001E0002000E0204603B0BDE8F08300BF5B
:10845000081300200044004000380140004800405C
:10846000F0B50124B0FBF4F58D4201D34C43F9E79C
:108470000026D4B1B0FBF4F504FB1500B4FBF1F415
:108480001EB9002D01DC002CF3D1092D03F1010EE2
:10849000EFB204DD002A14BF3725572500E0302550
:1084A0003D441D7001367346E3E71C70F0BDF0B526
:1084B0000124B0FBF4F58D4201D34C43F9E70026CB
:1084C000D4B1B0FBF4F504FB1500B4FBF1F41EB914
:1084D000002D01DC002CF3D1092D03F1010EEFB2C8
:1084E00004DD002A14BF3725572500E030253D4420
:1084F0001D7001367346E3E71C70F0BD03685A1C1B
:108500000260197070472DE9F843089E002B07465A
:1085100088461446334614BF4FF030094FF0200907
:1085200013F8012B0AB9254603E0002CFBDD013CC2
:10853000F6E7002D04DD38464946C047013DF8E71F
:10854000354624EAE474A01B284415F8011B11B138
:108550003846C047F7E7BDE8F883024B186809F0D2
:1085600020BF00BF680F0020F8B507460C464868DA
:10857000002115461E460BF083FE58B128460BF02D
:1085800097FC10490BF0E8FC01464FF07E500BF0D1
:1085900097FD6060616830460BF0D6FB01463046BF
:1085A0000BF08EFD25680646294638460BF0CAFBBF
:1085B000014630460BF0D0FC014628460BF0C4FBC8
:1085C0002060F8BDDB0FC9402DE9F0410278034679
:1085D000202A00F10100F9D0092AF7D02D2A02D172
:1085E0000346414D04E02B2A08BF03464FF07E5559
:1085F0001C460026234614F8012BA2F13007F9B2DD
:1086000009290DD8394930460BF0A6FC06463846F4
:108610000BF04EFC014630460BF096FB0646E9E7B0
:108620002E2A17D1314F234614F8010B3038C2B22D
:10863000092A0FD80BF03CFC39460BF041FD0146EE
:1086400030460BF081FB2949064638460BF084FC86
:108650000746E8E71A7802F0DF02452A39D15A784E
:108660002D2A02D10233012704E02B2A14BF013343
:1086700002330027013B002413F8012F303AD1B216
:10868000092903D80A2101FB0424F5E7B4F59A7FF0
:1086900028BF4FF49A74A0464FF07E53B8F1070FED
:1086A00007D9184612490BF057FCA8F108080346F1
:1086B000F4E704F0070434B118460C490BF04CFC05
:1086C000013C0346F7E719462FB130460BF0F8FCA2
:1086D00004E04FF07E5130460BF03EFC0146284648
:1086E0000BF03AFCBDE8F081000080BF00002041A3
:1086F00020BCBE4C30B5054687B00C4603A800210F
:108700000C220EF070FF284600210BF0E1FD20B195
:10871000284628490BF018FB03E0284625490BF0B2
:1087200011FB25490BF018FC0BF0DCFD054680EA37
:10873000E0706946A0EBE5700AF0B2FE002DACBF18
:1087400020232D2368468DF80C300EF090FF012871
:1087500007D130238DF80D308DF80E308DF80F30A5
:108760000CE0022805D130238DF80D308DF80E3045
:1087700004E0032804BF30238DF80D30694603A8B8
:108780000EF058FF03A80EF072FF0338C5B22A4658
:1087900003A920460EF096FF0023635520460749A3
:1087A0000EF048FF03AB204659190EF043FF204658
:1087B00007B030BD6F12033A00007A44A0C601082A
:1087C00070B50646B6FBF2F40846154614B12046CD
:1087D000FFF7F6FF05FB1464024B1B5D00F8013B3D
:1087E00070BD00BFA2C601082DE9F04F81468A4640
:1087F00016461C4689B000253178002900F0DB8040
:10880000252902D00136484674E072784FF00008FE
:10881000302A0CBFB278B71CA2F1300312BF4FF060
:10882000000BF71C4FF0010B092B19D8A2F13003F4
:10883000D9B2092905D80A2202FB083817F8012BFA
:10884000F4E7A2F16103052B02D8A2F1570305E07A
:10885000A2F14103052B03D8A2F137030A2BEADD6D
:108860006C2A30D13A787E1C642A00F083800BD8C1
:10887000252A3DD003D8002A00F09D80BCE7582A65
:108880000CD0632A19D0B7E7732A22D002D86E2AF7
:1088900037D0B1E7752A5CD0782AADD1271D206882
:1088A000A2F1580462424FF01001624155E02CD908
:1088B000582A32D0632A2AD13E4648462178271DBD
:1088C000D04701350FE0642A63D00ED9732A14D142
:1088D0003E46236848460093514642460023FFF730
:1088E00012FE271D05443C4686E7252ADFD13E4679
:1088F00048462521D04701357EE70AD86E2A06D1A1
:108900003E46236804341D6076E7002A53D03E4675
:1089100072E7752A26D0782AF9D1A2F1580304F11A
:10892000040C5A422068CDF80CC04FF010015A4197
:1089300005ABFFF795FDDDF80CC03E46644605AB80
:1089400000934846514642465B46FFF7DCFD05442E
:1089500052E72068271D0A21002205ABFFF7A7FD7B
:108960003C46ECE704F1040CCDF80CC020680A2169
:108970000022DDE72068271D002808DA2D238DF866
:10898000143040420DF115030A210022E6E705AB41
:10899000FAE7206804F1040C00280ADA2D238DF888
:1089A000143040420DF11503CDF80CC00A2100220D
:1089B000BFE705ABF8E7284609B0BDE8F08F0EB475
:1089C0000FB505AB53F8042B0190064901A803939A
:1089D000FFF70AFF019B00221A7004B05DF804EB58
:1089E00003B07047FD8400080FB413B50B4904AB06
:1089F00008680B4953F8042B09680193FFF7F4FE4C
:108A00000446084B186809F0C0FC0028F9D020463D
:108A100002B0BDE8104004B0704700BFDC00002089
:108A2000D8000020680F002080EAE073A3EBE07319
:108A30008B4206DB002801DD401A704702D0084453
:108A400070470020704770B504460BF04BFC203097
:108A5000402857D820462C490BF03AFC28B1204634
:108A60002A490BF06FF90446F4E7204628490BF039
:108A700011FC28B1204625490BF066F90446F4E7BD
:108A8000204624490BF024FC30B1224920460BF04B
:108A900059F901461F480AE020461F490BF0FAFB2E
:108AA00040B11C4920460BF04FF901461A480BF023
:108AB00049F90446214620460BF04EFA0546204669
:108AC00029460BF049FA1549064628460BF044FAA8
:108AD00013490BF037F9014628460BF03DFA1149CE
:108AE0000BF032F9014628460BF036FA0E490BF02E
:108AF00029F9014630460BF02FFA014620460BF0CB
:108B000023F970BD002070BDDB0F4940DB0FC94069
:108B1000DB0F49C0DB0FC93FDB0FC9BF9A7C2E3684
:108B2000FAAF4F393587083CA4AA2A3E08B5034955
:108B30000BF00AF9BDE8084085E700BFDB0FC93F2D
:108B40002DE9F04F056885B0814628460C46FFF7B1
:108B5000EDFF80462846FFF776FFD9F80450064619
:108B60002846FFF7E3FF07462846FFF76CFFD9F8D2
:108B7000089005464846FFF7D9FF82464846FFF76A
:108B800062FF4146814650460BF0E6F94146834676
:108B900048460BF0E1F95146019030460BF0DCF904
:108BA0004946029030460BF0D7F9394603905046BB
:108BB0000BF0D2F94946206007F100400BF0CCF9E8
:108BC00029466060A56002980BF0C6F9014601983D
:108BD0000BF0BAF82946E06003980BF0BDF90146A6
:108BE00058460BF0AFF83946206106F100400BF013
:108BF000B3F92946606158460BF0AEF90146039877
:108C00000BF0A0F82946A06101980BF0A5F90146E8
:108C100002980BF099F84146E06138460BF09CF958
:108C2000206205B0BDE8F08F2DE9F04107688AB0F9
:108C3000466885680446084601A9FFF781FF019947
:108C400038460BF089F90499804630460BF084F9D8
:108C5000014640460BF078F80799804628460BF00D
:108C60007BF9014640460BF06FF8029920603846C8
:108C70000BF072F90599804630460BF06DF901460C
:108C800040460BF061F80899804628460BF064F9DD
:108C9000014640460BF058F80399606038460BF0E7
:108CA0005BF90699074630460BF056F901463846FF
:108CB0000BF04AF80999064628460BF04DF9014693
:108CC00030460BF041F8A0600AB0BDE8F081074BD8
:108CD00010B51A881C4622EA00009042188002D083
:108CE000012009F0EFFA208810BD00BF68110020B4
:108CF000064B10B51A881C4610439042188002D0CB
:108D0000012009F0DFFA208810BD00BF68110020A3
:108D1000024A936823EA000090607047F02900201F
:108D2000024A936818439060704700BFF029002002
:108D300008B5104B1A780023D9B2914207D20E49D8
:108D4000002051F82310013309680880F4E732202D
:108D500009F05DFA094B1B685A0309D5084B9B685B
:108D60005B0305D4BDE8084040F2DC5009F04FBA7F
:108D700008BD00BF24280020F427002090290020EF
:108D8000F02900204B4A69232DE9F34113704FF479
:108D9000FC635380BE231371EF2382F8DD37002379
:108DA0001946164682F8DE37F25C0133B3F5FC6FE4
:108DB00081EA0201F8D13F4B3F4A83F8DE173F4B6F
:108DC00004275A6002F188325A600020013F17F0F0
:108DD000FF075ED0394B3422394CDA6004F1784811
:108DE000A8F5FC38C8F3090353B100234FF4005031
:108DF00056F80880019305F0B5F90428E6D11CE087
:108E00004FF4302005F0AEF90428DFD12B4D4FF49C
:108E100030202B6943F002032B616C612B6943F016
:108E200040032B6105F09EF941F6FD732A69042881
:108E300003EA02032B61D8D0C8E7204D4FF400505D
:108E40002B6943F001032B611FFA88F3238005F09F
:108E500089F9042813D1A31C0193019B4FEA1848F8
:108E6000A3F800804FF4005005F07CF941F6FE7342
:108E70002A69042803EA02032B6106D0A6E741F61B
:108E8000FE732A6913402B61A0E70E4B04349C4209
:108E9000A4D10A4A0428136943F08003136102D164
:108EA00007F0CAFD10B90A2009F024FA02B0BDE8A3
:108EB000F08100BFF0290020230167450020024017
:108EC00000F80108E0FF01082DE9F04107F0B4FDCA
:108ED00010B90A2009F00EFAB74CB8494FF4FC62F9
:108EE00020460EF075FB94F8B4374FF4CC71022B8A
:108EF00084BF002384F8B43794F8B427B04D01FB45
:108F000002F3E01800F53B702344286093F8400317
:108F100001FB0242022803F54E7384BF0020187241
:108F200092F84033A74A13700C2202FB0343A64A6F
:108F300003F2B673136046F20903A26813401BB92B
:108F40004FF40050FFF7ECFEA368DF0703D54FF4A2
:108F50000050FFF7DDFEA3685E0409D50820FFF787
:108F6000D7FE4FF40050FFF7D3FE0120FFF7D0FEED
:108F7000A368180706D54FF40050FFF7C9FE01207B
:108F8000FFF7C6FEA368990413D54FF40040FFF71E
:108F9000BFFE894B93F88631012B03D14FF400605B
:108FA000FFF7B6FE4FF48030FFF7B2FE4020FFF728
:108FB000AFFEA3685A0603D54FF48030FFF7A8FE32
:108FC000A36803F40852B2F5085F0AD11B0508D55F
:108FD000794B93F88631012B03D14FF40060FFF7F2
:108FE00097FE94F8DC21744B2AB193F8E02112B17A
:108FF000002283F8E0214FF0000C6746734E744B5B
:109000001E6004EB0C03B3F8F4E14FEA5E0101F0DB
:1090100077314FEA9E0303F03333C1EB0E00C11AE0
:109020004FEADE0303F01133CB1A03EB231303F0F3
:109030000F32FF2392FBF3F31EF00108C3EB03236F
:1090400018BF0137A2EB030318BFFFB2012B0ADDE3
:10905000022B40F0AE80B8F1000F00F0AA801EF0A5
:10906000BC0F00F0A6800CF1080CBCF1280FC8D191
:10907000013F012F00F29D8007F0BBFC3022002150
:1090800054480EF0B0FA544F544BD5F800801F608E
:10909000534B002108F17900C3F8008009F058F81B
:1090A000504B80F0010018704F4B07F126021A60F8
:1090B0004E4B07F1D8021A6098F8000007F072FCD6
:1090C00028684B4B00F5C5721A6002F0D5FD494B7C
:1090D00007F194021A60484B00221A809A71474B9C
:1090E0002D6807F12C021A60454B05F219121A601F
:1090F000444B05F289121A60434B07F108021A60CB
:10910000424BDFF844811F60414B07F19C021A601B
:1091100007F1A603C8F800303E4BB4F866011E60A4
:109120000AF0C2FEC8F80800B4F868010AF0BCFEF4
:1091300095F85C3008F1040288F8043095F878302E
:10914000C8F80C0088F8053094F8DF31286E88F8EC
:109150001030314BC8F814501A60304B05F16402DE
:109160001A602F490AF0F8FE01464FF07C500AF0D1
:10917000A7FFB5F816412B4B186020460AF098FE61
:10918000014629480AF09CFF28490AF0E5FE284AD2
:10919000284B1560284A186005F168031360274AB8
:1091A00005F211151560264A1760264A1360BDE8BE
:1091B000F08100F0B1F85FE7F029002000F8010825
:1091C000B80F002048290020E00F00207A2B002053
:1091D000602400206C0E0020342B0020A00E002004
:1091E000A40E002008000020742500209C0500200B
:1091F000B00E0020600E0020AC0D0020D025002015
:10920000D4240020DC080020C8280020CC2800201E
:10921000F0070020B4080020042600203C2600208F
:10922000DB0F494038260020000061444C3D0F44CC
:1092300010070020EC07002004070020DC070020B6
:10924000E40700200C0600208411002008B5FFF779
:1092500099FDFFF739FEBDE80840012009F032B85A
:1092600010B50446B0F9000007F0CDFFB4F90200D4
:1092700007F0C9FFB4F90400BDE8104007F0C3BF10
:1092800010B50446006807F0BEFF606807F0BBFF3A
:10929000A068BDE8104007F0B6BF2DE9F74F0120E8
:1092A00008F0CAFE002480B3012C2ED84FF04C0ADF
:1092B0000AFB04F7DFF85C8008EB070B0BF14806AC
:1092C000B57815B10134E4B2EDE790F9003090F8CB
:1092D00004E018460E4B03228DE8240001212A46A3
:1092E00053F82E30FFF76CF8814650B158462946A6
:1092F00052460EF078F901231C4448F80790B370E9
:10930000E4B2012008F07EFECDE703B0BDE8F08FA7
:1093100044A701089C11002000212A2210B5114801
:109320000EF061F9104B0022194610480424105C1D
:10933000013283F8F201052083F8F74182424FF0B1
:10934000000483F8F60183F8F94183F8F80103F18A
:109350000803EAD10123A1F8F431522381F8F03156
:1093600010BD00BFE02B0020F0290020C7C6010877
:1093700070B50646441E14F8011F89B1094D2846F0
:109380000EF067F90028F6D005F1080398423FBFB8
:10939000054B401BC018A31B38BF80F88A31EAE791
:1093A00070BD00BF62DC0108F029002007B51C4B2E
:1093B00003F19C02C3F898201A4A92F892215AB1FC
:1093C000012A14D1032183F89E10072183F8A020DD
:1093D00083F89F100C2208E0022183F89E100321DD
:1093E00083F8A02083F89F10072283F89C200E4A60
:1093F0000E4B40201A6008F01FFE70B101220023BE
:1094000090F9000040218DE80C00094A4FF4E13347
:10941000FEF7D6FF003018BF012003B05DF804FB53
:109420009C110020F0290020C1DC00082000002051
:109430004DDE00082DE9F04F8DB01F46BDF95830C4
:10944000B34C01939DF86030039205460C220E4602
:1094500004F1A400002102930EF0C5F800211422AB
:1094600004F1B0000EF0BFF8002384F8C430A94B1B
:1094700093F800909846A84B03F11802B9F1010F38
:1094800088BF1346C4F8C830FCF7C2FE8246834644
:1094900070B3A24BB5F5807FC4F8B030A04BC4F8D0
:1094A000B430A04BC4F8BC309F4BC4F8C0309F4BC5
:1094B00001D1002216E0BB2D01D9012212E0612D5D
:1094C00001D902220EE0292D01D903220AE0132D31
:1094D00001D9042206E0092D01D9052202E0002D60
:1094E000E7D006221A71012384F8C43002236AE00F
:1094F000192008F08CFE68201521524608F00CFD5A
:1095000078B38B4A622DC4F8B0208A4AC4F8B420DC
:10951000894AC4F8B820894AC4F8BC20824AC4F8F1
:10952000C020824A0FD004D80A2D13D0142D0FD09A
:109530000CE0BC2D05D0B5F5807F07D182F805A0E1
:109540000AE0012300E00223537105E00323FBE757
:109550000423F9E70523F7E7012384F8C430042343
:1095600031E0B9F1030F40F0E783FCF70DFE00286E
:1095700000F0E283724BBB2DC4F8B030714BC4F8DD
:10958000B430714BC4F8BC30674BC4F8C030674B83
:1095900001D901220FE0612D01D902220BE0292D12
:1095A00002D983F806900AE0132D01D9042202E0C3
:1095B000092D02D905229A7101E00622FBE7012359
:1095C00084F8C4300723614A1370614A136843F07A
:1095D000010313605F4B00221A709946082E33D89E
:1095E000DFE806F0383238101D22102D2D004FF024
:1095F000000A0CAB03F818AD53205146012208F0C5
:109600004BFC60BB444B98F8001003F11802012991
:1096100088BF1346C4F8C830FCF7FAFD80BB98F841
:109620000030012B40F2A08000210CAB03F8181D84
:109630001820012208F030FC002840F0B58098F88E
:109640000030032B00F0C080012E40F2D380414B4C
:1096500000261E7098F80030012BD3D8C7E79DF87C
:109660001830E52BCED13C4B84F8CCA0C4F8A43004
:109670003A4BC4F8A830042389F800300223B2E042
:1096800006210A4606AB682008F006FC9DF81D106E
:1096900001F001029DF81B1001F001014B0043EAAB
:1096A00082019DF8192002F001030B430AD05BB23E
:1096B000012B01D1002302E0022B0ED1012384F8FB
:1096C000CD3011E005AB68200C21012208F0E4FB4D
:1096D0009DF8143013F00F0303D1052008F00AFEA3
:1096E00002E0042BEAD1E5E71D4BC4F8A4301D4B82
:1096F000C4F8A83094F8CD30002B0CBF6F236E2334
:1097000084F8AC30012389F8003003236BE000BFFC
:109710009C110020E333002064A701088560000845
:10972000FD5A0008B55D000890C1793D2000002079
:1097300029610008CF5B00089D5B00087D5B000885
:10974000515F0008B95E0008955E000858000020CF
:10975000A0100020E233002091590008A95C000805
:10976000FD6000083D5B000800220CAB03F8182DDB
:109770001C200D21012208F08FFB00283FF454AF7C
:109780009DF818302A2B02D01A2B7FF44DAFCB4A0C
:1097900084F8CE30C4F8A420C94A022389F80030E6
:1097A000C4F8A82004231EE09DF81830FB2B7FF49A
:1097B00046AFC44BC4F8A430C34BC4F8A83001234F
:1097C00089F8003005230EE0FCF7DEFC00283FF4AA
:1097D0003BAFBE4BC4F8A430BD4BC4F8A830012346
:1097E00089F800300823BB4A5370BB4A136843F022
:1097F0000203136098F80030012B05D109F016FC24
:10980000B64B4FF400525A61042F00F2BB81DFE8DF
:1098100017F00500C2016900050080010A2008F068
:10982000F6FC7720A021012205AB08F035FB0028CB
:1098300058D01E210122772008F06EFB4FF42F60D4
:1098400008F0DAFC0027A7F160010026C9B2022265
:1098500006AB77208DF818608DF8196008F01CFBB6
:109860009DF819309DF8182043EA02229C4B03F121
:10987000D0017A520237102FE5D1B3F8DE1032460C
:1098800001F00F0701F47F41A3F8DE1033464FF0DB
:10989000010E22F001002044B0F8D000002818BFCB
:1098A0004FF0000ED60703D5C0B24340082002E0B7
:1098B00083EA1023FAE71E0448BF83F4C05301383B
:1098C0004FEA4303F7D10132102AE2D13943844AE7
:1098D000A4F8DE10BEF1000F04D1C3F303339F429E
:1098E00000F0058294F8E0907D4EB9F1000F40F051
:1098F0001B827A4C09F09AFB4FF48047042305A998
:109900002046ADF814708DF8163005F0EAF84FF4E3
:1099100000532361734808F023FD0E21022005F057
:10992000CBF80823069706A801278DF81D308DF87F
:109930001C908DF81E704FF0030804F037FD2823AB
:1099400004A88DF810308DF811808DF812908DF8E4
:10995000137009F0F1FA142008F059FC7720D02197
:109960003A4605AB08F098FA002800F090809DF880
:109970001430A6F80481552B86F8FB3040F0878020
:10998000D1213A4605AB772008F086FA9DF81430CD
:10999000772003F00F021B0986F8FC2086F8FD30C3
:1099A000162206ABAA2108F077FA9DF818209DF838
:1099B000193043EA0223A6F8E4309DF81A209DF8F6
:1099C0001B3043EA0223A6F8E6309DF81C209DF8E0
:1099D0001D3043EA0223A6F8E8309DF81E209DF8CA
:1099E0001F3043EA0223A6F8EA309DF820209DF8B4
:1099F000213043EA0223A6F8EC309DF822209DF89E
:109A0000233043EA0223A6F8EE309DF824209DF887
:109A1000253043EA0223A6F8F0309DF826209DF871
:109A2000273043EA0223A6F8F2309DF828209DF85B
:109A3000293043EA0223A6F8F4309DF82A209DF845
:109A40002B3043EA0223A6F8F6309DF82C209DF82F
:109A50002D3043EA0223A6F8F83041F2707386F8FD
:109A6000E070A6F8083146F67813A6F80A311E4BC6
:109A7000C6F80C311D4BC6F810311D4BC6F8143119
:109A80001C4BC6F818311C4BC6F81C314CE11B4A64
:109A9000136823F480431360114B124AD3F820114A
:109AA000914209D0D3F82411914229D0D3F828113A
:109AB00091422BD1022224E0002222E0DB5D00084B
:109AC0000D5C00086D590008655C00080559000828
:109AD000F55E000858000020A01000200010014092
:109AE0009C1100206D5D000859590008C95A0008F2
:109AF000335900087D5A0008295800080004014025
:109B0000012203EB82030022C3F820214FF400530B
:109B100063618B4C94F82C61002E40F0FF80142080
:109B200008F075FB04F22D137620D021012208F0F5
:109B3000B3F994F82D31582B2DD104F59873882161
:109B40001822762008F0A8F97620F421312208F0B6
:109B5000E3F9012384F82C317A4BA4F80861C4F8A6
:109B60001031794BC4F80C3145F6D813A4F80A31FA
:109B7000764BC4F81431764BC4F81831754BC4F8E1
:109B80001C31CBE0012F06D0734B744A9F701368D1
:109B900043F004031360714E694C336813F0020FF5
:109BA00002D0D4F8A4309847029B63B315F0FF0F9E
:109BB000336809D140F2596213F0020F40F2712369
:109BC00018BF13467D2208E09A0759BF4FF47A73F5
:109BD0001A464FF4FA634FF47A721799994205DBEB
:109BE000B1F57A6F0B46A8BF4FF47A63511E0B4450
:109BF000B3FBF2F3013BDBB203FB022284F84C31EE
:109C0000C4F8502106E09DF8083084F84C31179BC9
:109C1000C4F85031D4F8B0309847514B039F93F8B3
:109C20000090504B03F11802B9F1010F94BF99460F
:109C300091464D4D00232B700FB1022F70D14FF084
:109C400000080CAB03F8188D1E200A210122DFF852
:109C5000F0B0C4F8549108F01FF998B19DF818308D
:109C6000482B63D1414B0222CBF85831404BCBF803
:109C70005C3103232B70384BDA70336843F00803F0
:109C8000336001E0804651E03A4B93F858210AB125
:109C900084F8C42093F859210AB137490A7093F81F
:109CA0005A3103B12B7033681B071AD5019B642608
:109CB00093FBF6F528460AF0FBF8019B074606FBE6
:109CC000153000B20AF0F4F82C490AF045F90146C3
:109CD00038460AF039F82A490AF03EF9C4F860011A
:109CE00002E00023C4F860314FF0010B24E042F29F
:109CF0001073A2F80831A2F80A31224B0327C2F8E8
:109D00000C31214BC2F81031204BC2F81431204BDA
:109D1000C2F818311F4BC2F81C3135E7042733E76E
:109D2000012FB1D91F4684E702272DE7012FABD9B8
:109D3000002785F8008082E758460DB0BDE8F08F17
:109D40009C110020255800082758000829590008B0
:109D5000315A0008C155000858000020A01000200A
:109D6000E333002094A70108E433002047EB000808
:109D7000EDE70008F0290020E23300208988883CC4
:109D8000000020411F590008215A000815590008F9
:109D9000115A0008055400080120002108F054BEA3
:109DA000174AF0B5164692F86431D2F868E1042BF0
:109DB00010D85C1C0EEBC3039D1CE4B208D09A883B
:109DC000D10705D5104203D008E00131052907D19C
:109DD0002346ECE786F864310020F0BD9F7800212F
:109DE0000C2202FB01F3064D05F5B67C1CF803209E
:109DF0009742EAD12B4485F86441D3F87001F0BD55
:109E00009C1100208A6810B50C6A036814430A6923
:109E100023F4FF4314434A6923F0700314438A690F
:109E20001443CA6914434A6A14438A6A2243134397
:109E30000360CB6843600B6883604B68C36010BDF0
:109E4000426A806A131A58425841704741717047FC
:109E500043799B070AD5436A8269D154436A0169F1
:109E60000133B3FBF1F201FB1233436270474379D4
:109E700013F001031FBFC36803F1FF32C369006A17
:109E80001DBF181A1040C0B218467047437910B56C
:109E900013F0010304460DD0FFF7E9FF58B1236A20
:109EA0006269E168D05C0133B3FBF1F201FB12336C
:109EB000236210BD184610BD90F83B3210B57BB937
:109EC00090F83A3290F83942A34209D2B0F84012E1
:109ED00001229A400A430133A0F84022DBB2F3E7A3
:109EE00010BD8379DB0748BFB1FA81F1D0F8343176
:109EF00048BF49095A681B8909B11361704753610A
:109F0000704710F80A3C0133DBB20A2B84BF10F80B
:109F1000131C054A00F80A3C82BF002322F81130C6
:109F200000F80A3C704700BFDC220020334A70B5BD
:109F3000136C9068194440F68C23081A984291607B
:109F4000D060516013463BD9127893F94510104602
:109F50008A420BD1111F082908D893F846101829F6
:109F600001D8013103E083F8442002E0002183F8A6
:109F7000461093F944402149A24219D191F8474033
:109F8000B4B10C310024944206DA51F8046F1C4D30
:109F900025F814600134F6E70C2805D01849002490
:109FA00021F810400130F7E71648017801310170BF
:109FB00083F84520002201211A7083F8471070BDF4
:109FC00092F84710C9B140F2DA51A0F2EF248C4266
:109FD00008D811780B2905D80B1D0131117042F8F2
:109FE000230070BD002283F84720074B03F13002A5
:109FF000002143F8041F9342FAD170BD04010020F0
:10A00000DC220020CC05002010010020024A136C45
:10A01000013319441164704704010020024B53F8C6
:10A0200020301B6819807047F4270020074BA1F5EA
:10A030007A7153F820301A681B8959434FF47A73A8
:10A0400091FBF3F189B21180704700BFF427002023
:10A050001FB50123ADF80830ADF80410002301A9A5
:10A06000ADF80A30ADF80C30ADF8062004F08BF8EE
:10A0700005B05DF804FB38B5A0F513746379A579D4
:10A08000DB0745D594F8383205F00105F3B1226BB2
:10A090001068838DC3F34E03838494F83C3223B15C
:10A0A000B4F842320133A4F84232917A6A00FFF7E1
:10A0B000CFFF012384F83B32002384F8393284F83F
:10A0C0003A3284F83832A4F8403238BD94F83B3242
:10A0D0002046012B04BF94F8393284F83A32FFF756
:10A0E000EBFE94F83B22236B3AB9012284F83B2221
:10A0F0001868997A05FA02F207E0002284F83B22F8
:10A1000095421868997A08BF0222BDE838409FE757
:10A1100038BD10B5A0F5127494F83C22BAB9A36A00
:10A12000616A994228D0591CA069A162C35C206968
:10A13000DBB25B0043F400738142A4F83E324FF07F
:10A140000A0384F83D3228BFA262012312E094F989
:10A150003D327BB1B4F83E1220464B08A4F83E32A3
:10A1600001F00101FFF7BDFE94F83D32013B84F898
:10A170003D3201E084F83C3294F83832002B4ED165
:10A1800094F839320133DBB2092B84F8393203D128
:10A190002046BDE810408FE60A2B40D194F83B32B0
:10A1A0002BB9B4F8403243F00103A4F8403263798C
:10A1B000D9071CD5B4F84002820501D4C30705D4E1
:10A1C000B4F844320133A4F8443210E0E36AC0F337
:10A1D00047000BB198470AE0E3696269D054E3692C
:10A1E000E1680133B3FBF1F201FB1233E3610122B9
:10A1F00084F8382294F83B220023012A84F839326B
:10A200000DD1A27984F83B32236B12F0010F18684C
:10A21000997A0CBF02220022BDE8104018E710BD59
:10A22000F0B5046D8279A389467923F4005312F0C6
:10A23000020F4FEA03434FEA13430CBF00214FF4D0
:10A24000005112F0040FA38114BF4FF4806E4FF041
:10A25000000E16F0010F8768054614BF0420002089
:10A26000B307238A48BF40F008029BB223F440534F
:10A2700043EA01032382A18948BF90B289B221F445
:10A28000B05121F00C014EEA010140EA0102A28125
:10A29000A38A87B023F440731B041B0CA38201A87C
:10A2A00003F016FF039B049E254A944218BF1E46E6
:10A2B000A389192272431BB2002BB4BF7E00BE00DB
:10A2C000B2FBF6F66427B6FBF7F00001010907FBC5
:10A2D0001163A28912B2002AB7BFD9001A01323124
:10A2E000B1FBF7F2A7BF3232B2FBF7F302F007027D
:10A2F0001043A8BF03F00F03AA79A8BF184380B288
:10A3000012F0010F20812B6D06D00E498B4202BF47
:10A31000042001F54841086112F0080F9A8A0BBF2A
:10A3200022F0080292B2120442F0080208BF120C96
:10A330009A829A8992B242F400529A8107B0F0BD93
:10A3400000380140004400402DE9F04F504C4FF4DC
:10A35000147685B0804691461D4606FB004627468A
:10A3600008B94C4B02E0012804D14B4B3363103346
:10A37000C6F834314FF4147303FB08F3474AFC1852
:10A38000FA5003226271224603F59C733B44E1625A
:10A39000A36100214FF48070D4F8343134324FF08F
:10A3A000010B62612162E161A162616284F83C1289
:10A3B00084F83912A4F84212A4F84412C4F80890A0
:10A3C000A571E060206184F838B284F8468258684C
:10A3D0001B890222ADF80C3003A910238DF80E3032
:10A3E0008DF80F20019204F07CFB236B019A597BBE
:10A3F00058681B898DF80E1003A9ADF80C308DF844
:10A400000F2004F06EFB30465946FFF76AFD3220FC
:10A4100007F0FDFE224BD4F834A11B681A46B2FBAC
:10A42000F9F1B1F5803F03D3012AF8D95208F6E7D4
:10A430001C4A5046B3FBF2F289B2D2B200F004FEDD
:10A440004FF4147000FB08F0174B07EB000800F501
:10A4500012703C180022C8F848325046214600F0DD
:10A460003BFED8F8307015F0010F0CBF022200221D
:10A470003868B97AFFF7ECFD0C4B3846C8F84C3217
:10A48000211D002200F028FE304605B0BDE8F08F07
:10A49000441300200CBF01082CBF0108C4A7010809
:10A4A0006000002040420F0013A1000877A00008C0
:10A4B00003460A4690F84602D96A9B7944E71FB5DD
:10A4C0000123ADF808300023ADF80C30ADF80A30A8
:10A4D000084BADF804101B7801A9012B08BF03231A
:10A4E000ADF8062008BFADF80C3003F04CFE05B007
:10A4F0005DF804FB0001002038B510F80E2C04466E
:10A5000050F8043C52B9012200F80E2C20F80C1C23
:10A51000997A18680222BDE83840D0E730F80C2C50
:10A5200020F80A1C891A89B220F8081C074A10F87A
:10A530000F0C002522F8101004F80E5C1868997AA8
:10A540002A46FFF7BCFF04F8065C38BDDC22002079
:10A55000044B53F820301BB107289CBF1B6819809F
:10A56000704700BF2C0200202DE9F7438E460546B8
:10A57000DFF8A092114699F8A04400681646984664
:10A580007246631C89F8A03400F00AFD2B8901A9EA
:10A59000ADF8043018238DF80630686802238DF872
:10A5A000073004F09EFAAB7A09F2A447240127444D
:10A5B0002A6849460C2B00F2F680DFE813F00D0004
:10A5C000F400F400F4005100F400F400F4008A00F8
:10A5D000F400F400F400C200138CDFF83CC223F056
:10A5E00001031B041B0C1384138CB2F804E0108BC2
:10A5F000624520F073004FEA00404FEA10409BB2E2
:10A600001FFA8EFE40F0700014D00CF5006C62450D
:10A6100010D00CF5406C62450CD00CF5806C624596
:10A6200008D00CF5806C624504D023F0020343F09F
:10A63000030307E023F00E032EF4407E43F00303F0
:10A640004EF4807EA2F804E01083A2F834801384D4
:10A65000138B23F008031B041B0C43F0080336E0A4
:10A66000138CDFF8B4C123F010031B041B0C1384FC
:10A67000138CB2F804E0108B624520F4E6404FEAF8
:10A6800000404FEA10409BB21FFA8EFE40F4E040BB
:10A6900008D00CF5006C624504D023F0200343F091
:10A6A000300307E023F0E0032EF4406E43F0300364
:10A6B0004EF4806EA2F804E01083A2F83880138470
:10A6C000138B23F400631B041B0C43F400631383FC
:10A6D00069E0138CDFF840C123F480731B041B0C6A
:10A6E0001384138CB2F804E0908B624520F0730061
:10A6F0004FEA00404FEA10409BB21FFA8EFE40F036
:10A70000700008D00CF5006C624504D023F400738F
:10A7100043F4407307E023F460632EF4405E43F497
:10A7200040734EF4805EA2F804E09083A2F83C806F
:10A730001384938B23F008031B041B0C43F00803C2
:10A7400030E0138CDFF8D0C023F480531B041B0CC3
:10A750001384108CB2F804E0938B20F4005023F49F
:10A76000E6431B0400041B0C000C62451FFA8EFE1E
:10A7700043F4E04340F4405003D00CF5006C6245D4
:10A7800003D12EF4804E4EF4804EA2F804E0938361
:10A79000A2F840801084938B23F400631B041B0CED
:10A7A00043F4006393832B7B43B1B2F844306FEAE8
:10A7B00043436FEA53439BB2A2F8443013889BB2E1
:10A7C00043F001031380AB7A0C2B19D8DFE803F0B8
:10A7D000071818180B1818180F18181813000B1949
:10A7E00002F134000AE00B1902F1380006E00B19FF
:10A7F00002F13C0002E00B1902F14000C3F8A4048E
:10A8000038460C44A4F8AC64C4F8A82403B0BDE8EE
:10A81000F08300BF44130020002C014004F030B846
:10A8200004F02EB804F02CB808B508480CF01FFF4F
:10A83000C0B209280246054B04DC01302021C0B219
:10A840009954F6E700221A5408BD00BFBD2100202C
:10A8500008B507480CF00BFFC0B21428044B04D80D
:10A86000421C20211954D0B2F7E700221A5408BD27
:10A87000BD2100202DE9F74F07F0A4FCA64C80462F
:10A8800026686568A768861BF643451BC71BED4312
:10A89000FF43F60FED0FFF0F2EB93FB9002D00F06B
:10A8A0008782B9462CE04FF0000929E0B14627E045
:10A8B00003EB8A0BBBF802301A050ED413F4805F49
:10A8C0001DBF964A9BF801101268954A954B14BF1C
:10A8D00052F82120126843F82A20BBF80230D8052C
:10A8E00016D499050AD5904B1B7813F0040F0CBFB2
:10A8F0008E4A8F4A8B4B126843F82A2009F10109CE
:10A90000207B5FFA89FA8B4982450B68D0D326E019
:10A91000894A5046594606F0F7FC884B1B885A0670
:10A9200003D550465946864A16E0580703D5504687
:10A930005946844A10E0190703D550465946824AC1
:10A940000AE09A0703D550465946804A04E0DB07DF
:10A95000D4D5504659467E4A06F0D6FCCEE7DFF8FD
:10A9600008E20093BEF906307822A3F57A735343C8
:10A970004FF47A7293FBF2F3F34603F22B13019335
:10A9800000225FFA82FE864517D2009B03EB820EFF
:10A99000BEF802E01EF4806F0DD040F2671ADFF8B7
:10A9A0008491019B39F822E09E449EFBFAFC0AFB4D
:10A9B0001CEE29F822E00132E3E74DB308F5C3337A
:10A9C000A0336360637B544A13BB9373614B1B6872
:10A9D00013F0020F0AD0DFF894E19EF800E0BEF118
:10A9E000000F03D04FF0010E82F80EE0DA0506D515
:10A9F000594B5B791BB1A37B43F00203A3734A4B12
:10AA00001B7813F0050F02BFA37B43F00403A3736D
:10AA100094F80EE0BEF1000F03D13F4B5B7B002B9F
:10AA20004FD094F80DC01CF0010FACF10C031DD1F8
:10AA3000BCF1030F07D8DFF8E8901EF0040F3B4A83
:10AA400008BF4A4600E0364AACF1040CBCF1070FDF
:10AA500005D8DFF81CC11EF0010F18BF6246DBB23B
:10AA6000032B0ED81EF0020F3C4B06E0DBB2032B8B
:10AA700006D82F4B2A4A1EF0020F18BF1A4600E0D4
:10AA8000274A4FF0000C5FFA8CF383420DD20B681B
:10AA900003EB8C035B881B0642BFD2F80090214B6E
:10AAA00043F82C900CF1010CEDE785B1BEF1000FDD
:10AAB00008D0637B184A0133DBB2142B06D1002384
:10AAC00004E025B1637B002BF3D100E05373002E2B
:10AAD00052D0234A3223B2F90250B2F90020002D9D
:10AAE000B8BF6D42002AB8BF524295FBF3F592FB06
:10AAF000F3F2EDB2D3B2AB4238BF2B46194A13B1D1
:10AB000092FBF3F300E0134643442360E37B024AE5
:10AB100083BB01232FE000BFA8180020D024002011
:10AB2000ACBF0108220D0020E133002010B0010865
:10AB300000B0010874110020DCA701086811002092
:10AB4000E2A70108E8A70108EEA70108F4A7010899
:10AB5000FAA7010890290020AC0D002018B00108C8
:10AB600084100020400D0300CC290020F0100020AC
:10AB700020B001080023D3738F4D904B2D78E27BDA
:10AB8000ADB9002F00F00F818D4B267B1A788D4BCD
:10AB900002F0040293F800C08B4BD2B2D3F800E06D
:10ABA0000B680021894D03EB86060F46B5E01AB904
:10ABB000874A1A61002508E0864AFAE70A68AB006E
:10ABC000D6187688760604D40135EBB28342F5D3E5
:10ABD000D7E7814EB6F90060192E25DD12F803E0A3
:10ABE00094F814C00EF00F09E14526690CDCDFF87B
:10ABF000CCC19CF815C0BCEB1E1FDEBFD6F800C050
:10AC0000DFF8D8E143F80EC012F803E094F816C05C
:10AC10000EF00F09E14533DBDFF8A0C19CF815C049
:10AC2000BCEB1E1F2CDC26E0193629DA12F803E0F3
:10AC300094F814C00EF00F09E14526690CDCDFF82A
:10AC40007CC19CF817C0BCEB1E1FA2BFD6F800C089
:10AC5000DFF888E143F80EC012F803E094F816C05C
:10AC60000EF00F09E1450BDBDFF850C19CF817C06F
:10AC7000BCEB1E1F04DBD6F800E0584E43F806E09C
:10AC8000554EB6F90260192E1BDD12F803C094F878
:10AC900014E00CF00F09F14526690CDCDFF81C917B
:10ACA00099F81590B9EB1C1FDEBFD6F80090DFF8BD
:10ACB0002CC143F80C90D25C02F00F0CF4451EDD61
:10ACC00082E7193680DA12F803C094F816E00CF027
:10ACD0000F09F14526690CDBDFF8E09099F8159033
:10ACE000B9EB1C1FDEBFD6F80090DFF8F0C043F8C8
:10ACF0000C90D25C02F00F0CF445FFF665AF94F8AF
:10AD000017E0BEEB121FA2BF3668344A9E505BE7C5
:10AD10005888000504D404330435B342F8D122E046
:10AD20004AB101EB0C0A06209AFBF0F900FB19A0CE
:10AD300001280DDC01E057B9012793F801900EEBD3
:10AD400089003EF829A090F80290C07803E01746E9
:10AD5000002081468246013125F802AC85F800903A
:10AD60006870C9B2D7E7174A1378013B13F0FF03A5
:10AD700008BF06231370124B1B785B0741BFBBF95A
:10AD800006304FF47A72A3F57A7303EBC30348BF1E
:10AD900093FBF2F3124A46BF0133DBB2012392FB6D
:10ADA000F3F34344A36003B0BDE8F04F03F0A6BD46
:10ADB00003B0BDE8F08F00BFDB0D0020A818002015
:10ADC000E133002028000020D0240020240D0020A2
:10ADD0001CB00108ACBF010884100020220D002027
:10ADE000400D0300026D70B515880446ADB2A9068A
:10ADF00013D5036B8BB9C36A1BB1908880B2984797
:10AE00000BE0E169928840694E1CD2B2E66142547F
:10AE1000E169E268914228BFE3612B0613D5636ABA
:10AE2000A26A9A42236D0AD0511CA069A162825C79
:10AE30009A802369994206D30023A36270BDDA6821
:10AE400022F08002DA6070BD026B0346C16810B563
:10AE5000406942B11A6C8C1A013A08BF0A46005D7B
:10AE60001A64C0B210BD1A6A805C01328A4228BFDF
:10AE70000022C0B21A6210BD436B13B190F84400B7
:10AE80007047836A406A1B1A584258417047036BE7
:10AE900013B15B68016C01E0C369016A8B423CBF7E
:10AEA000C2689B18581AC0B27047836A8169426BA6
:10AEB0001944D160416A994297BF0169CB1ACB1AF4
:10AEC000536096BF0023536083624FF0000380F805
:10AED0004430136888BF816243F0010313607047F8
:10AEE000436A8269D154436A02690133934228BF9D
:10AEF00000234362436B1BB11B68DB0705D4D4E717
:10AF0000026DD36843F08003D36070474171FFF74F
:10AF100087B98160FFF784B92DE9F04105460E46F7
:10AF2000078A83899BB21F40002F37D0B7FA87F278
:10AF30004FF00043D340DB4399B21F40A2F11B0303
:10AF40002982042BF0D8DFE803F0221F1C1903002C
:10AF5000746A24B1013C0023A4B2736201E0AC8D99
:10AF6000A4B2D6F82080B8F1000FDDD0D8F80030B8
:10AF7000404621469847D8F80480F4E73068A98E07
:10AF800008E07068298F05E0B068A98F02E0F068DA
:10AF9000B5F84010036889B29847C5E7BDE8F0816D
:10AFA000254B10B55A43254B254C1B680139B3FB83
:10AFB000F2F20388013AA04289B292B29BB212D057
:10AFC00004F50064A0420ED0B0F1804F0BD0A4F580
:10AFD0009834A04207D004F58064A04203D004F561
:10AFE0008064A04202D123F070039BB2154CA042B2
:10AFF00006D004F58064A0421CBF23F440739BB2CA
:10B0000003800F4B8185984202850FD003F50063C2
:10B0100098420BD003F54063984207D003F5806354
:10B02000984203D003F58063984201D10023038640
:10B030000123838210BD00BF40420F00600000204A
:10B04000002C01400010004073B505460068FFF772
:10B05000A7FF2A680124138800269BB243F001034E
:10B060001380EB7A01A88DF804308DF805408DF837
:10B0700006608DF8074007F05FFFEB7A1B2B0BD1C2
:10B08000192301A88DF804308DF805408DF806606D
:10B090008DF8074007F050FF02B070BD0C4B800ADE
:10B0A00098420CD004D8B0F5801F0CD10120704715
:10B0B000084B984205D04933984206D003E002205D
:10B0C000704703207047FE2070470020704700BF84
:10B0D00001001000020010002DE9F8430468074643
:10B0E000204688469146FFF7D9FF03284BD8BA7A05
:10B0F0009108B8F1000F06D1A589AEB202258D40A6
:10B1000026EA0505A5810A2303FB00131F4A42F81E
:10B110002380043342F82390B8F1000F07D0BD7AA2
:10B12000A189AD080223AB400B439BB2A381282326
:10B13000434303F120011144EFF31286502585F3B8
:10B14000128803F10C051C331544134455F8047F91
:10B1500017B10F60296804319D42F7D100230B60BD
:10B16000F3B283F31188282303FB0020036A23B181
:10B17000A3899BB243F0010304E0A38923F00103F8
:10B180001B041B0CA381BDE8F88300BF2828002006
:10B19000004827E6C0180020004823E614190020C4
:10B1A00000481FE6681900200B4B4FF400525A600C
:10B1B0004FF6FE730948D0F8DC2011680B4013608D
:10B1C000D0F8CC20D0F8D0309A4201D0A8306CE62C
:10B1D000012380F8EC30704700000240C0180020C6
:10B1E0002DE9F0431D46A64B8DB098428846174680
:10B1F0009DF850605CD1A34BA34AA449C3F8A82092
:10B2000003F1FC02C3F8BC2003F5FE72C3F8C020B2
:10B210004FF48072C3F8B420C3F8B8209C4AC3F836
:10B22000B070C3F8D820A2F54842543AC3F8F420CD
:10B23000C3F8F020C3F8F800C3F8DC10954B9A6906
:10B2400042F480429A615A6942F001025A61022333
:10B250008DF803304FF40073ADF80030330701D59B
:10B260001C230FE0AC0706D518238B4869468DF8E0
:10B27000023003F036FCE8070AD54FF48063ADF8DE
:10B2800000304823844869468DF8023003F029FCD9
:10B290000E238DF804300022012301A88DF805301B
:10B2A0008DF806208DF807307C4C07F045FEA1E0B4
:10B2B0007B4B98424ED1734B734ADF655A654FF40E
:10B2C00080721A665A6603F53F729A6603F57F72BA
:10B2D000DA66744AC3F8A400C3F89C20C3F8A0201F
:10B2E0006C4B3107DA6942F40032DA615A6942F094
:10B2F00001025A614FF002038DF803304FF004034E
:10B30000ADF8003001D51C230EE0AA0706D518239E
:10B31000614869468DF8023003F0E3FBEB0709D57D
:10B320000823ADF8003048235B4869468DF80230A9
:10B3300003F0D7FB26238DF804300022012301A857
:10B340008DF805308DF806208DF80730564C07F043
:10B35000F3FD4FE0554B984240F0ED80494B4A4A8F
:10B360009F601A6003F2FC425A6103F2FC529A6138
:10B370004FF48072DA601A614D4A18659A64DA6493
:10B38000444B3407DA6942F48022DA619A6942F068
:10B3900008029A614FF002038DF803304FF4806386
:10B3A000ADF8003001D51C230FE0A80706D51823FF
:10B3B000404869468DF8023003F093FBE9070AD54F
:10B3C0004FF40063ADF8003048233A4869468DF8E1
:10B3D000023003F086FB27238DF80430002201237E
:10B3E00001A88DF805308DF806208DF8073007F09C
:10B3F000A3FD244C4FF00009012384F84430C4F825
:10B400002090C4F81C90C4F82890C4F82490C4F884
:10B410002C806571A760A6712046FEF701FFEA0740
:10B4200052D5206B002847D0E36CCDF80C900193E7
:10B430004FF480530A9380230693E368CDF8149069
:10B440000493202309936369CDF81C900293CDF8EF
:10B450002090CDF82C9002F0C3FD01A9206BFEF7DF
:10B46000D1FC226B216D136843F0010313608B8ABA
:10B470009BB243F040038B8253689BB2236423E06A
:10B4800000380140C018002000A801084400024014
:10B4900058000240001002400008014068190020D6
:10B4A00000440040044400401419002000480040BB
:10B4B00004480040000C01404FF6DF72236D1A80F3
:10B4C000DA6842F02002DA60AB072CD5606B28B353
:10B4D000A36C002501934FF480530A9380230693B5
:10B4E0002369029504931023039305950795089506
:10B4F00009950B9502F074FD606B01A9FEF782FCC3
:10B50000636B1A6842F002021A60226D5D605D6032
:10B51000938A9BB243F08003938204E0226DD36848
:10B5200043F08003D360226D204693899BB243F49D
:10B530000053938100E000200DB0BDE8F08300BF10
:10B5400010B508F0B5FC0021044608F0C1FE08B1B2
:10B55000204601E004F10040054908F0B1FD05492D
:10B5600008F0FAFCFDF7E2FA034B186010BD00BFCB
:10B570008096184B35FA8E3C4C000020F8B59C4B59
:10B5800004461B68187818B1012800F06A819AE215
:10B59000242C984D0CD006D80A2C00F0D9800D2C04
:10B5A00000F0D68048E12A2C06D02C2C04D043E1B0
:10B5B00028706870A87050E18F4B69782F78002050
:10B5C0008C4A58542FBB1978D770472921D1597804
:10B5D00050291ED19978472907D1D978472904D114
:10B5E0001979412901D10121D1709978824A5229D2
:10B5F00003D1D1784D2900F0688299787E4A472995
:10B6000007D1D178532904D11279562A04BF0322D5
:10B61000EA70EA78774E022A39D0032A4CD0012A00
:10B6200040F08580BA1E072A00F28180DFE802F030
:10B6300004080F131A257F2A07F086FE686076E05B
:10B640001B78532B73D16B685B426B606FE007F024
:10B650007BFEA8606BE01B78572B68D1AB685B4220
:10B66000AB6064E01B78302B644B1A788CBF42F0DF
:10B67000020222F002021A7059E0002007F0C4FE14
:10B68000287354E0002007F0BFFEE8814FE0072F49
:10B6900006D0082F4BD1012007F0B6FE708246E09D
:10B6A000012007F0B1FE41F2184358434FF47A737A
:10B6B000B0FBF3F030823AE0022F07D0032F0AD11B
:10B6C000002007F0A1FE4E4B187030E0002007F07C
:10B6D0009BFE30752BE02AD93A1F9210337D013240
:10B6E000D2B2013B02EB8303DBB2102B1FD8F91E51
:10B6F000C2F1010201EB8202D2B2012A0BD0042A6C
:10B7000011D100205E1E07F07FFE3E4B00229855AF
:10B710003D4B9A5507E03D4A5E1E0020935507F0C9
:10B7200073FE3B4B98553B4A136801331360314B12
:10B730002A2C18BF9A7807F101074FF000000CBFC0
:10B74000012254402F7068700CBF5A759C7084E0C1
:10B75000687D002848D0304B13F8012D2F495A70CE
:10B760008B42F9D1244A234C13785278402B85BF61
:10B77000373B1B011B01DBB298BF03F0F003402AEB
:10B780008CBF373A303AD2B21344AA78DBB29A422D
:10B7900027D121230B702249E0780B68012803F19F
:10B7A00001031E4A0B600AD002281CD172231370B9
:10B7B000228A1C4B1A80628A1B4B1A8013E0672373
:10B7C00013700E4B1B789F070ED5184B62681A60DA
:10B7D000A2685A60227B164B1A70E289154B1A80B8
:10B7E00002E03F230B70002000236B7535E000BFA3
:10B7F0003C070020BC1F0020BC290020A410002012
:10B80000FC0F00202D1000201D100020FD0F002037
:10B810000D100020D4210020700200205C020020C6
:10B82000E0210020A6100020E40F0020AC10002032
:10B83000AA100020A81000206B78687D0E2B9FBFF7
:10B84000A54A591C5170A54A98BFD454A24A18B9A8
:10B8500093785C40947000E00020003018BF012015
:10B86000F8BD9D4B0022997D082900F22C81DFE86C
:10B8700001F0050B0F15202B475D6700B52C40F03C
:10B880002281DA75012239E0622C08BF022235E0FC
:10B8900003229A751C765C769C7614E104229A75D4
:10B8A0005A7E997E2244D2B25A760A449A76DC763F
:10B8B00009E105229A755A7E997E2244D2B25A76BF
:10B8C0000A449A769C83FEE006229A755A7E997EF7
:10B8D0002244D2B25A760A449A769A8B02EB042416
:10B8E000A4B2B4F5AC7F82BF7B4A0121D17500229E
:10B8F0009C83DA83002C40F0E68007229A75E2E010
:10B900005A7E997E2244D2B25A760A449A76DA8BCB
:10B91000B2F5AC7F3EBF7049891881F820400132F2
:10B92000998B92B29142DA83E7D9CCE008229A75DA
:10B930005B7EA34200F0C780674B0122DA750DE001
:10B94000674D9A7515F8012D6A70664A9542F9D1CE
:10B95000997E614AA14206D03F232B70624A536808
:10B9600001335360AFE06148016801310160D07D6F
:10B9700010B13E232B70A6E021212970D17E06292B
:10B9800041D004D8022907D0032923D0F8BD1229B9
:10B9900059D0302967D0F8BD5021546A29705449D4
:10B9A0004C60946A0C60116B4FF47A7491FBF4F163
:10B9B000504C218092F878114F4A19B1117841F01A
:10B9C000020102E0117821F002011170012283F8D6
:10B9D000792169E05321297092F82510CE0705D509
:10B9E00092F82420D51E6A426A4100E0024602F025
:10B9F000010183F87811002A56D13F490A7822F0D4
:10BA000002020A7050E04F21297092F82B10CC07E7
:10BA100005D592F82A20D11E4A424A4100E002464A
:10BA200002F0010183F8781122B933490A7822F033
:10BA300002020A7093F84F10304A1170B3F84C109C
:10BA40002F4A118030E05621546B29702D490C800B
:10BA500042F21074916B91FBF4F12B4C2180012187
:10BA600082F87A1120E04921297092F82410274A9F
:10BA7000102988BF10211170254914780022A24294
:10BA80000ED20E7A234D56554E7A234D5655CE7A08
:10BA9000224D565511F80C6F214D56550132EEE7E7
:10BAA00020490A6801320A6093F879310A4A002B6A
:10BAB0003AD092F87A31BBB3002182F8791182F83A
:10BAC0007A111846F8BD0020F8BD1279432A7FF498
:10BAD00094AD0222EA7090E5BC1F0020BC29002032
:10BAE000700200205C0200201C070020E0210020E2
:10BAF000AC100020A8100020A4100020AA100020E4
:10BB000056000020A6100020E40F0020FC0F0020AB
:10BB1000DC1F0020FD0F00200D1000201D10002054
:10BB20002D100020D4210020F8BD0449044B0968E1
:10BB3000002218705A6199611A777047B429002061
:10BB40001C070020F8B5101A0D461F4608F0B0F982
:10BB50000446781B08F0ACF9174B079E196808F0EB
:10BB6000FBF921460546204608F0F6F92946074626
:10BB7000284608F0F1F90146384608F0E5F80CF0DF
:10BB8000A3F90E4908F0E8F908F0D2FB069B294614
:10BB9000186004F100400CF00BF8094908F0DCF9DA
:10BBA000084908F0D1F808F09DFB0028BCBF00F55B
:10BBB0000C40A0303060F8BD4C0000202C7D8E3F42
:10BBC000A00CB34500A00C4644F25063984203DD3C
:10BBD000A0F50C40A0387047034B9842BCBF00F55D
:10BBE0000C40A030704700BFB0B9FFFFF7B5036845
:10BBF000174C184D23600B68174E63600068FFF701
:10BC00009FFC95E80300154B0196009394E80C0007
:10BC1000FFF798FF3668124B60681E606B68114F23
:10BC2000C01A08F045F9104B196808F095F908F0AA
:10BC300059FB2A68236878609B1A3B600B4B1E6097
:10BC40000B4B1B68DA880B4B1A8003B0F0BD00BFAA
:10BC500040270020AC1000204C270020482700205F
:10BC600088270020502700204C000020802700203B
:10BC7000B00E00207C27002070B50446407908F003
:10BC800013F91E4908F01CFA1D4D1E4E2860E07B7A
:10BC900008F00AF9194908F013FAEE606860A07913
:10BCA00008F002F9184908F00BFA184D2860207CBA
:10BCB00008F0FAF8114908F003FA6860A07E08F06D
:10BCC000F3F8134908F0FCF9EE60A860E07908F099
:10BCD000EBF80D4908F0F4F90E4D2860607C08F08F
:10BCE000E3F8064908F0ECF96860E07E08F0DCF85B
:10BCF000074908F0E5F9EE60A86070BD0000C84291
:10BD0000582700200000FA44000020416827002046
:10BD100000007A448C27002010B50C4C23789B0738
:10BD200013D50B4B1B78042B0FD90A4A0A4B10680A
:10BD3000526818605A60FFF703FC084B1A88084BDA
:10BD40001A80237843F00103237010BDA410002053
:10BD5000AA100020AC100020E80F00207C1000206A
:10BD60009C270020164B13B51B681B0325D5154BCC
:10BD7000154C1B7815498DF80030154B20681B7841
:10BD80008DF8013008F0E8F808F0D2FA11498DF882
:10BD90000200606808F0E0F808F0CAFA8DF80300C5
:10BDA000A06808F0C5FA0C4B8DF804001B780A2037
:10BDB00069468DF80530FBF735F902B010BD00BFBC
:10BDC0009029002082290020A42900200000204181
:10BDD000A029002000007A4486290020054A137813
:10BDE00083F001031370044A00231360034A1360B5
:10BDF000B8E700BF862900209C2900209829002050
:10BE0000094A137818441346C0B210F0800F18BFC7
:10BE100080381070054A19781378994201BF0023C1
:10BE20001370014A137070475126002050260020DD
:10BE300010B50A4B0A4A1B7842609C18094A0460F4
:10BE400012789A4225BFD31A0B60C3F180030023F6
:10BE50002EBF4B600B604A6010BD00BF5126002012
:10BE600052260020502600201FB5684602A9FFF781
:10BE7000DFFF044B02981B6803440398184405B085
:10BE80005DF804FBC00500202DE9F04F89B0019357
:10BE900000238246994602910392039A934205DA5F
:10BEA000029A52F8232001339144F6E7019B4D4654
:10BEB000002B56D102F04EFF002852D101987DE0B0
:10BEC0000222404E8DF81C201A0C4FF480578DF83A
:10BED0001D2006201A0A8DF81E208DF81F3002F052
:10BEE0005DFF7761062007F07BF8374B0122376151
:10BEF000D0461A7077612646002007A9042207F071
:10BF000039F8029F4FF0000B039B9B451EDABC469D
:10BF100057F8042B4FEA8B03002A48D0B24236D39D
:10BF200032465AF803100020CDF814C0049307F0ED
:10BF300021F8049BDDF814C05AF8032032444AF873
:10BF40000320DCF800309E1BCCF800601D4B4FF442
:10BF500080521A611D4A2D1B13681C44019B1460FA
:10BF600053B34DB3194B1B68DCB22A19B2F5807F6D
:10BF7000174A88BFC4F58074D26898BF2C46934294
:10BF80009ED3144A00231370134A137014E0002048
:10BF9000D8F8001006F0EEFF57F8043CD8F800205F
:10BFA000F61A1344C8F80030002347F8043C0BF19C
:10BFB000010B08F10408A7E7C5EB090009B0BDE8CB
:10BFC000F08F00BF000C0140BD050020C00500201F
:10BFD0000C000020502600205126002030B50B4CCC
:10BFE0000B4D22782B7885B09A420CD0684602A976
:10BFF000FFF71EFF0123684602A90222FFF744FF54
:10C0000000232B70237005B030BD00BF51260020E7
:10C010005026002030B50E4D0E4C2A78237885B07E
:10C020009A4211D0684602A9FFF702FF002302A935
:10C0300002226846FFF728FFFFF7E2FE20782B7800
:10C040001B1A5842584100E0012005B030BD00BF26
:10C05000512600205026002038B50E4C4FF4805554
:10C0600045F2082002F09AFE6561062006F0B8FF4E
:10C07000094B01222561C7201A70656106F0B0FFE7
:10C08000064A002325611370054A1370054A1360A0
:10C0900038BD00BF000C0140BD0500205026002027
:10C0A00051260020C005002001480249FEF734BF98
:10C0B00000080040A028002001480249FEF72CBFDC
:10C0C00000040040782800204FF080400149FEF72E
:10C0D00023BF00BF5028002001480249FEF71CBFC3
:10C0E000002C01402828002001480249FEF714BF17
:10C0F000002C0140282800202DE9F04F054690F83B
:10C1000050008DB008910592099318B13228A8BF4C
:10C11000322000E0012007F0CBFE0146AA4807F0DC
:10C12000CFFFAA4B04461888002808BF012007F05B
:10C13000BFFEA749069007F00FFF01900199204626
:10C1400007F002FE0146019807F0BAFFA14B0790E5
:10C150001B889A0724D5A049B1F90030B1F9020033
:10C1600083EAE37280EAE071A2EBE372A1EBE07193
:10C1700091420C46B8BF1446B4F5E17F12DA914201
:10C1800003DD0028D8BF404203E0002BCCBF184697
:10C19000584207F08DFE914907F092FF064603E0F2
:10C1A000002601E04FF07E564FF000090395002471
:10C1B000CDF8089063000493894B33F9140007F01D
:10C1C00077FE884907F0C8FE08F08CF807F070FE8B
:10C1D000854907F0C1FE804B824633F9140007F011
:10C1E00067FE7C4B07461B889B077ED0014607F005
:10C1F000ABFD7E4B804633F9140007F059FE014633
:10C20000404607F0A1FD08F06DF8059B5B4298429F
:10C2100003DB059B8342A8BF0346754A0499885EE9
:10C22000099A1B1A32F91400184407F041FE80469F
:10C2300007F040FB70B16F4B40466F4914F8039014
:10C2400007F03EFF0146484606F00CFF6A4907F03A
:10C2500083FE8046287F07F027FE684907F07CFEB2
:10C260008346287A07F020FE0146404607F074FE18
:10C27000634907F071FE08F035F881460BF1004084
:10C2800008F030F8814505DB584608F02BF84845A2
:10C29000A8BF484607F00CFEDFF88891029001998C
:10C2A000404607F059FE59F8241007F04DFD554956
:10C2B0004FEA840B804607F0EDFF38B940465249FB
:10C2C00008F006F820B1DFF8408101E0DFF83481A2
:10C2D00049F80B80A87C07F0E7FD0146404607F0CF
:10C2E0003BFE4A4907F038FE81463A4BB3F800B0AE
:10C2F0001BF0010F40F09880394B049ADFF81C8145
:10C30000D35E002BB8BF5B42B3F5206F4FEA8403C6
:10C310000A9303DD002348F824302AE03C493846DC
:10C3200007F01AFE039B0B90587807F0BDFD0B9A9F
:10C330000146104607F0C4FE514607F003FD01997F
:10C3400007F00AFE58F8241007F0FEFC3149804639
:10C3500007F0A0FF38B940462F4907F0B9FF20B1D8
:10C36000DFF8B48001E0DFF8AC802C4A0A9B42F889
:10C370000380039BD87A07F097FD284B53F82410CD
:10C3800007F0EAFD264907F0E7FD1BF0020F8046A3
:10C390004CD03846029907F0D5FC0146304607F0EC
:10C3A000DBFD0146029807F0CFFC494607464046B0
:10C3B00007F0C8FC0146304607F0CEFD014648466E
:10C3C00007F0C2FC804631E083F9223E780F00205E
:10C3D000BD37863568110020841000200000E1433D
:10C3E0009C0F00200000A03ECDCC4C40DA33002052
:10C3F0008829002048AF0108000020410000A0402B
:10C400006F12033C0000F0C10000F0410AD7A33DC9
:10C410000000A043000040C3000040434021002032
:10C420000AD7233C38210020C846029F8B4B185D59
:10C4300007F03EFD0146504607F08EFD884907F0A3
:10C440008BFD0146384607F07DFC95F851200346E8
:10C450003AB18449844B01EBC4011B68FCF784F8B2
:10C460000346824F504657F824100A9307F06AFC9F
:10C47000019907F025FE47F824A007F1080A5AF8A9
:10C4800024B01037594607F05DFC0146079807F0C5
:10C4900063FD0146584607F057FC83464AF82400DE
:10C4A000385D07F005FD0146584607F055FD704917
:10C4B00007F052FD07460A9B4146184607F044FC28
:10C4C000394607F03FFC0BF09BFA6A4A049B049242
:10C4D000D0520A9BDFF8C0B1184607F003FF4BF8B3
:10C4E0002400404607F0FEFEDFF8B0A1DFF8B0817F
:10C4F0004AF8240007F1004007F0F4FE039B049A79
:10C50000013348F82400039317460CB9012451E67F
:10C51000089A594B9479B3F90430640028345C4389
:10C52000564B6411B3F9040007F0C2FC4FF07A5186
:10C5300007F012FD0BF064FA201A07F0B9FC002C8A
:10C54000B8BF6442322C06464D4C02DD0023A36086
:10C5500025E0069807F0C6FE20F0030007F0A8FCCF
:10C560000190687B07F0A0FC0146304607F0F4FC20
:10C57000019B81464349184607F0A2FD0146484603
:10C5800007F0EAFC07F0AEFEA36818443E4B984261
:10C59000A8BF18463D4B9842ACBFA060A360A368FB
:10C5A0006FF0FF005B13B3F5807FA8BF4FF480737B
:10C5B0009842B8BF184607F07BFC0446304607F0A7
:10C5C00091FEEB785843801107F072FC304B064621
:10C5D0001B78032B12D9B5F84E90B9F5FA7F0DD21E
:10C5E00007F080FEC9F10003984203DB484503468B
:10C5F000A8BF4B46184607F05BFC064695F851204D
:10C600006AB1530803D09A42A8BF1A4600E001223B
:10C61000154B30461F491B68FBF7A6FF064621460F
:10C62000304607F091FB07F05DFE80B2B88000B2A3
:10C6300007F03EFC0BF0E4F9B880304607F052FEFC
:10C64000CBF80800204607F04DFE0023CAF808008A
:10C65000C8F808300DB0BDE8F08F00BF4C210020B5
:10C66000A69B443BE4240020FC2400205021002011
:10C67000F7CC923848250020841000209C0F002021
:10C680000025002000803B45FEFFFF0F020000F068
:10C6900024280020F4240020502500205C250020C0
:10C6A000682500202DE9F04F89B00593BC4B00268A
:10C6B000B3F90290B3F90030B9F1000FB8BFC9F176
:10C6C0000009002BB8BF5B429945B8BF9946804628
:10C6D000B2463446B9F5FA7F04910392A8BF4FF4ED
:10C6E000FA79019000960296AE4D2B88990754D0A6
:10C6F000AB4B610033F91420AB4B33F9143003EB2F
:10C700004202039B5B429A4203DB039B9342A8BF16
:10C710001346A64A8F5E059ADB1B32F914001F18D8
:10C7200007F0C8F890B1A24B384613F804A007F000
:10C73000BFFBA04907F0C4FC0146504606F092FC3E
:10C740009C4907F009FC07F0CDFD074698F8083032
:10C7500064227B4393FBF2F398F81C206FF0040AE9
:10C760000AFB02FA534504DB02EB820A9A45A8BF92
:10C770009A4642F21072904B53F82400384490428B
:10C78000A8BF10468D4A9042B8BF104643F8240017
:10C7900098F812305843031302932D8805F00303D1
:10C7A000012B38D07E4B864933F91430A600009314
:10C7B000019B51F8247093F801E0824B33F9140087
:10C7C00080EAE073A3EBE073B3F5206F16DC009A08
:10C7D00050235A4392FBFEF3042290FBF2F0181A06
:10C7E0000744B7F57A5F784BA8BF4FF47A579F425A
:10C7F000ACBF41F8247041F8243002E0002341F836
:10C8000024308B597D2693FBF6F6019BDB7A73432C
:10C81000402693FBF6F6AA0712D5009A09FB06F507
:10C8200009FB02F70298C9F5FA7303FB0A7703FBC9
:10C8300000534FF4FA7297FBF2F193FBF2F505E027
:10C84000EB0755BF354651460099029D5D4B0427C5
:10C8500033F914305D4A93FBF7F3A25C6FF04F0796
:10C86000534393FBF7F398F851204FEA440BCF184A
:10C8700072B13846069207F01BFB5549554B01EB48
:10C88000C401069A1B68FBF76FFE07F02BFD0746F5
:10C890004C4B514A3BF803003BF9021003B25B1AC0
:10C8A000042193FBF1F102F1040E5EF824302BF821
:10C8B00002000C3252F8240042F8243098F850203C
:10C8C00018444FEA840C08444EF8241082B1CDF885
:10C8D0001CC0069207F0ECFA40493E4B01EBC40144
:10C8E000069A1B68FBF740FE07F0FCFCDDF81CC055
:10C8F0003B4BDFF808E11B5D7A195843202390FB7E
:10C90000F3F3D21A2BF80E20364A5B424CF8023071
:10C91000019B3548354901334CF801504CF8007003
:10C92000019375460CB90124DEE61D4B244EB3F984
:10C930000440049BD6F808E09B790F335B00634307
:10C94000204C5B11B4F90470002BA3EB0707B8BFB0
:10C950005B42322B98F80D400BDC04FB07E4244BC0
:10C96000A342A8BF2346234CA342ACBFB360B4602C
:10C9700001E00023B36098F8034004FB07F31E4C6A
:10C980009B112478032C3CD9B8F84E40B4F5FA7FBB
:10C9900037D26742BB4233DBA342A8BF234630E015
:10C9A0008410002068110020DA330020882900203C
:10C9B00048AF01080000204164210020F0D8FFFFAB
:10C9C000002500209C0F002080C1FFFF4C2100208B
:10C9D000E4240020FC2400206C21002030250020CD
:10C9E0006021002068250020502500205C250020C3
:10C9F000FEFFFF0F020000F0242800204825002041
:10CA00003B46B4686FF0FF0644F34F34B4F5807FC3
:10CA1000A8BF4FF48074B442B8BF344683601E1977
:10CA20000023AE808C60936009B0BDE8F08F2DE9E3
:10CA3000F04F87B00393B34B81461D88029105F0F8
:10CA40000205ADB2019295B1AF4BB3F90250B3F903
:10CA50000030002DB8BF6D42002BB8BF5B429D4235
:10CA6000B8BF1D46B5F5007FA8BF4FF40075CB4693
:10CA70000026A54BA54933F91620A54B4FEA460AD7
:10CA800033F91630520083EAE374A4EBE374B4F58F
:10CA9000206F4FEA860851F8260011DC042493FB2E
:10CAA000F4F3D31A0344B3F57A5F9A48A8BF4FF45E
:10CAB0007A538342ACBF41F8263041F8260002E0A9
:10CAC000002341F8263051F808709BF80B30FF1115
:10CAD0009BF801405F438B4B54431B88BF119B075E
:10CAE0004FEAA41456D08C4B3AF903301A44019BF8
:10CAF0005B429A4203DB019B9342A8BF1346874ADD
:10CB00003AF902209B1A039A32F916201A44049229
:10CB100006F0D0FE049A98B1814B10469B5D0493B9
:10CB200007F0C6F97F4907F0CBFA049B0146184687
:10CB300006F098FA7B4907F00FFA07F0D3FB02469C
:10CB400042F21070784958F8013013448342A8BF6C
:10CB5000034676488342B8BF034648F8013099F847
:10CB6000081099F81C004A4300EB8000D2114142A2
:10CB70008A4203DB8242A8BF0246114699F812207E
:10CB8000641A53431B13FF1A6F436C4303EB67276D
:10CB900001EB64245E4B04223AF9033093FBF2F27A
:10CBA000634B9B5D534399F85120A4EBA31472B1DE
:10CBB0002046049207F07CF95E495F4B01EBC60109
:10CBC000049A1B68FBF7D0FC07F08CFB0446504925
:10CBD0005A4B3AF801003AF903E002B2CEEB0202F6
:10CBE0004FF0040E92FBFEF22AF803009E440C3331
:10CBF00058F80EC058F8030048F80E20604410445E
:10CC000099F8502048F803C08C467AB105910492F7
:10CC100007F04EF94A49484B01EBC601049A1B68DC
:10CC2000FBF7A2FC07F05EFBDDF814C0454BDFF814
:10CC300030E19B5DE21943435B11D21A2AF80E20C2
:10CC400041484249424A5B4248F8004048F8017076
:10CC500048F802300BF1010B74460EB9012608E7C3
:10CC6000294BBCF90470B3F90450029B274E9B7901
:10CC7000D6F808E00F335B006B435B11002BA3EB8E
:10CC80000707B8BF5B42322B99F80D500BDC05FB50
:10CC900007E5304BAB42A8BF2B462F4DAB42ACBF94
:10CCA000B360B56001E00023B36099F8035005FB61
:10CCB00007F32A4D9B112D78032D0CD9B9F84E504E
:10CCC000B5F5FA7F07D26F42BB4203DBAB42A8BF88
:10CCD0002B4600E03B46B5686FF0FF0645F34F3545
:10CCE000B5F5807FA8BF4FF48075B542B8BF354613
:10CCF00083605E190023A6808D60936007B0BDE855
:10CD0000F08F00BF68110020841000200025002053
:10CD10009C0F002080C1FFFFDA330020882900200B
:10CD200048AF01080000204164210020F0D8FFFF37
:10CD30004C210020E4240020FC240020802100203D
:10CD40003025002060210020502500205C25002097
:10CD500068250020FEFFFF0F020000F024280020BD
:10CD6000482500202DE9F04F89B00593AE4B0027F0
:10CD7000B3F90280B3F90030B8F1000FB8BFC8F1C1
:10CD80000008002BB8BF5B429845B8BF9846824662
:10CD9000B946BB463C46B8F5FA7F0492A8BF4FF4AB
:10CDA000FA7802900397A14D2B88990757D0022C4F
:10CDB00055D09D4B610033F914209D4B33F914304D
:10CDC00003EB4202049B5B429A4203DB049B9342C7
:10CDD000A8BF1346974A8E5E059A9B1B32F9140032
:10CDE0001E1806F067FD90B1934B304613F804B05F
:10CDF00007F05EF8914907F063F90146584606F0DE
:10CE000031F98E4907F0A8F807F06CFA06469AF84F
:10CE100008306422734393FBF2F39AF81C206FF0FE
:10CE2000040101FB02FB5B4505DB02EB820293423E
:10CE3000A8BF13469B4642F21072814B53F8240060
:10CE400030449042A8BF10467E4A9042B8BF104678
:10CE500043F824009AF812305843031303932988A7
:10CE600001F00303012B01D1022C3DD16E4B764D15
:10CE700033F91490029BA00093F801E0734B55F82E
:10CE8000247033F9146086EAE673A3EBE673B3F516
:10CE9000206F1CDC022C14D0502303FB09F292FB00
:10CEA000FEF3042296FBF2F69E1B3744B7F57A5F39
:10CEB000674BA8BF4FF47A579F42ACBF2F502B50FF
:10CEC00007E089EAE973A3EBE973642BE4DD00234F
:10CED0002B505D4B7D27C35893FBF7F7029BDB7A02
:10CEE0007B43402793FBF7F78A0713D5022C11D019
:10CEF00008FB07F508FB09F60398C8F5FA7303FB6E
:10CF00000B6603FB00534FF4FA7296FBF2F193FBAE
:10CF1000F2F508E0CB0704D5022C02D0039D594658
:10CF200001E03D46494663000193484B042633F92E
:10CF30001430484A93FBF6F3A25C6FF04F0653435C
:10CF400093FBF6F39AF85120CE18E2B1022C069228
:10CF500030460BD106F0ACFF069A530803D09A4234
:10CF6000A8BF1A4600E001223B4905E006F0A0FFF9
:10CF70003A49069A01EBC401394B1B68FBF7F4FAF6
:10CF800007F0B0F90646314B019A0198D15A354B5A
:10CF90000AB2C05E4FEA840C121A042092FBF0F22F
:10CFA0000198C15203F10801143351F824E053F8F9
:10CFB000240041F82420704410449AF8502043F88B
:10CFC00024E082B1CDF81CC0069206F071FF26491C
:10CFD000234B01EBC401069A1B68FBF7C5FA07F067
:10CFE00081F9DDF81CC0214B214A1B5D0199584392
:10CFF000202390FBF3F073191B1A8B521D4B4042F8
:10D000004CF803601C4B01344CF803501B4B032CB1
:10D010004CF80300029B03F1010302937FF4C3AEBB
:10D0200009B0BDE8F08F00BF841000206811002017
:10D03000DA3300208829002048AF01080000204191
:10D0400064210020F0D8FFFF002500209C0F002065
:10D0500080C1FFFF4C210020F4240020E4240020A4
:10D06000FC24002094210020302500206021002095
:10D0700048250020502500205C2500206825002040
:10D080000028114AB8BF404290FBF2F330B50F4C74
:10D090003C2504FB030068430D4D90FBF2F22D6824
:10D0A0002D7B25B903EB830303EB830301E0C3EB83
:10D0B000031302EB830304FB02020B804FF47A7329
:10D0C00092FBF3F24A8030BD80969800806967FF3A
:10D0D00094100020022803D0431E58425841704744
:10D0E000064B1B681B7823B1054B1868C0F3C04082
:10D0F0007047044B1878C0F3800070479C050020EF
:10D100007C0F0020E133002010B50A4C5E28014658
:10D11000206805D15D2105F044F920683E2105E035
:10D120005D2903D105F03DF920683D21BDE810409F
:10D1300005F037B9B4210020A0F17D03012B70B5B3
:10D1400004460D460A4E05D830687D2105F029F9C0
:10D1500084F020043068214605F023F935B12B888E
:10D160001C4404EB142404F0FF042C8070BD00BFA9
:10D170005811002010B5054C206805F00FF918B1C2
:10D18000206805F008F9F6E710BD00BF281100205F
:10D1900010B50446C0B2FFF7B7FFC4F30720BDE8DF
:10D1A0001040B1E7024B5E21186805F0FAB800BFE5
:10D1B000B421002038B50546054C5E21206805F0F5
:10D1C000F0F820682946BDE8384005F0EAB800BF0D
:10D1D000B421002013B5044601A90068FFF750FFF1
:10D1E0001320FFF7E7FFBDF90400FFF7D1FF1B2075
:10D1F000FFF7E0FFBDF90600FFF7CAFF2320FFF7A6
:10D20000D9FF2368002BB4BF53204E20FFF7C0FF87
:10D2100001A96068FFF734FF1220FFF7CBFFBDF9CB
:10D220000400FFF7B5FF1A20FFF7C4FFBDF90600A1
:10D23000FFF7AEFF2220FFF7BDFF6368002BB4BFEE
:10D2400057204520FFF7A4FF02B010BD674B73B510
:10D250001878FFF73FFF664D04462B78834220D0B5
:10D26000C8B1644B1B68E3B193F90000022300933B
:10D27000614B04211B6800225B78003318BF012337
:10D2800001934FF41653FBF79BF85C4B186040B1C9
:10D2900001232B7005E0594E3068FBF77DF83460B0
:10D2A0002C70574B574D1878FFF714FF2B78044616
:10D2B000834218D088B1544B1B68A3B100220124CB
:10D2C00093F9000008214FF4964300940192FBF774
:10D2D00077F84E4B186028B905E04C4E3068FBF7E4
:10D2E0005BF834602C704A4B4A4D1878FFF7F2FE19
:10D2F0002B78044683422E4643D0002838D0464B34
:10D300001A68002A3DD0D37992F90000002B4FF023
:10D310000202424C08BF02230092002254F823303C
:10D3200001921021FBF74CF83D4B0546186040B3C5
:10D330003C4C94F84A30022B0BD094F89620022AE9
:10D3400001D14C3405E023B1002A04F14C0418BF8C
:10D350000024354B1C6044B1204600214C220AF0C9
:10D3600042F90223256084F84A300123337008E033
:10D370002B4E306805F014FB3068FBF70DF8346075
:10D380002C702A4B2A4D1878FFF7A4FE2B78044600
:10D39000834229D000B3274B1B682BB3264A93F94D
:10D3A00000001268032352782021002A0CBF0822B3
:10D3B0000922009301924FF461430022FBF700F829
:10D3C0001E4B186080B11E4A012313702B701D4B39
:10D3D0001A681D4B1A6007E0184E3068FAF7DCFF38
:10D3E000174B34601C702C7002B070BDA405002077
:10D3F00064100020A005002094100020B42100201B
:10D40000A5050020B41000203811002028110020AC
:10D41000B00500203E110020AC05002044A7010803
:10D42000401100209C11002044110020BC05002068
:10D4300054110020B8050020B40500205811002028
:10D440005C110020B429002060110020642928BF4D
:10D450006421F8B501FB00F5642495FBF4F406465D
:10D46000E4B20027FBB2A34204D29F2001F0D1FC1A
:10D470000137F7E7B4420BD2142195FBF1F5C4EB69
:10D480008410663DC4EB80002844C0B201F0C1FCAA
:10D490000134E4B2B44201D29A20F7E7F8BD2DE995
:10D4A000F74304F08FFE924C6368C31A002BC0F25E
:10D4B000678300F5433303F5A07363608D4B1D78DC
:10D4C000237AC5F38005EB1A18BF012325724DB1ED
:10D4D000002B00F05583884B5A789A7001225A70BD
:10D4E0001A702BE0844A2BB1D37843F00203D37037
:10D4F00093785370D67806F0020101F0FF0339B932
:10D500007D498968411A002903DB06F0010300E028
:10D51000012303F00107784917707BB1F2070DD59D
:10D520000A7905230132D2B2B2FBF3F303EB830392
:10D53000D31A724ADBB20B71D35C4B706E4EDFF8BC
:10D54000088233787BB3F37823F00203F3706C4BDB
:10D550000344AE20B36001F080FC08B101F082FC0E
:10D5600088F80000002800F00B83B02001F075FC63
:10D57000402001F072FC002001F06FFC102001F04F
:10D580006CFC4FF48067013F0020BFB201F03CFC0F
:10D59000002FF8D1384601F0D4FC7278594B53F87B
:10D5A000220001F051FC98F80030002B00F0E882D6
:10D5B0007378062B00F2B282DFE813F00700B002A6
:10D5C000180078006A018701EC014F494F4A504B1F
:10D5D0005048FBF7F4F9012001F0B3FC4D4801F08D
:10D5E00033FC022001F0ADFC4B48ACE14B4F3B68F3
:10D5F0009B0735D5DFF854810A23B8F80010DFF80F
:10D600005091B1FBF3F203FB121399F8001092B2A0
:10D610009BB200913F484249FBF7D1F9FDF718F959
:10D62000012001F08EFC3B4801F00EFC3D4B99F8C7
:10D6300000201868B8F80030067902FB1631642320
:10D640004B43C17802208E1B5643B3FBF6F6F6B26D
:10D6500001F077FC31461520FFF7F8FE032600E0C5
:10D6600001263B681F0540F159822F4B2F491F6847
:10D67000642397FBF3F2096803FB127300912548BA
:10D680002B49FBF79CF9FDF7E3F8304601F059FC14
:10D69000204801F0D9FB00F0F9FF0746701C01F0AB
:10D6A00050FC15203946FFF7D1FE37E20120214F0B
:10D6B00001F047FC204801F0C7FB3B68980749D5BB
:10D6C0001E4A1448B2F90210B2F900300091B2F9C2
:10D6D00004201B4901921B4AFBF771F9FDF7B8F8CA
:10D6E000022001F02EFC0B4801F0AEFB032632E0D5
:10D6F000B4210020E133002090240020CCC6010892
:10D70000404B4C0018A80108D1C60108DAC6010830
:10D71000E5BF0108BD210020E1C6010890290020D5
:10D72000ECC601088C100020981000209C100020EE
:10D7300004C70108A010002019C701086E100020BE
:10D740002FC701083EC701084D020020901000209D
:10D750005400002002263B68D9071AD57B4A7C4832
:10D76000B2F90210B2F900300091B2F904207949FF
:10D770000192794AFBF723F906F10108FDF768F8F1
:10D78000304601F0DEFB5FFA88F8714801F05CFB7F
:10D7900046463B681A0718D5704A6D48B2F9021020
:10D7A000B2F900300091B2F904206A4901926C4A42
:10D7B000FBF705F9771CFDF74BF8304601F0C1FB8C
:10D7C000FFB2634801F040FB3E46664A6149B2F948
:10D7D0000030B2F902205E480092634ADFF8B0914F
:10D7E000B2F90020771C0192604AFBF7E8F8FDF7D8
:10D7F0002FF8304601F0A5FB554801F025FB5449B0
:10D80000D9F80000FAF776FF514809F030FFFFB26F
:10D81000C1B2092909D84B1CDBB2214420224A722B
:10D820000021E21891721946F3E7DFF82481D9F854
:10D8300004004144FAF75EFFFDF70AF8384601F0AC
:10D8400080FB404601F000FB4146D9F80800FAF79A
:10D8500051FF404609F00BFF0236F6B2C7B2092F5E
:10D8600009D87B1CDBB2274420227A720021E218FF
:10D8700091721F46F3E73E4BB3F9000006F018FB28
:10D8800008EB0701FAF736FFFCF7E2FF304657E0F6
:10D890000026384F3B78B34240F240810E2E00F014
:10D8A0003D817008013001F04CFB304605F0D2FD9F
:10D8B0003B78B34206D9202001F0ABFA701CC0B20D
:10D8C00005F0C8FD0236F6B2E3E72B4E2B4996F879
:10D8D000B4271F48FBF773F8012001F032FB1C4806
:10D8E00001F0B2FA264B27491F7819483A46FBF750
:10D8F00066F8022001F025FB154801F0A5FA0C237B
:10D9000003FB0766204996F8B72796F8B637104804
:10D91000FBF755F8FCF79CFF032001F012FB0C48C5
:10D9200001F092FA96F8BC1796F8BA2796F8BB372A
:10D93000074800911549FBF742F8FCF789FF0420DE
:10D9400001F0FFFA024801F07FFAE7E09C0F0020A7
:10D95000BD2100202FC7010842C70108A20F0020E7
:10D960005EDC0108882900207C10002046C70108E1
:10D970002026002038120020F02900204AC7010884
:10D980004829002056C7010867C7010878C7010861
:10D99000142600207C4B1B681B0640F1BB80236AC9
:10D9A000616A7A4A8B421CBF536292F828304FF06A
:10D9B00001011CBF013303F003034FF0000018BF47
:10D9C00082F8283001F0C9FA94F82830704A00260D
:10D9D000D05C01F01EFA0220012101F0BEFA6D4B6D
:10D9E0003620F35C0136C3EBC30393FBF0F0C0B207
:10D9F000062828BF06206038C0B201F00AFA102EAF
:10DA0000EDD1654B65491B78654813F0020F654BF6
:10DA10001A7814BF59234E23FAF7D1FFFCF718FFE9
:10DA2000022001F08EFA5E4801F00EFA5E495F4B6B
:10DA30004E680A685A4892FBF3F25D4996FBF3F38D
:10DA4000FAF7BDFFFCF704FF032001F07AFA54480F
:10DA500001F0FAF9574B58491A885148FAF7AFFFC5
:10DA6000FCF7E2FE042001F06CFA4D4801F0ECF9FD
:10DA7000524B53491A884A48FAF7A1FFFCF7D4FEE3
:10DA800004210A2001F069FA454801F0DDF94D4909
:10DA9000E26A4348FAF793FF4B4EFCF7C5FE0520B8
:10DAA00001F04FFA3E4801F0CFF97268B368474978
:10DAB0003B48FAF784FFFCF7B7FE05210A2001F086
:10DAC0004CFA374801F0C0F93369F2684049D21A7C
:10DAD0003348FAF774FFFCF7A7FE062001F031FA8D
:10DAE0002F4801F0B1F9B2683A492D48FAF767FFBB
:10DAF000FCF79AFE06210A2001F02FFA284801F0CF
:10DB0000A3F935491522264809F0DCFDFCF78CFE07
:10DB1000072015E7F37843F00203F370002D2FD1AF
:10DB20002E4B00219B791220032B97BF2C4A3F25B7
:10DB30009B181D7F01F011FA284601F06AF91320A5
:10DB4000002101F00AFA274B1B78002B264B18BF47
:10DB500072201B7808BF2120002B18BF522001F033
:10DB600058F91420002101F0F8F994F83050084BCE
:10DB7000585D013505F0030501F04BF984F830508C
:10DB800003B0BDE8F08300BF90290020B42100203D
:10DB90008AC701082D100020A41000208FC701089B
:10DBA000BD210020AA100020AC1000208096980013
:10DBB000A0C70108A6100020ADC70108E40F00208F
:10DBC000B5C70108BCC701081C070020C3C701086E
:10DBD000CCC70108D3C701085C020020AC0D0020AF
:10DBE00018A80108DB0D0020400E0020084BDA6861
:10DBF000D10709D4DA68520708D4DB6813F0100F94
:10DC000014BF032004207047012070470220704792
:10DC10000020024003788B4286BF024B33F811008C
:10DC200000207047E82100200022134670B52349E8
:10DC300014180C44247E83EA0423082413F4004FB0
:10DC40004FEA430318BF83F4815304F1FF3418BF34
:10DC500083F0010314F0FF049BB2EFD10132192AC3
:10DC6000E5D100F1190200F11A050A440D44167EAF
:10DC70002A7E02EB062292B29A421ED10F4B93F8F3
:10DC80003950E2B2AA4215D2431C03EB4203DBB285
:10DC9000CA1801330B44127E1B7E03EB02239BB296
:10DCA0004FF4AF6253431B1303F5487321F814304C
:10DCB0000134E6E7012381F83A3070BDE821002005
:10DCC00003788B420BD9074B89001A78064B19440D
:10DCD000C86B02B1400800F5777080B27047002031
:10DCE000704700BF3C120020E821002007299DBF9B
:10DCF000034B03EB8101B1F86C000020704700BFBB
:10DD0000E8210020034B03EB4101B1F88C00C0086F
:10DD1000704700BFE821002008B5084B03EB8101E4
:10DD2000D1F8AC0006F0C0F8054906F015F9054930
:10DD300006F00AF806F0FCFA80B208BDE8210020DF
:10DD40000000203F00005C44014B33F81100704795
:10DD5000CC290020024B03EB4101B1F8F4007047DD
:10DD6000E8210020024B03EB4101B1F8F4007047B9
:10DD7000E82100200020704770B5054604F022FA23
:10DD8000314CD4F80C31C4F80C01C31AB3F5FA5F66
:10DD9000C4F8103182BF002384F8143184F815319F
:10DDA00094F814312BB9A12D02BF274A012182F822
:10DDB000151194F81511244A29B1D118EDB2013387
:10DDC0000D7682F8143194F8145194F81631AB4260
:10DDD00039D11D4B93F81731052B02D0062B03D0F8
:10DDE0002CE00020FFF720FF637E1E2B26D10020B1
:10DDF0000246C1B26B1E994219DA21440B7E0821FA
:10DE0000DBB283EA0206F60744BF83F01803C3F3CC
:10DE1000460301F1FF3154BF5B0843F0800311F06A
:10DE2000FF01C2F34702ECD101301A46E1E7234477
:10DE30001B7E9A4202D10320FFF7F6FE002384F8EE
:10DE4000153184F8143170BDE821002010B5044666
:10DE500004F0B8F941F288310E4BE4B2D3F818213E
:10DE6000C3F81801821A8A42C3F81C2184BF002219
:10DE700083F8202193F8202106490F2A134418BF64
:10DE8000013283F8214112BF81F82021012381F85A
:10DE9000313110BDE821002010B5044604F092F99C
:10DEA00041F288310E4BD3F83421C3F83401821A81
:10DEB0008A42C3F8382184BF002283F83C2193F8BA
:10DEC0003C210749142A134418BF013283F83D410D
:10DED00012BF81F83C21012381F8523110BD00BFEF
:10DEE000E821002038B5044604F06CF9274A274998
:10DEF000D2F85431C2F85401C31AB3F57A6F84BF13
:10DF0000002382F8583192F8583133B9A82C3BD10C
:10DF100081F85931A1F85A3106E0022B02D181F87B
:10DF20005C4101E0242B02D8D11881F85D4192F8C0
:10DF30005C1101330231DBB249008B42134D82F890
:10DF4000583118DAB5F85A31E0B283EA00200823D4
:10DF500010F4004F4FEA400018BF80F4815003F1E5
:10DF6000FF3318BF80F0010013F0FF0380B2EFD140
:10DF7000A2F85A0138BD01318B4201BF002385F858
:10DF80005831012385F8593138BD00BFE821002000
:10DF900010B5044604F016F940F6AC510F4AD2F819
:10DFA0008431C31A8B42C4BF002382F8883192F8AF
:10DFB0008831D11881F8894123B90F2C0DD1074937
:10DFC000C1F884010133DBB2192B044982F888318E
:10DFD0000CBF0123002381F8A23110BDE8210020ED
:10DFE0004FF6FE7302681340036000230360436032
:10DFF0008360C360284B984201D1284A27E0284B10
:10E00000984201D1254A2AE0264B984201D1234A61
:10E010002DE0254B984201D1204A30E0234B984215
:10E0200001D11E4A33E0224B984204D11B4A536867
:10E0300043F470032EE01F4B984204D1174A5368F3
:10E0400043F0706326E01C4B984204D11B4A53688E
:10E0500043F00F031EE01A4B984204D1174A53684D
:10E0600043F0F00316E0174B984204D1134A53686B
:10E0700043F470630EE0144B984204D10F4A536886
:10E0800043F4704306E0114B984204D10B4A5368A5
:10E0900043F47023536070470800024000000240C0
:10E0A0001C00024030000240440002405800024080
:10E0B0006C0002408000024008040240000402405C
:10E0C0001C04024030040240440402405804024050
:10E0D0001F4A10B5536803F00C03042B03D0082B20
:10E0E00004D01C4B14E01C4B1B6811E053685168B2
:10E0F000C3F38343C90303F1020301D4174906E0C4
:10E10000516811F4003F1449096818BF49084B438E
:10E11000036053681249C3F30313CC5C0368E34004
:10E1200043605468C4F302240C5D23FA04F4846051
:10E130005468C4F3C2240C5DE340C3605268C2F368
:10E1400081320A44127CB3FBF2F3036110BD00BFBD
:10E150000010024000127A002C00002000093D004F
:10E1600038A8010810B50446FFF740FD012806D184
:10E170001CB1FFF73BFD013CF8E7052010BD002C6A
:10E1800008BF052010BD0A88F0B54B888E88B1F80D
:10E1900008E0CC88002A3AD1028C43F0010322F037
:10E1A00001021204120C0284058B078CADB225F01B
:10E1B000F30545EA0E1189B241EA06027A49BFB277
:10E1C000884212D001F5006188420ED0B0F1804F34
:10E1D0000BD0A1F59831884207D001F580618842C3
:10E1E00003D001F58061884202D127F0020701E0E7
:10E1F00027F00A071F4302830784038B23F00C03D5
:10E200001B041B0C0383038B9BB21C4344E0042AB6
:10E2100044D1028C22F010021204120C0284018BF1
:10E22000058C21F440721205120D42EA0E325E494D
:10E2300092B242EA06228842ADB292B212D001F501
:10E24000006188420ED0B0F1804F0BD0A1F598311B
:10E25000884207D001F58061884203D001F58061D2
:10E26000884207D125F0200141EA03139BB243F015
:10E27000100304E025F0A00143F010030B430283D8
:10E280000384038B23F440631B041B0C0383038B65
:10E290009BB243EA0424A4B20483F0BD082A028C92
:10E2A0003ED122F480721204120C0284828B3E4D05
:10E2B00092B222F0F307018C47EA0E1292B2A84202
:10E2C00089B242EA060212D005F50065A8420ED0D6
:10E2D000B0F1804F0BD0A5F59835A84207D005F5D1
:10E2E0008065A84203D005F58065A84207D121F4D6
:10E2F000007141EA03239BB243F4807304E021F4EC
:10E30000206143F480730B4382830384838B23F067
:10E310000C031B041B0C8383838B9BB21C4341E0C7
:10E3200022F480521204120C0284858B018C25F495
:10E3300040752D052D0D45EA062545EA0E321A4D8C
:10E3400089B2A84292B212D005F50065A8420ED05B
:10E35000B0F1804F0BD0A5F59835A84207D005F550
:10E360008065A84203D005F58065A84207D121F455
:10E37000005141EA03339BB243F4805305E047F672
:10E38000FF5543F480530D402B4382830384838BDA
:10E3900023F440631B041B0C8383838B9BB243EAEF
:10E3A0000424A4B28483F0BD002C0140016830B580
:10E3B000CD43154B1C682C401C605A682A405A609B
:10E3C000027902F1804202F5823214682143116021
:10E3D00002689C68D5432C409C60D9682940D9606C
:10E3E0004179102909BF996801F18043114399606F
:10E3F00015BF03F58233D96819680A4316BF0A436B
:10E40000DA601A6030BD00BF00040140054B1A6895
:10E410005B69034004D0104214BF01200020704704
:10E420001846704700040140CA78F0B5D40648BFCA
:10E430008C780D8802F00F0348BF234315F0FF0FBF
:10E440001DD0016800240126A64006EA0507B74250
:10E4500011D14FEA840E0F2606FA0EF621EA0601C4
:10E46000282A03FA0EF641EA060101D1476102E0CB
:10E47000482A08BF07610134082CE4D10160FF2D50
:10E480001FD94168002404F108070126BE4006EAAE
:10E490000507B74211D14FEA840E0F2606FA0EF691
:10E4A00021EA0601282A03FA0EF641EA060101D103
:10E4B000476102E0482A08BF07610134082CE2D115
:10E4C0004160F0BD0F4B1A6842F001021A605968B2
:10E4D0000D4A0A405A601A6822F0847222F480328F
:10E4E0001A601A6822F480221A605A6822F4FE0226
:10E4F0005A604FF41F029A60044B4FF000629A601A
:10E50000704700BF001002400000FFF800ED00E07F
:10E510002DE9F8435B4C0368013AC4F8A4318388C1
:10E520000D46A4F8A831072A42D8DFE802F0040A11
:10E53000101822292F35B4F8A4310B80B4F8A63175
:10E5400013E0B4F8A6310B80B4F8A43105E0B4F8B8
:10E55000A4315B420B80B4F8A6315B4205E0B4F80D
:10E56000A6315B420B80B4F8A4316B80B4F8A831BB
:10E570001DE0B4F8A4315B420B80B4F8A63112E080
:10E58000B4F8A6310B80B4F8A4310CE0B4F8A4318F
:10E590000B80B4F8A63105E0B4F8A6315B420B80DD
:10E5A000B4F8A4315B426B80B4F8A8315B42AB8015
:10E5B000354B1B79002B62D1B5F9000005F078FCD2
:10E5C0008046B5F9020005F073FC0746B5F9040072
:10E5D00005F06EFCD4F8AC110646404605F0BCFCD4
:10E5E000D4F8B8118146384605F0B6FC01464846D5
:10E5F00005F0AAFBD4F8C4118146304605F0ACFC06
:10E600000146484605F0A0FB09F0FAF9D4F8B0112C
:10E610002880404605F0A0FCD4F8BC11814638465D
:10E6200005F09AFC0146484605F08EFBD4F8C81167
:10E630008146304605F090FC0146484605F084FBD3
:10E6400009F0DEF9D4F8B4116880404605F084FC86
:10E65000D4F8C0118046384605F07EFC014640469D
:10E6600005F072FBD4F8CC110746304605F074FC77
:10E670000146384605F068FB09F0C2F9A880BDE8FC
:10E68000F88300BFE82100202C00002038B50F4B94
:10E690001B689C890E4B186880F31000201A05F047
:10E6A00007FC0C4905F058FC0546204605F000FC27
:10E6B0000146284605F004FD05F014FE6428A8BFB5
:10E6C000642020EAE070C0B238BD00BF8C1000208A
:10E6D0009C1000200000C84244F6FB71084B1A68E9
:10E6E000137803EB431300FB03135078C0EB0030A7
:10E6F000B3FBF0F39078B3FBF0F080B2704700BF4B
:10E700008C10002008B50A480A2290F8D13100EB9D
:10E710004303B3F8E01100F5F87089B220F8081C43
:10E7200003F042FE80B2FFF7D7FF024B188008BD0E
:10E73000E821002090100020114BD3F8783203EB31
:10E740004002117E01290DD002290FD0022805D9DF
:10E75000032807D10B4A1268D20401D5D889704723
:10E76000988A7047084B33F810007047507E00EBD2
:10E77000800000EB800000F2EE2080B2704700BF06
:10E78000E821002090290020CC29002042F201023B
:10E79000034B1B681A420CBF01200020704700BFCA
:10E7A000902900200F4B10B593F87C221C46012ABB
:10E7B0000CD007D3022A0CD10B4AD36883F008038C
:10E7C000D36006E0084B08221A6102E0064B0822DB
:10E7D0005A6103F0F7FC00F5F42000F59070C4F8DE
:10E7E000800210BDE8210020000C014037B5062250
:10E7F000044603216B461E2003F04EFB9DF80130BA
:10E800009DF80000154D43EA002000B205F050FBD2
:10E81000296805F0A1FB05F065FD9DF80330208017
:10E820009DF8020043EA002000B205F041FBA96810
:10E8300005F092FB05F056FD9DF80530A0809DF88F
:10E84000040043EA002000B205F032FB696805F0DD
:10E8500083FB05F047FD608003B030BD340000202D
:10E8600010B5054C23681869FFF7D0FD18B123686F
:10E870001A69024B5A6110BDF012002000040140D9
:10E8800038B50D4B0D4D99680D4B1A681C465288D2
:10E89000114203D003F096FC286007E003F092FCDD
:10E8A0002B68984282BFC01A064B186023685A68CA
:10E8B000054B5A6138BD00BF000C01407024002098
:10E8C000180700200000002000040140084A1368D7
:10E8D0009B020BD5074B002119704FF6FE730649BA
:10E8E000086803400B604FF400135360704700BF8B
:10E8F00000000240E03300206C0002402DE9F047A8
:10E90000664D6B686649581C0A788E4602F0FF0611
:10E910000AB10346F6E737466B60687CEB6895F80A
:10E920001080AA7C39B2202900F09C80DFF880C1D9
:10E930000CEB8103DC789B783CF82110C3F1FF03DA
:10E940009BB2002B65D04FF03C0CB1FBFCF9C3F13E
:10E95000FF0363431B12B9F1050F5DD8DFE809F02F
:10E96000030B1A293A4AE01A4143B1FBFCF0DAB230
:10E970001044C0B251E0B1FBFCF00CFB101189B2A5
:10E98000DAB2C1F13C01E31A4B43B3FBFCFC204675
:10E9900094442CE0B1FBFCF00CFB1011E21A89B29C
:10E9A0004A43B2FBFCF25FFA83F84244D2B22046FB
:10E9B00032E0B1FBFCF90CFB191189B2E01AC1F18C
:10E9C0003C014843B0FBFCF05FFA83F84044C0B21E
:10E9D000224621E0B1FBFCF80CFB1811D8B289B239
:10E9E000E31A01FB03F2B2FBFCFC224684445FFA0B
:10E9F0008CF412E0B1FBFCF80CFB181189B2D8B210
:10EA0000C1F13C01E31A4B43B3FBFCF20244D2B226
:10EA100003E02246204600E044464FEA042C4CEA3C
:10EA2000004C4CEA020C17234FF0010808FA03F8D7
:10EA300006F1170118EA0C0FA1EB0301DFF874804F
:10EA400014BF4FF011094FF0090989B213F1FF33D8
:10EA500008F80190E8D218360137B6B2BFB2114BB0
:10EA6000A0465FE7EB6001238EF8003040F22A33C6
:10EA7000AA740D4A69810D4985F8108068742E8149
:10EA8000536000238B840B889BB243F001030B80FF
:10EA9000136843F001031360BDE8F0877024002081
:10EAA000E0330020802400206C000240000400407D
:10EAB000220D00207102002001F0030301F0FC018F
:10EAC00001F1804101F5803110B59B008C680F2267
:10EAD0009A4024EA02028A608A68984002438A6067
:10EAE00010BDF0B5B1F800E000234EFA03F2D507EF
:10EAF00025D58E784FEAD30CF40648BFCC7806F0C3
:10EB00000F0203F0070748BF2243BF0050F82C5004
:10EB10000F24BC4025EA0404BA402243282E40F8C2
:10EB20002C2005D1C46801229A4024EA020205E0A3
:10EB3000482E04D1C46801229A402243C2600133A6
:10EB4000102BD2D1F0BD2DE9F0437A4A87B013687B
:10EB5000904693B11A681AB17749886902438A616D
:10EB60009A889868ADF8002002228DF80320694643
:10EB700004228DF80220FFF7B4FF322003F047FB98
:10EB8000002111221E2003F0C7F9012160221E205E
:10EB900003F0C2F9642003F03AFB002402A8FFF757
:10EBA00025FE274626460A25022101221E2003F0C3
:10EBB000B3F9322003F02BFB02A8FFF717FEBDF9D3
:10EBC0000820BDF90A1014448A42A8BF0A46BDF9BC
:10EBD0000C300F4493421E44A8BF134613F5805FC8
:10EBE00009DD564A013DD36883F01003D360DBD1C1
:10EBF0004FF0010901E04FF000091E200021122210
:10EC000003F08AF90A25022101221E2003F084F96B
:10EC1000322003F0FCFA02A8FFF7E8FDBDF9082056
:10EC2000BDF90A10A41A8A42A8BF0A46BDF90C30E1
:10EC30007F1A9342A6EB0306A8BF134613F5805F25
:10EC400007DD3E4A013DD36883F01003D360DAD17B
:10EC500001E04FF00009204605F02AF90146384846
:10EC600005F02EFA374D20F000402860384605F0B8
:10EC70001FF90146324805F023FA20F00040686091
:10EC8000304605F015F901462F4805F019FA20F035
:10EC90000040A860002170221E2003F03DF90121F0
:10ECA00020221E2003F038F91E200221002203F04A
:10ECB00033F9642003F0ABFAB9F1000F04D14FF03F
:10ECC0007E532B606B60AB60D8F80030194E1A7B16
:10ECD00062B31A7D52B3184900258A69012442F0B3
:10ECE00001028A61187B197DFFF7E6FE174803F0E1
:10ECF00037FB3368164A1B6904A8536104930C233D
:10ED00008DF815308DF814508DF81640FFF74EFB36
:10ED1000336801A85B7D8DF806508DF8043003231D
:10ED20008DF805308DF8074004F006F907B0BDE80E
:10ED3000F08300BFF012002000100240000C0140E0
:10ED400000406F463400002001C05E4661E80008C4
:10ED5000000401400F4B73B518781C4698B1052389
:10ED60000D4D8DF800304FF4805600238DF80130A2
:10ED700001A86E616946022204F0FCF82E619DF83C
:10ED8000050000F0010000F00100207080F001009B
:10ED900002B070BDBD050020000C0140064B70B5EF
:10EDA00006461C461D68FFF7D5FF18B923685B1B94
:10EDB000B342F8D970BD00BFB4290020F7B50323D2
:10EDC0008DF80430030C8DF805308DF80700030A28
:10EDD00006200F4614468DF80630FFF7DFFF78B1A6
:10EDE000084D4FF4805601A904226E61002004F002
:10EDF000C1F838460021224604F0BCF820462E61B6
:10EE000003B0F0BD000C0140024640213C2003F05D
:10EE100083B870B500EB8000094CA0F1A1059C38C7
:10EE200025440444074B15F8010F1E787040FFF786
:10EE3000EBFFA542F6D13046BDE87040E4E700BFE5
:10EE40004CA80108E533002010B5441E14F8010F4A
:10EE500010B1FFF7DEFFF9E710BD024680213C202C
:10EE600003F05AB810B5D420FFF7F7FF8020FFF762
:10EE7000F4FFA820FFF7F1FF3F20FFF7EEFFD320BC
:10EE8000FFF7EBFF0020FFF7E8FF4020FFF7E5FF6B
:10EE90008D20FFF7E2FF1420FFF7DFFFA120FFF72F
:10EEA000DCFFC820FFF7D9FFDA20FFF7D6FF1220DA
:10EEB000FFF7D3FF8120FFF7D0FFCF20FFF7CDFF73
:10EEC000D920FFF7CAFFF120FFF7C7FFDB20FFF7CC
:10EED000C4FF4020FFF7C1FFA420FFF7BEFFA6201C
:10EEE000FFF7BBFFAF20FFF7B8FFA620FFF7B5FF86
:10EEF000AE20FFF7B2FF2020FFF7AFFF0020FFF7A3
:10EF0000ACFFB020FFF7A9FF4020FFF7A6FF0020CD
:10EF1000FFF7A3FF1020FFF7A0FF4FF48064013C30
:10EF20000020A4B2FFF770FF002CF8D18120FFF77A
:10EF300094FFC820FFF791FFAF20FFF78EFF01205D
:10EF400010BD08B55038C0B2FFF787FF0020FFF7AB
:10EF500084FFBDE8084010207FE710B50446503913
:10EF6000C8B2FFF77AFF04EB4400400000F00E0047
:10EF7000FFF773FF06206043BDE81040C0F30310A5
:10EF800010306AE7012828BF01202DE9F04F06461E
:10EF9000734F142000FB0671724BD1F8A4421E7609
:10EFA0005C61714BD1F8B422DD69B1F8AC822A43BF
:10EFB000DA61A288B1F8AEA222F44072D1F8A85268
:10EFC000120489B0120C4AEA0809A28003A9C5F804
:10EFD000109002228DF80E0028460193ADF80C9097
:10EFE0008DF80F20FFF77DFD019B00971F464FF026
:10EFF000080BAA6818EA020F03D10A2003F0FCF8F4
:10F00000F7E70A20C5F8148003F0F6F8C5F8108079
:10F010000A2003F0F1F8BBF1010BEAD1C5F814A006
:10F020000A2003F0E9F8C5F814800A2003F0E4F898
:10F03000C5F810800A2003F0DFF80222C5F810A0FE
:10F04000284603A98DF80F201C228DF80E20ADF85C
:10F050000C90FFF746FD454A03A894423A690BBF5E
:10F0600042F4001242F480023A613A610BBF3A69FD
:10F070003A6922F4001222F480023A61A38823F450
:10F0800040731B041B0CA38023889BB243F0010335
:10F090002380A588FFF71CF80599354B25F03F051F
:10F0A000B1FBF3F32D042D0C1D43ADB2A5802288D6
:10F0B000002522F001021204120C22802D4A03A81E
:10F0C000B1FBF2F100298AB208BF012242F40041EB
:10F0D0004FF4967253434FF47A7293FBF2F3013379
:10F0E0009BB22384A1832388009A9BB243F001033F
:10F0F0002380238823F4816323F002031B041B0C69
:10F1000023804FF480432381142303FB062696F8C3
:10F11000B13201248DF80C308DF80D508DF80E5061
:10F120008DF80F4003F008FF96F8B0329DF80F20DD
:10F130008DF80C308DF80D508DF80E501AB103A8D3
:10F1400003F0FAFE08E05A0903F01F039C4002F1A5
:10F150002003094A42F8234009B0BDE8F08F00BF00
:10F160004CA8010870240020001002400054004008
:10F1700040420F00804F120000E100E038B500244B
:10F180000B4D6059254403F001FD696811B1094830
:10F19000F9F72AFCA96811B10748F9F725FC0748D7
:10F1A000103403F0F3FCB4F5F07FE9D138BD00BFB3
:10F1B00018AB01080CC8010812C8010828D20108C0
:10F1C00070B50546284608F052FA064658B91A4B5B
:10F1D0001A485A791A4BBDE8704003EB8203D3F802
:10F1E000DC11F9F701BC28461649324608F048FA06
:10F1F00060B9154803F0CAFC144C54F8041F19B147
:10F200001348F9F7F1FBF8E7124805E00024124B28
:10F2100053F8241021B91148BDE8704003F0B6BC82
:10F220002846324608F02CFA01340028EFD1024B70
:10F230000B4D5C71C6E700BFF029002018C801081B
:10F2400018AB010824C8010829C80108F4AC01085A
:10F250003CC8010828D20108F8AC0108F2C5010831
:10F2600007C30108F0B585B0044608F000FA082885
:10F2700026D1621EE01D1F4912F8013F096819449A
:10F28000497801F00301022908BF203B8242137034
:10F29000F1D1254604F1080715F8016B16483146EF
:10F2A00008F0D7F920B12846314608F0D2F910B15C
:10F2B000F8F73CFB1CE0BD42EED12046FAF758F8C7
:10F2C0000E4803F063FC00230D4A04A91A4492F887
:10F2D0008A210A440849595C0133082B02F80C1CA6
:10F2E000F2D10023074801A98DF80C30F9F77CFB17
:10F2F00005B0F0BD6800002062DC010840C80108CC
:10F30000F0290020CCD001082A4B2B4C1E6880B578
:10F310002068F9F71DF83046F9F71AF820684179A6
:10F320008D0703D441F0020103F02CF8234B08228F
:10F330001A61234D10221A612B689A0341BF0623DC
:10F340006371E37923F0010344BF43F00203E371E7
:10F35000206803F023F890B1184F08237B61164B07
:10F36000186803F018F88046FCF708F908B102F0B5
:10F3700095F83046414603F014F808233B613046C7
:10F3800003F00CF878B10D4F4FF01008C7F8148057
:10F390003046D4F8009002F0FEFF0146484603F0E4
:10F3A00000F8C7F810802B689B03D1D5FEF777F8DB
:10F3B000CEE700BF642900208C240020000C01400F
:10F3C000902900202DE9F041054608F050F92C4B1A
:10F3D00004469E6888B92B4803F0D8FB2A4B53F8A3
:10F3E000241041B10123A340334202D02748F9F74A
:10F3F000FBFA0134F2E7264821E028462549224657
:10F4000008F03EF958B9244803F0C0FB234C54F8E7
:10F41000041F0029EFD01D48F9F7E6FAF7E72B782B
:10F4200000262D2B03BF013504F1FF344FF00108F6
:10F430004FF00008144B53F8267027B91848BDE860
:10F44000F04103F0A3BB28463946224608F018F9DC
:10F4500098B90120B040B8F1000F03D0F9F758FC7B
:10F46000104802E0F9F75CFC0F4803F08FFB3946C7
:10F47000BDE8F0410D48F9F7B7BA0136DAE700BF49
:10F48000F029002046C8010860AD01083CC8010809
:10F4900028D2010824C8010850C801085CAD010841
:10F4A000F2C501085CC8010865C80108CBD0010895
:10F4B00010B5084803F06AFB074B00241C741C6459
:10F4C000064B1C7003F00EF903F004FD044B1C60A6
:10F4D00010BD00BF6DC801088C240020E633002059
:10F4E0006429002070B5064600240B4BE518AA8855
:10F4F00016420AD0E1580948F9F776FA2846002161
:10F5000003F0D5FA064803F041FB40F69443143467
:10F510009C42EAD170BD00BFC4B1010899C801087E
:10F5200028D2010808B50848F9F75EFAFCF794FDFF
:10F53000FFF710FC18B9642002F069FEF8E70348F1
:10F54000BDE80840F9F750BAA3C80108B0C80108DF
:10F550002DE9FF410A48068885684488B0F8048090
:10F56000C768FCF781FCCDF8008002900197314616
:10F570002A4623460348F9F737FA04B0BDE8F0817C
:10F580000C000020B8C80108F0B504788BB005461F
:10F590000CB1002436E04A4B19680E2303FB04111A
:10F5A000B1F91D51B1F91921B1F91B31009591F84B
:10F5B000205101F58C70019591F8215101F5907160
:10F5C000029590F90700039091F902103D480491CB
:10F5D00021460134F9F708FA082CDCD16DE02D2B17
:10F5E00014D1072C1BDC284608F096F80AAB661CE1
:10F5F00003EB440424F8100C15F8013F303B092BB1
:10F60000FAD934462B78002BE9D104E0A3F130027B
:10F61000092A09D8E5E7082CBDF8182009D00BB055
:10F62000BDE8F040F8F782B9202BF8D10135264625
:10F63000E7E7072AF3D840F2DC55BDF81A00204B63
:10F64000A0F2EE2189B2A9421B68E8D8BDF81C10CF
:10F65000A1F2EE24A4B2AC42E1D8BDF81E7004B20F
:10F660003EB2A642DBDB0DB2AE42D8DCA542D6DB11
:10F67000BDF92440642CD2D1BDF8266034B2112CDF
:10F68000CDDCBDF82050B42DC9D8BDF82240B42C33
:10F69000C5D812B24FF00E0E0EFB0233A3F81B11A9
:10F6A0006421A3F81901A3F81D7183F8205183F890
:10F6B000214183F81F1183F822610BB0F0BD00BF18
:10F6C000B80F002015C90108F0B504468FB02046D8
:10F6D00007F0CDFFC5B21DBBAB4803F057FAAB4CEA
:10F6E00094F8D61009B9AA4853E049B294F8D42046
:10F6F00094F8D530009194F8D710A648019194F968
:10F70000D8100734029194F9D210039194F8D310D1
:10F71000049129460135F9F767F9102DE0D1E2E7A8
:10F7200020469D49052207F0ABFF0546B8B929469A
:10F730009A48702207F057FF2846994B19680E2304
:10F7400003FB001301300022082883F8232183F8EB
:10F75000242183F8252183F82621F0D112E12046C7
:10F760009049042207F08CFF05462046002D4AD11F
:10F77000202107F06EFF002800F00481461C30466F
:10F7800007F075FF2C460746874B53F824502DB9D8
:10F7900086480FB0BDE8F040F9F726B93046294653
:10F7A000FAB207F06DFF01340028EDD1774A164612
:10F7B00002F17001002382F8DA3082F8D63082F844
:10F7C000D53082F8D43007328A42F3D1784901EB40
:10F7D000C40191F8A022934210DAD1F8A472C3EBCD
:10F7E000C302B0183A44176800F1D401C0F8D470CD
:10F7F00090880133888092798A71E7E729466D48BD
:10F80000F9F7F2F88FE06C49072207F039FF054657
:10F810002046002D49D1202107F01BFF064607F0A6
:10F8200026FFC4B26CBB6548F9F7DEF82146644890
:10F830000134F9F7D9F80E2CF8D15548F9F7D4F876
:10F84000002460482146F9F7CFF80025544A0123E7
:10F8500011680E2202FB0412D2F82321AB4013429E
:10F86000594B5A495A4808BF19460135F9F7BCF8AF
:10F870000E2DEBD146480134F9F7B6F8082CE0D14B
:10F8800080E03046534907F04BFF2C4600284CD00F
:10F89000022C4FD007F040FF06AB43F824004D493F
:10F8A000002007F03DFF0134F0E74A4907F038FF38
:10F8B000002460B1082C38D007F02EFF06AB43F8C7
:10F8C00024004449002007F02BFF0134F1E7082C05
:10F8D0002BD1069B0F2B28D8DDF81CE0BEF1070FBB
:10F8E00023D8089F0D2F20D8099E06F16402C82A4C
:10F8F0001BD80A9DFF2D18D80B98642815D80C9991
:10F90000642912D8884210DA0D9C032C0DD8324A93
:10F91000C3EBC303134483F804E05F719E71DD7190
:10F92000187259729C722D4CD1E60FB0BDE8F040B0
:10F93000F7F7FCBF069B072B20D807990D291DD888
:10F940000278722A0DD06E2A18D1154A0E2012683C
:10F9500000FB032301228A40D3F8231121EA02028B
:10F9600009E00F4A0E20126800FB032301228A409F
:10F97000D3F823110A43C3F8232101E0F7F7D6FF98
:10F980000D4CA4E60FB0F0BD3DC90108F0290020E0
:10F9900028D2010868C90108C2C50108C42A00208C
:10F9A000B80F0020EDC50108F8AC0108F2C5010848
:10F9B00018AB010801C6010835C9010816C80108BD
:10F9C00084C90108B9C701085DD50108A3D401089D
:10F9D00089C901088DC90108C02A002007C3010890
:10F9E0002DE9F743047805468CB9324D95F8AF12EE
:10F9F000B5F8AC2295F8AE322F480091214601347B
:10FA0000F8F7F2FF102C05F10405EFD14EE007F0F6
:10FA100083FE0F28044636DC2846202107F019FE15
:10FA2000264EE4B2D6F84480451CA40000272846A0
:10FA300007F072FE5FFA87F9B9F1010F83B208D0BF
:10FA4000B9F1020F0BD0B3F5B47F24D2726C13530B
:10FA50000AE0FF2B1FD8736C2344987004E0FF2B3F
:10FA600019D8736C2344D87028462C2107F0F1FD77
:10FA7000054608B1013502E0B9F1020F0BD101379B
:10FA8000032FD4D112E00E4800210F2203B0BDE8AD
:10FA9000F043F7F7C8BE08EB04000021042207F08A
:10FAA000A2FD03B0BDE8F043F7F740BF03B0BDE8E7
:10FAB000F08300BFF02900208FC901088C240020AA
:10FAC00080C501082DE9F04FAC498BB0044607F022
:10FAD00093FDAB49002820460CBF0125072507F000
:10FAE0008BFDA8490028204608BF022507F084FDA9
:10FAF000002808BF0425E90740F1FB80A24803F075
:10FB000045F8002002F04CFEA04CA14803F03EF85E
:10FB1000A04803F03BF862799F4BA04803EB8203B7
:10FB2000D3F8DC11F8F760FF9D48F8F75DFF264633
:10FB30000027D6F814800021404604F0A1FB20B134
:10FB40009848F8F751FF002669E039469648D6F8FC
:10FB500018B0D6F81CA0D6F82090F8F745FF40461C
:10FB6000002104F097FB10B1202003F007F806A94C
:10FB70004046F8F7BFFD01468C48F8F735FF584678
:10FB8000002104F087FB10B1202002F0F7FF06A946
:10FB90005846F8F7AFFD01468448F8F725FF504670
:10FBA000002104F077FB10B1202002F0E7FF06A946
:10FBB0005046F8F79FFD01467C48F8F715FF484688
:10FBC000002104F067FB10B1202002F0D7FF06A946
:10FBD0004846F8F78FFD013701467548F8F704FFEE
:10FBE0000C2F06F11006A4D1AAE749B294F8D4204C
:10FBF00094F8D530009194F8D7106E48019194F99B
:10FC0000D8100734029194F9D210039194F8D310CC
:10FC1000049131460136F8F7E7FE102E03D094F830
:10FC2000D6100029E1D100260E2777430024624A2E
:10FC30000123926CA3403A44D2F80A20134240F0C8
:10FC4000948001340E2CF2D10136082EECD15B48A1
:10FC500002F09CFF4D4B5A4C9F6854F8041F19B199
:10FC60005848F8F7C1FEF8E70E46574B53F82640C0
:10FC70004CB10123B3403B4203D054482146F8F72E
:10FC8000B3FE0136F1E7524802F080FF21463F4BB8
:10FC90000AAA0B4493F88A3113444E4A8A5C013114
:10FCA000082903F8102CF2D1002306A94A488DF840
:10FCB0002030F8F799FE494802F068FF4848F8F705
:10FCC0005FF9484802F062FF4548F7F735FE4648BD
:10FCD00002F05CFF4248FFF783FE4448F8F784FED9
:10FCE0004020FFF7FFFB424802F050FF3C48F8F786
:10FCF000E9F9AA0726D53F4802F048FF3E4802F03E
:10FD000045FF374802F08CFD3C4802F03FFF344885
:10FD1000F7F796FD3A4802F039FF3148F8F782F8D4
:10FD20003848F8F761FE2E48F7F712FF364802F020
:10FD30002DFF2B48FFF728FC2C48F8F755FE8020B4
:10FD4000FFF7D0FB6B0716D5304802F01FFF304895
:10FD500002F01CFF224802F03DFD2448F8F744FE63
:10FD60004FF48070FFF7BEFB05E03146224629487C
:10FD7000F8F73AFE65E70BB0BDE8F08FA3C90108BC
:10FD800017CE0108AAC90108B0C90108F02900204E
:10FD9000BEC90108D0C9010818AB0108DCC90108B7
:10FDA000E7C90108F4C9010801CA010815C801081A
:10FDB000CCD0010809CA01088C24002028CA0108F7
:10FDC0005CAD010838CA010860AD010846CA0108E7
:10FDD00053CA010862DC01085FCA010868CA010849
:10FDE00007C3010877CA010883CA010828D201089D
:10FDF00091CA01089ECA0108B1CA0108BFCA010818
:10FE0000C9CA0108D8CA0108E6CA0108F2CA01082D
:10FE100003CB010815CB01082DE9F84F2E4E0446FF
:10FE200037683846F8F782FE05463846F8F70BFE85
:10FE3000766880463046F8F779FE83463046F8F714
:10FE400002FED4F8049006462946484604F084F899
:10FE5000A76882464146384604F07EF8014650467F
:10FE600003F070FF21688246584604F075F8414659
:10FE70000446484604F070F8314604F06DF8014637
:10FE8000204603F061FF31460446384604F064F82A
:10FE9000294604F061F80146204603F055FF01466B
:10FEA000504607F085FE0D4904F056F80C4904F061
:10FEB00007F90C4B196803F047FF0B4904F000F9F0
:10FEC00007F09EFD83B21A0444BF00F5B47083B2FC
:10FED00018B2BDE8F88F00BFD82400200000E1442C
:10FEE000DB0F4940FC120020000020412DE9F04FBB
:10FEF00089B00593A24B80461B880492980737D59A
:10FF000040F2E632129B9F48DC89B0F900301B1B9F
:10FF100003F2F315954203D8002BB8BF5B4201E012
:10FF20004FF4FA73B0F9022040F2E630121B02F2ED
:10FF3000F314844203D8002AB8BF524201E04FF4C0
:10FF4000FA729342B8BF13460522C3F5FA7393FBC6
:10FF5000F2F30A22643B534398F81C20D210534317
:10FF6000642293FBF2F3134423EAE373DBB200E071
:10FF70006423C1460193CB1C03930024039B022CF2
:10FF800013F8016F804F03934FEA440A05D1B7F984
:10FF900004301B365E4376114AE07C4B37F914205F
:10FFA00033F9143003EB4202049B5B429A4203DBB9
:10FFB000049B9342A8BF1346754A32F90A50059A2A
:10FFC0005B1B32F9145003EB050B03F073FC88B193
:10FFD000704A5846155D03F06BFF6F4904F070F8E6
:10FFE0000146284603F03EF86B4903F0B5FF04F0E4
:10FFF00079F98346624A1288D10714D437F90A5036
:020000040801F1
:100000001B366E4393074FEA261611D598F8125007
:100010009DF9042005FB0BF35343642293FBF2F399
:1000200006EB231604E098F8085005FB0BF52E119B
:100030005A4B042533F90A30594F93FBF5F5751BDC
:1000400099F8016007F108036E43E35C98F851B03A
:100050005E430293642396FBF3F6F611BBF1000FA7
:100060001CD0022C30460CD103F022FF5FEA5B0368
:1000700004D05B45A8BF5B461A4600E0012249490F
:1000800006E003F015FF5A4607F10C0101EBC4012D
:100090007B6AF8F769FA04F025F90646424B99F8AD
:1000A0000B7019883E4B01FB05F203F1280E5EF838
:1000B0002400D21207FB02073C4AB7F5001FA8BF75
:1000C0004FF40017974203F13400B8BF174650F8B9
:1000D000242040F824504FF6FF700909B0FBF1F1DD
:1000E000AA1A4A4303F1400103F14C054EF824706B
:1000F00051F824E055F8240045F824E098F85050D1
:10010000921170444FEA840C7F13104441F824206C
:100110008DB1CDF818C0079303F0CAFE079B2A469D
:1001200003F1580101EBC4015B6AF8F71DFA04F012
:10013000D9F8DDF818C099F81530F2195843029B28
:10014000013443431846642390FBF3F0184B00122C
:10015000024423F80A2003F108024CF80260032C41
:1001600003F1140203F120034CF802704CF8030071
:1001700009F101097FF402AF09B0BDE8F08F00BFBB
:1001800068110020CC29002084100020DA330020E0
:100190008829002048AF0108000020419C0F002062
:1001A000D8240020F4240020780F00200000E0FF75
:1001B000482500202DE9F04F9D4B91B05B68054626
:1001C0009C4898479C4B9B489C4E1A780146FEF7EA
:1001D0009FF933889A4C002B00F08680D4F89C302D
:1001E00004F1A0071B7804F1AC0A02934FF0000859
:1001F000B6F800904FEA4803B9F57A7F02BF0022B3
:100200003A60CAF810208B4A019332F918003A6814
:1002100002443A6003F04CFEDAF810200132012A61
:10022000CAF8102007D10022CAF80400CAF800005A
:10023000CAF808202EE0DAF8003005921946039338
:10024000049003F07FFD059A8346104603F030FECC
:100250000146584603F034FF039B0146184603F05D
:1002600073FD0246DDF810C01146CAF8040060466E
:10027000039203F067FD0146584603F06DFEDAF87D
:10028000081003F061FD039ACAF80C00CAF80020B8
:10029000CAF80800019B6749DFF8C0B10022B9F134
:1002A000010F5A5223F80B202AD1DAF81000012846
:1002B00008DD013803F0FCFD0146DAF80C0003F01C
:1002C000FFFE00E0002007F0FFFD029B73B10390EA
:1002D000184603F0EDFD039A0146104603F0F8FFBF
:1002E00020B14FF47A73338000231CE03A684FF456
:1002F0007A7102F5FA7292FBF1F2019B2BF803205E
:1003000008F10108B8F1030F07F104070AF1140A14
:100310007FF46EAFB9F1010F02D1484601F0B0FF92
:100320003388013BDFE7464E424906F1E80031F8E9
:10033000132030F81300121A21F813200133032B75
:10034000F1D1404B1B6813F0020300F00F833E4BCA
:1003500006F1EE005B6898473C4B06F1EE001A7818
:100360000146FEF7D5F8B6F8F43006F1EE07002B9B
:1003700042D0D6F8F8000023B4F8F4204FEA830CFA
:10038000B2F5C87F324A04BF002142F8231037F982
:1003900013E052F80C102A4E714442F80C10002160
:1003A00027F8131020F813100133032BE4D1B6F80B
:1003B000F430012B1BD1D6F8FC304FF4C87E03F18A
:1003C000C80292FBFEF20280D6F80021C83292FBEE
:1003D000FEF24280D6F804311E4AC83393FBFEF386
:1003E00012889B1A838029806980F8F72FFFB4F860
:1003F000F430013BA4F8F430174B1B685A0740F166
:100400009080B4F808210E4B322A29D1D3F8F82075
:100410001188A3F80A1151889288A3F80C11A3F847
:100420000E212A88A3F810216A88A3F8122119E066
:100430004C1200209C0F002060120020DE330020B0
:10044000D8240020A010002040120020E233002019
:10045000D42500201C00002090290020C025002069
:10046000002A3ED0D4F8F8000023B4F808214FEA5F
:10047000830E322AC24A04BF002142F8231037F902
:1004800013C052F80E10BF4E614442F80E10002205
:1004900027F8132020F813200133032B1146E4D151
:1004A000B6F80831012B17D10C2086F8202186F8E8
:1004B000213101F0E5FED6F8F830B6F80A211A80AD
:1004C000B6F80C215A80B6F80E219A80B6F8103191
:1004D0002B80B6F812316B80B4F80831013BA4F8D8
:1004E000083194F82231A74ADBB1D2F81431322610
:1004F00093FBF6F3D2F8F800002182F82211038072
:10050000D2F8183193FBF6F34380D2F81C319E4A9F
:1005100093FBF6F312889B1A838029806980F8F791
:1005200095FED4F8F820B4F8EE3011884FF00008AA
:100530005B1AA4F8EE305188B4F8F0305B1AA4F8D6
:10054000F0309288B4F8F2309B1AA4F8F23001F03F
:1005500039FED4F824610546831B1846019303F045
:10056000A3FCD4F82811029003F0F6FCC4F824513F
:100570004546D4F82C71854E97F800B00390844A14
:100580000DF11C0A32F9150003F092FC039903F0F7
:10059000E3FC4AF82500BBF1000F2BD0584603F0CE
:1005A00087FC01464FF07E5003F08AFD0246DFF8DB
:1005B000089211464FF07E50059203F0C3FB59F8A4
:1005C000251003F0C9FCA9F14201049031F915008E
:1005D00003F06EFC059A114603F0BEFCDDF810C076
:1005E0000146604603F0B0FB49F8250003F07AFEAF
:1005F000708003E0674A32F81520728036F9022FC6
:100600000135032D02FB0288B9D1642303FB08F8EE
:100610005D4B61481B8807A95B4398FBF3F8A8F181
:1006200049081FFA88F8F8F7FFFAB8F13B0F7D6820
:1006300010D9544BB3F94801D3F8445103F038FCB6
:100640000146284603F044FE544B68B31A7842F042
:1006500008022CE04FF07E51284603F075FB01465E
:100660004FF07E5003F02CFD81464FF00008DFF87C
:1006700028B128465BF8281003F06EFC484A039026
:1006800032F9180003F014FC039B0146184603F0EE
:100690005BFB494603F060FC4BF8280008F10108B9
:1006A000B8F1030FE3D1C4E71A7822F00802294613
:1006B000D4F840011A7007F07BFA81462060D4F824
:1006C0003C01D4F844B100F10045D4F840010146A2
:1006D00003F042FC59468046584603F03DFC014673
:1006E000404603F031FB07F0EFFB0146284607F0D8
:1006F0005FFA2C4980466060484603F02DFC07F005
:100700007FF9294D27492880404603F025FC07F052
:1007100077F9264B68801B681B074FD5244807A92B
:10072000F8F782FABD684FF07E51284603F00CFBC3
:1007300001464FF07E5003F0C3FC82464FF0000BA1
:100740001B4B284653F82B10049303F005FC194962
:10075000039031F91B0003F0ABFB039A01461046EE
:1007600003F0F2FA514603F0F7FB049B43F82B0029
:100770000BF1010BBBF1030FE2D1184655E000BFAE
:10078000EC250020D82400201C0000206C10002044
:100790009C0F0020C625002014260020A410002055
:1007A0006E1000204C3D0F4488290020A01000202E
:1007B00024260020A20F002008260020704D51465C
:1007C0002846F8F731FA28686B680146039303F06E
:1007D000C3FB039B82461946184603F0BDFB014646
:1007E000504603F0B1FAD5F808B08246594658464B
:1007F00003F0B2FB0146504603F0A6FA07F064FB93
:100800000021824603F03CFD70B92868514603F090
:1008100057FC51462860686803F052FC51466860F6
:10082000A86803F04DFCA8605548FFF7F5FA554B52
:1008300055491880029803F08FFB524B08F100488D
:10084000054609F10049B3F90000CDF82C80CDF838
:10085000289003F02DFB4D4900F1004003F07CFB94
:10086000DFF83C810C90B8F9000003F021FB0D90FB
:10087000B8F9020003F01CFB0E90B8F9040003F075
:1008800017FB0AA90F900DA8F8F7CEF97B78012B7A
:100890001AD13F4B3F4F1B7813F0040F0ED1D7F8FE
:1008A0005801402390FBF3F3C01A03F001FB0F99AA
:1008B00003F04AFA03F016FDC7F85801D7F85801BB
:1008C000402390FBF3F001E0334B188803F0F0FA7B
:1008D00001460F9803F036FAD4F860110F902846BD
:1008E00003F032FA0146284603F0EAFBD4F85C71C3
:1008F000054639460F9803F025FA0146284603F0CD
:100900002BFB0146384603F01FFA0746C4F85C018A
:100910000D9807F075F8D4F864512978F8F784F841
:10092000D4F868311844C4F868010E9807F068F8E4
:100930002978F8F779F8D4F86C311844C4F86C01C8
:10094000384607F05DF86978F8F76EF8D4F870313A
:10095000124A184401991368C4F870011944D4F874
:10096000743111600133C4F8743105E0A6F8EE303B
:10097000A6F8F030A6F8F23011B0BDE8F08F00BF55
:10098000400000207C100020BD37863535FA8E3CB3
:10099000E1330020D82400201C000020C4330020B4
:1009A0006E10002001380A4B042804D8DFE800F05C
:1009B0000507090B0D00074A08E0074A06E0074A49
:1009C00004E0074A02E0074A00E0074A1A6070475D
:1009D0005C00002065CD0008EDFE0008D938010854
:1009E0002FCA0008A5C60008F9C000080846F6F797
:1009F00029BA10B50D4C206801F06CFB206800226C
:100A0000047A02FB02F3193B634303F6C413534316
:100A1000192193FBF1F3064921F812300132072A1C
:100A2000EFD1BDE81040034901F00CBBE00F0020FE
:100A3000380F0020342B00200E4B1A78692A15D16C
:100A40005A88B2F5FC6F11D11A79BE2A0ED193F8EB
:100A5000DD270020EF2A0BD113F8012B5040064A66
:100A60009342F9D1B0FA80F04009704700207047F6
:100A7000704700BF00F80108E0FF01082DE9F04FC2
:100A8000D84C85B000214FF4FC62204606F0ABFD47
:100A9000D54B04F53B721A60D44B00251D70D44B26
:100AA00004F2B6721A60692323704FF48070032336
:100AB0006371F8F735F9202284F86A216E224FF429
:100AC000167384F87C210A22A4F8663184F87D210B
:100AD000FA232B22A4F8683184F87F21BC23212239
:100AE000A4F8643184F880214FF4FA732322A4F827
:100AF0006E3184F8812101234FF4C87284F8623189
:100B000084F87E31A4F8822184F8863100220523FE
:100B100084F8B457A4F87251A4F87051A4F8745131
:100B200084F8585184F8595184F85A51A4F85C510A
:100B3000A4F85E51A4F8605184F8635184F86B51B5
:100B400084F86C51A4F88451A4F8885184F81D529B
:100B500084F81C52C4F82022C4F8242284F82852B5
:100B600084F82B3240F2DC53A4F8983140F24C4325
:100B7000A4F89A3140F26C73A4F89C3140F27533BA
:100B8000A4F89E3140F643032946A4F8A031234639
:100B900084F8295284F82A5284F8925184F89351A7
:100BA00001925818023100251E2224298D4C80F80C
:100BB000A25180F8A321F4D140F27E41A4F844115F
:100BC00040F23A71A4F8461140F27E51A4F84C115B
:100BD00040F2EA5140F2DC50A4F84E1140F2B45118
:100BE0004FF4FA63A4F8C831A4F8CC31A4F8D0319A
:100BF000A4F8D431052384F8DE31DFF8EC91C82362
:100C000001274FF47A7A4FF0320B1926A4F8E2311B
:100C10004FF4C87384F895210292A4F8E631A4F841
:100C20004A010390A4F8501184F8DF6184F89451CC
:100C300084F89651A4F8C6A1A4F8CAA1A4F8CEA13C
:100C4000A4F8D2A184F8D65184F8DC5184F8DD717F
:100C500084F8E07184F8E17184F8E47184F8E85173
:100C600084F8EA71A4F848A1A4F852B1A4F8543168
:100C7000A4F856B184F8EB5184F8EC5184F8ED7186
:100C800084F8EE51F8F748FBD9F80030029A27743F
:100C9000E773A573A581DA721A735522DA700F22F1
:100CA0005A7122229A710E221A7435229A762122C2
:100CB0001721DE715A74642653224FF028085975A3
:100CC0009975DA762D210A224FF05A0E1E77782672
:100CD000597383F808E09A749E721D7083F801803E
:100CE00083F80280DD7583F804B09D731D76DD7393
:100CF0005D7683F8098019754FF4FA71A3F84E10E8
:100D00003C494FF07F5C9963D9633B49C3F820C0ED
:100D1000C3F824C0394EDFF8FCC083F85020996234
:100D2000039837490292019ADE621E63C3F848C0F5
:100D30004FF07E564FF04B0C1A6459649F7783F83E
:100D4000525083F851805E6383F84CC084F8B6E754
:100D5000A4F8C0074FF0410E042084F8B7E784F8E8
:100D6000B8B784F8B95784F8BD5784F8BE5784F8EB
:100D7000BA5784F8BB5784F8BC57A3F85850A3F867
:100D80005A50A3F8565083F85C001966152183F871
:100D900068101C491C48D9661C4983F8648019678F
:100DA0001B4983F86580596783F87870F8F7E0FA93
:100DB000D9F80030029A18464FF4487183F811515F
:100DC00083F8125183F8138183F8147183F8185152
:100DD000A3F8161184F8D821C82284F8D921A4F8E0
:100DE000DAA119E0F0290020B80F002048290020DE
:100DF000E00F00208FC2F53C00002040CDCCCC3E5F
:100E00000000A0409A99193F49D00108F6287C3F7C
:100E10003D0A773F000040400E2202FB05326FF092
:100E2000170482F81941032482F81A416FF02F0445
:100E300082F81B41072482F81C416FF0230482F8DA
:100E40001D41052482F81E4101355A2480F82041B5
:100E500080F821416422FF24082D80F81F2180F8AA
:100E600022414FF0000100F10E00D5D1C820A3F8B7
:100E70008A01142083F88C01A3F890211E204FF4DE
:100E8000967283F88D01A3F892210120282283F81D
:100E9000891183F88E01A3F894210B465C4D0199CA
:100EA0005A191033C02B5161F8D105F52B70002170
:100EB000402206F098FB0023564FEA18D959043314
:100EC0000868382B524CC2F8AC02F5D104F50B700F
:100ED0000021802206F087FB07F13801702204F51B
:100EE0000B7006F075FB012500F07EFA4FF000084C
:100EF000082084F8DC8784F8DA5784F8DB57F7F7A2
:100F00000FFF1020F7F70CFF4023A4F8FC31052356
:100F100084F893314FF47A73A4F844314FF4FA63B0
:100F2000A4F846314FF4FA43A4F85431D9F800300C
:100F30000322A4F80C8084F8925125741A7024229C
:100F40005A709A7084F8D981DFF8DC800227D8F8CB
:100F50000030822284F8D8711A7014225A711A71E2
:100F600064229A712C48F8F703FA2C4B2C492D4A2D
:100F70006661E661666226636663E66326646664AC
:100F800066656666A66626676667C4F88060C4F80C
:100F90008460C4F88860D9F800602362E362E36487
:100FA0002365A3652366A367C4F89030A161A1629D
:100FB000A263A264E165E166E267C4F88C20314671
:100FC00004F284404FF4CC7206F002FB04F21C6081
:100FD00031464FF4CC7206F0FBFAD8F800301A68AC
:100FE000C4F8C2275A68C4F8C6279A68C4F8CA2742
:100FF0001A68C4F8CE275A68C4F8D2279A6884F8C9
:10100000D854C4F8D62784F8707605B0BDE8F08FC0
:10101000F02900204CAF010852D00108000080BF29
:10102000240FD4BE240FD43EE00F0020074B93F8CA
:10103000DC37012B08D1064A064BD0681B68834277
:1010400034BF00200120704700207047F0290020A5
:101050000C000020C005002038B5094B93F8DC5780
:1010600065B9084C2068F7F797F9074B25601B789E
:10107000022B03D1BDE83840F8F70FB938BD00BFE7
:10108000F0290020D4310020D1310020064B93F804
:10109000DC371BB1012B05D1FAF7BCBF034B186835
:1010A00001F073B900207047F0290020D4310020EE
:1010B000F8B5011F06460023083051F8042F02F14D
:1010C00020043F2C3BD802F108040F2C06D8023232
:1010D000032A04D9002B08BF012300E00223814228
:1010E000EBD1012B30680ED0022B1AD0736800F0C0
:1010F000030003F003039B0043EA0010B36803F00E
:101100000303184317E000F00F0040F04000F5F72C
:1011100099FEB068736800F00F0040EA0310C0B297
:1011200009E000F03F0040F08000F5F78BFE3079D9
:10113000F5F788FE307ABDE8F840F5F783BE06F192
:101140000C0734463A46002552F8043DAD0003F141
:101150008001FF2910D903F50041B1F5803F02D28B
:1011600045F0010508E003F50003B3F1807F34BFCB
:1011700045F0020545F00305B242E5D165F03F00B8
:10118000C0B2F5F75FFE05F00303022B207807D00D
:10119000032B0CD0012B13D1F5F754FE60780FE030
:1011A000F5F750FE6078F5F74DFEA07808E0F5F70A
:1011B00049FE6078F5F746FEA078F5F743FEE07843
:1011C0000434F5F73FFEBC424FEAA505DBD1F8BD7C
:1011D00010B50446C0B2F5F735FEC4F30720BDE8EC
:1011E0001040F5F72FBE10B504467F2C06D964F0E9
:1011F0007F00C0B2F5F726FEE409F6E7E0B2BDE8ED
:101200001040F5F71FBE430083EAE070EBE72DE9DD
:10121000F047314B86B093F8DC370746012B01D0FD
:1012200004464AE006F023FA0546064603A9684646
:10123000FAF7FEFD039B049A029713442B443F2BBD
:10124000059519D90023684603A90322FAF71CFE65
:10125000039B3BB9049B2BB9204A13705370059B29
:10126000ABB301E0FAF7CCFD039B049A059E13444F
:1012700033447F2B2BD8029FDFF860903946CA4653
:101280001AF8024BC4F18008B04528BFB0460AEBFB
:1012900004004444E4B2424606F09AF9802C89F8EE
:1012A000004014D1C8EB0606504607EB0801324651
:1012B00006F08EF989F8006009E0254614F8011B54
:1012C00021B1074B186801F06CF8F6E7ED1B2846D2
:1012D00006B0BDE8F08700BFF029002050260020AE
:1012E000D43100200FB407B504AB53F8042B0549E3
:1012F00000200193F7F778FA03B05DF804EB04B02F
:10130000704700BFED09010810B54B88DC0641BFEE
:101310002F4B14791B6853F8244044BF2D4B43F8DE
:1013200020404B889B0641BF294B54791B6853F8DA
:10133000244044BF274B43F820404B881C070ED560
:10134000254B0C781B78B3EB141FA1BF204BD4782E
:101350001B6853F82440A4BF1E4B43F820404B8821
:101360009B070ED51D4B0C781B78B3EB141FDFBF0A
:10137000174B54781B6853F82440DCBF154B43F8D7
:1013800020404B88DC070FD5154C0B78247803F0F0
:101390000F03A342DFBF0E4B14781B6853F82440A1
:1013A000DCBF0C4B43F820404B885B070FD50B7814
:1013B0000C4903F00F0309788B42A1BF044B9278CC
:1013C0001B6853F82220A4BF024B43F8202010BD15
:1013D000D0240020220D0020BF180020BD180020BE
:1013E000BC180020BE180020254A0023F0B515685F
:1013F0001C461A462348244903700B702E19768820
:101400004EB92F5D3FB9037000230A704B70077807
:101410001C461A460CE0360548BF013204F10404AC
:1014200003F1010348BFD2B2802CDBB2E6D1EAE778
:10143000E0B2B8420CD215F82400013406099E42ED
:1014400000F00F00A8BF731C9042A8BF421CEFE73A
:101450008A704B70C2F3470102F001020A444C1E2D
:101460000A490B480A70C3F3470203F0010313440F
:1014700004700849501E084A08701370F0BD00BF80
:1014800074110020B4180020D4260020BE180020BB
:10149000BC180020BF180020BD180020924B2DE979
:1014A000F04FDA68914D1A612A6891B0DA60904A7B
:1014B0000295136843F0200313608E4B1A78012ABB
:1014C0000CBF002201221A708B4B1A78910740F151
:1014D0004D838A490978042940F24883884909786C
:1014E00001F0040101F0FF0011B922F001021A70AD
:1014F0001B78DB0702D408B1FAF70EFC8149CA78E1
:10150000531C052293FBF2F202EB82029A1A7E4BE5
:10151000CA701F7892000023DFF81082DFF8109263
:1015200058F82310794C91FBF9FE04F1080040F8BB
:1015300023E0774844F8231000FB0E1142F21070AC
:1015400091FBF0F004F1100680B226F813004FF082
:10155000140C04F114060CFB036C04F13C0A5AF859
:1015600023605CF802504CF80210761B31440526CB
:101570004AF8231091FBF6F109FB0E114434012FB8
:1015800044F823104FEA830B444605D10238B0F5E6
:10159000797F98BF4BF808100BB90123BCE7594E6F
:1015A000029BB2461868336DC01A02F07DFC59499F
:1015B00002F086FD029B4FF07E511B6807463365A3
:1015C00002F068FE08B94FF07E574B4BCAF85470D2
:1015D0001B78514E13F00103504D12D00DAA00920A
:1015E0004F4B0EAA01920CCB94E80300FAF7AAFA2B
:1015F0000D9A6421B2FBF1F20E9B328093FBF1F362
:1016000000E033802B809AF858303E4D002B35D0C7
:10161000696D4FF07E5002F053FD0746EB6D206878
:10162000C01A02F045FC394602F096FC02F05AFE60
:101630002B6E86B2606836B2C01A02F039FC394BA4
:10164000196802F089FC394602F086FC02F04AFE75
:10165000B5F9662000B28118B5F964200220B318EC
:1016600091FBF0F193FBF0F389B29BB2A5F86A10FD
:10167000A5F86830A5F86610A5F8643001238AF84B
:101680005830294B61681B88206803F030031D4ED9
:10169000264DCAF86010CAF85C00002B00F0668284
:1016A00006F17403009306F178030193F26E336F31
:1016B000FAF748FA6B68306FC01A02F0F9FB194B61
:1016C000196802F049FC02F00DFEF36E2A68C6F8B4
:1016D00080009B1AF3670C4B1B78012B2AD0022B3E
:1016E00000F0E68042E200BF1C070020B429002081
:1016F000A0100020E60F0020A4100020AA10002057
:10170000E1330020D4260020AC0E0020D826002093
:10171000806967FF00007A441E110020201100201C
:10172000E80F00204C00002068110020AC100020C1
:1017300080969800D6F88430D6F8A0400293D6F868
:10174000943004F100400393D6F89830776D0593F8
:1017500002F0C8FD8146204602F0C4FDD6F89C3058
:10176000BB4C0493BB4B06901B684FF0000B0793D8
:10177000B94E4FEA4B0356F82B80A6F114024046AF
:1017800032F81B50089302F093FB029902F0E4FB3D
:1017900002F0A8FD401B1FFA80FA283626F81BA08D
:1017A0000FFA8AFA504602F083FB039902F0D4FB49
:1017B00002F098FD86B20AEB080002F079FB059969
:1017C00002F0CAFB394602F0C7FB216802F0BCFAFE
:1017D00002F088FD484504DB069B9842A8BF1846E6
:1017E00000E0484602F064FB206002F07BFD079BAE
:1017F000304486B2987802F057FB984902F0ACFB6F
:1018000001464FF07E5002F05BFC394602F09CFA34
:101810000146384602F054FC09906068D4F808A0EC
:10182000C0EB080002F044FB394602F049FC514687
:1018300002F088FA099A0146104602F08DFB014633
:10184000504602F081FA3135ADB2622D0146206179
:10185000C4F80480A0600ED9049802F07DFB02F069
:1018600041FD7F4AB0F5FA6FA8BF4FF4FA6090428D
:10187000B8BF104600E0002040F6B832064436B249
:101880009642A8BF1646774A089B9642B8BF1646AE
:10189000754A54F8140B9E52142202FB0BF2734942
:1018A0005050BBF1000F40F061814FF0010B5FE73A
:1018B000684BB6F8A8401F68736F3D8902935B08B8
:1018C0009D4228BF1D4623B29D4202DC1FFA85F9C6
:1018D0000AE06749706D02F03FFB02F003FD20440F
:1018E0001FFA80F9A6F8A890DAF87860DAF8AC4028
:1018F000341B2046FAF768F941F293130028D8BF49
:1019000040429842CCBF0020012078B3204602F02C
:10191000CFFA584902F020FBF7F795F804460298F1
:1019200002F0C2FA0146204602F016FB02F0DAFC91
:1019300040F6B83380B2AAF8B00000B29842A8BF0F
:101940001846484B9842ACBF3018F01848F6A043F0
:10195000984203DDA0F50C40A03804E00028BCBF8D
:1019600000F50C40A030CAF8B40001E0CAF8B46039
:10197000DAF8B4300026C3F50C502830039302F097
:1019800097FA3C4902F0E8FA0446F7F7CFF80F90CF
:101990002046F7F758F8DAF8B830DAF8C44005937B
:1019A000DAF8BC300E9004F10040089302F09AFC83
:1019B0000490204602F096FCDAF8C030DAF8548041
:1019C0002A4C09900793730048460A9302F070FA74
:1019D0000EAB53F8261002F0BFFADFF8A0A00546C0
:1019E0003AF9160002F064FA0146284602F0AAF914
:1019F00002F078FC05B2204BB5F57A7FA8BF4FF412
:101A00007A759D42B8BF1D460AF13C0AA8B22AF871
:101A1000160000B202F04CFA0599824602F09CFAD8
:101A200002F060FC089983B25046069302F094FAE3
:101A3000414602F091FA216802F086F902F052FC68
:101A4000049B98421CDB099B9842A8BF184618E0EB
:101A5000E80E0020B00E002050270020DB0FC94008
:101A600030F8FFFF48F4FFFFBA0E0020100F0020EF
:101A70000000C842D302373918FCFFFF3C27002082
:101A8000049802F015FA20608346B87802F00CFA48
:101A9000384902F061FA01464FF07E5002F010FB27
:101AA000414602F051F90146404602F009FB0B9015
:101AB0006068D4F808A0281A02F0FAF9414602F04A
:101AC000FFFA514602F03EF9DDF82CC001466046AF
:101AD00002F042FA0146504602F036F965600146CE
:101AE0002061A060079802F037FA02F0FBFB069B2A
:101AF0001434034458469A4602F0F4FB40F6B832D8
:101B0000504400B29042A8BF10461B4A0A9B904224
:101B1000B8BF1046194A1A4998521422724342F823
:101B200001B00EB901264EE73B792BB1039A64232D
:101B300092FBF3F3134A13803B88029A124C9A42A9
:101B40000DD9D4F8AC30A06FC01AFAF73DF842F2C4
:101B5000107380EAE072A2EBE0729A4206DD0B4B52
:101B600001221A70B4F8C820064B1A8011B0BDE8E3
:101B7000F08F00BFDB0FC94048F4FFFFBA0E002012
:101B8000E80E0020A80E0020D4260020AC0E002075
:101B9000054A08B5138801339BB21380034B1878AC
:101BA000FDF7F0F9002008BD7A0F002088240020FE
:101BB0009148F0B50368914A9C8AA4B2E1B211F051
:101BC000010F2ED0198821F400610904090C198035
:101BD000198889B241F4806119800021117051780F
:101BE00099B1917811B9D178FF290ED10121917065
:101BF0001179022901BF198889B241F40061198065
